:020000022000DC
:10600000000004203D970500F39502002D94020046
:10601000F3950200F3950200F395020000000000E2
:10602000000000000000000000000000F3950200E6
:10603000F395020000000000F39502008DEF0200CE
:1060400011D80200F39502003504030005A20200F6
:1060500015A20200F3950200F1F80200F395020088
:10606000F395020061ED020051ED020041FB0200D8
:10607000F3950200F3950200F3950200F3950200F8
:10608000F395020051FB0200F3950200F395020024
:10609000F3950200F3950200411E0500F3950200FE
:1060A000F3950200F3950200F3950200F3950200C8
:1060B000F3950200F39502000000000000000000CC
:1060C000F3950200F3950200F395020071F70200C8
:1060D00061FB0200F3950200F3950200F153030007
:1060E0004504030011A40200F3950200C1E8020078
:0860F00000000000F39502001E
:1070000040F8044B40F8045B40F8046B40F8047B04
:1070100040F8048B40F8049B40F804AB40F804BBF4
:1070200040F804CB40F804DB6846704781F000412B
:1070300002E000BF83F0004330B54FEA41044FEA5D
:10704000430594EA050F08BF90EA020F1FBF54EAF8
:10705000000C55EA020C7FEA645C7FEA655C00F094
:10706000E2804FEA5454D4EB5555B8BF6D420CDD65
:107070002C4480EA020281EA030382EA000083EAE8
:10708000010180EA020281EA0303362D88BF30BD88
:1070900011F0004F4FEA01314FF4801C4CEA1131DE
:1070A00002D0404261EB410113F0004F4FEA03333D
:1070B0004CEA133302D0524263EB430394EA050FC8
:1070C00000F0A780A4F10104D5F1200E0DDB02FA37
:1070D0000EFC22FA05F2801841F1000103FA0EF2CB
:1070E000801843FA05F359410EE0A5F120050EF191
:1070F000200E012A03FA0EFC28BF4CF0020C43FAC2
:1071000005F3C01851EBE37101F0004507D54FF0CE
:10711000000EDCF1000C7EEB00006EEB0101B1F51E
:10712000801F1BD3B1F5001F0CD349085FEA300064
:107130004FEA3C0C04F101044FEA445212F5800F6F
:1071400080F09A80BCF1004F08BF5FEA500C50F10C
:10715000000041EB045141EA050130BD5FEA4C0CEF
:10716000404141EB0101013C28BFB1F5801FE9D24C
:1071700091F0000F04BF01460020B1FA81F308BF6F
:107180002033A3F10B03B3F120020CDA0C3208DD3B
:1071900002F1140CC2F10C0201FA0CF021FA02F116
:1071A0000CE002F11402D8BFC2F1200C01FA02F186
:1071B00020FA0CFCDCBF41EA0C019040E41AA2BFAB
:1071C00001EB0451294330BD6FEA04041F3C1CDA73
:1071D0000C340EDC04F11404C4F1200220FA04F093
:1071E00001FA02F340EA030021FA04F345EA03013D
:1071F00030BDC4F10C04C4F1200220FA02F001FAFF
:1072000004F340EA0300294630BD21FA04F0294680
:1072100030BD94F0000F83F4801306BF81F4801119
:107220000134013D4EE77FEA645C18BF7FEA655C8C
:1072300029D094EA050F08BF90EA020F05D054EA5E
:10724000000C04BF1946104630BD91EA030F1EBF63
:107250000021002030BD5FEA545C05D14000494167
:1072600028BF41F0004130BD14F580043CBF01F55A
:10727000801130BD01F0004545F0FE4141F4700140
:107280004FF0000030BD7FEA645C1ABF194610461B
:107290007FEA655C1CBF0B46024650EA013406BF1C
:1072A00052EA033591EA030F41F4002130BD00BFDB
:1072B00090F0000F04BF0021704730B54FF4806498
:1072C00004F132044FF000054FF0000150E700BF19
:1072D00090F0000F04BF0021704730B54FF4806478
:1072E00004F1320410F0004548BF40424FF0000165
:1072F0003EE700BF42004FEAE2014FEA31014FEAA8
:1073000002701FBF12F07F4393F07F4F81F06051F6
:10731000704732F07F4208BF704793F07F4F04BF41
:1073200041F40021704730B54FF4607401F000451E
:1073300021F000411CE700BF50EA010208BF70477E
:1073400030B54FF000050AE050EA010208BF70476F
:1073500030B511F0004502D5404261EB41014FF4D8
:10736000806404F132045FEA915C3FF4D8AE4FF0E0
:1073700003025FEADC0C18BF03325FEADC0C18BFC3
:10738000033202EBDC02C2F1200300FA03FC20FA14
:1073900002F001FA03FE40EA0E0021FA02F1144461
:1073A000BDE600BF4FEA4102B2F1E04324BFB3F5AE
:1073B000001CDCF1FE5C0DD901F0004C4FEAC0026C
:1073C0004CEA5070B2F1004F40EB830008BF20F050
:1073D0000100704711F0804F21D113F13872BCBF0A
:1073E00001F00040704741F480114FEA5252C2F15F
:1073F0001802C2F1200C10FA0CF320FA02F018BFA8
:1074000040F001004FEAC1234FEAD32303FA0CFCFA
:1074100040EA0C0023FA02F34FEA4303CCE77FEA89
:10742000625307D150EA01331EBF4FF0FE4040F4D3
:107430004000704701F0004040F0FE4040F4000082
:10744000704700BF024B1A6912681A61704700BF8B
:10745000804E0120C460056146618761C0F81C80D0
:10746000C0F82090C0F824A0C0F828B0C0F82CD0F4
:1074700080ED0C8B80ED0E9B80ED10ABC0F808E02A
:1074800009F0B6BA2DE9F0412A4C00250326D4F8BC
:10749000EC700021013143189A0803F00303BA5C31
:1074A0005B0042FA03F303F00303022BF2D0D4F89B
:1074B000F83009018A0803EB001089B300EB82025F
:1074C0000368190729D1D4F8F810994225D8D4F8BF
:1074D000FC709F4221D95B1A48BF0F331B11D4F8AF
:1074E000ECE04FEA930C03F003011EF80C80490016
:1074F00048FA01F707F00307012F0ED106FA01F150
:1075000041EA080104EB85083F2D0EF80C109ABFE4
:107510000135C8F80831C4F8047104309042CFD165
:107520002DB1013D04EB8503D3F80801AFE7BDE8B9
:10753000F08100BF804E01202DE9F0473B4CD4E99B
:107540003E120023C0E90233C0E90433521AC0E9F5
:1075500000231D4683619C461F4619461A469A46DB
:1075600099469E46D4F8EC6016F80A304FEA49096D
:1075700043FA09F303F00303012B4DD0022B47D04C
:10758000002B3ED0D4F8F0600132B2EB860F4FEA08
:1075900086080FD0D4F8EC604FEA920A02F0030993
:1075A00016F80A304FEA4906334113F0030301D0BD
:1075B000012BD7D1012911D0022902BF466901361A
:1075C000466186698E4238BF816190450FD0012B9C
:1075D00026D04FEA920A02F00309C3E70669013692
:1075E000066186698E4238BF81619045EFD177454B
:1075F00000D9C7602D014FEA0C13C0E90153BDE863
:10760000F0870CF1010CC0F808C001371946B9E742
:10761000013545600131B5E7013545601946B1E7EF
:10762000BE4501D2C760BE460027D2E7804E01208A
:1076300050F8310010B1043818BF01207047000025
:10764000054B5B695A68824204D8801A043053F8AB
:10765000200070471B68F5E7804E0120014441F28D
:107660000553884204D3D8B2012838BF012070479F
:1076700010F8012B03EB43135340F2E708B5FFF773
:10768000DFFF023008BD08B5FFF7DAFF43780B6073
:10769000023008BD43688B422CBF591A002141605B
:1076A000704700002DE9F74F89469DF830101746C6
:1076B0000D9A11F0DF0F0646A2EB07023DD03029EC
:1076C00025490CA813BF804688464FF0100A4FF09A
:1076D000010A13F0800535D002EBD2746510A2EBDD
:1076E0006404002D35DDAB46DA45524673683068D8
:1076F000A8BF5A46414601929847019AABEB020B4C
:10770000BBF1000FF0DC2FB1736830683A46494690
:1077100098473D44002C0CDD2544A2455746A8BFA0
:107720002746736830683A464146E41B9847002C68
:10773000F3DC284603B0BDE8F08FDFF820804FF07F
:10774000100AC6E713F0010401D11546C9E7144633
:10775000D9E70025D7E700BF618406005084060002
:107760002DE9F04389B006460020119D9DF8488020
:10777000139F8DF80F000AB381421ADA2D228DF87B
:107780000F204942109A08ACA2F10A000DF110092D
:10779000B1FBF3FC03FB1C12092A8CBF1218303218
:1077A00004F8012D4C458E4661460ED07345EFD945
:1077B0000BE0A80727D52B228DF80F200029E1D157
:1077C00030238DF81F300DF11F0415F040099DF88E
:1077D0000F301CD023B30122CDE900822B460DF1DE
:1077E0000F013046FFF75EFF013F814608AACDE951
:1077F00000872B46121B21463046FFF753FF4844B3
:1078000009B0BDE8F0836A07D8D52022D4E7002B61
:10781000ECD004AA9442E9D904F8013C013CE5E724
:107820009946E3E790F9001003780029024601DB4E
:107830001846704703F07F004023184206D112F823
:10784000013F03F0C001802904D0704720EA030003
:107850005B08F2E703F03F0343EA8010EFE7431CC5
:1078600018460133027802F0C002802AF8D070472F
:1078700001440346002099421A4600D87047127806
:1078800002F0C002802A03F1010318BF0130F2E7C1
:107890007F289DBF024B185CC0F34000002070475A
:1078A000740D06007F289DBF024B185CC0F3C0001A
:1078B00000207047740D06007F289DBF024B185CA6
:1078C000C0F3800000207047740D06007F289DBF24
:1078D000024B185CC0F3001000207047740D0600C6
:1078E0007F289DBF024B185CC0F3401000207047FA
:1078F000740D060008B50246FFF7E8FF00B120321C
:10790000104608BD08B50246FFF7EAFF00B1203A6D
:10791000104608BD10B501440246E52400209142FE
:1079200003D8B0FA80F0400915E012F8013B20B10D
:107930001B0611D5431ED8B2F1E7BF2B09D9F72B8F
:1079400009D8DB0803F0060344FA03F303F003004D
:10795000E5E71B06E3D510BD0020FCE702398142B4
:107960000B4603D20233181A401070471A880239A6
:10797000002AF4D0F6E7B2EB131F70B54FEA1314E8
:1079800015D9121B03F00F0301EB440115460E46F7
:10799000012D31F8024B18BF3468DC40A4B2013D20
:1079A00020F8024BF3D104B9013A104670BD002211
:1079B000FBE7F0B5059F0024D21B2646A74210D155
:1079C00000EB470C01EB47010024A24214D10CEB61
:1079D00042031EB101212CF812100233181A401074
:1079E000F0BD31F8145033F814C06544354420F824
:1079F00014502E0C0134E1E731F8145035442CF8C2
:107A000014502E0C0134E0E7F0B4049F0025D21B83
:107A10002C46AF420BD100EB470601EB4705002394
:107A20009A420FD106EB4201F0BCFFF797BF31F845
:107A30001560344433F81560A41B20F81540241455
:107A40000135E6E735F813100C4426F813402414EA
:107A50000133E5E710B500EB410002EB410209B943
:107A6000084610BD30F8023D32F8024D1B1B002BBA
:107A700002DB04D10139F2E74FF0FF30F1E70120DA
:107A8000EFE710B5D0E90121034601EB42020020E7
:107A9000914204D31B78DB0748BF404210BD32F847
:107AA000024D44EA0040F3E72DE9F04371B19F181D
:107AB000D0E901940025A4F102084FF0010EAC4674
:107AC0001A44B9F1000F03D1BDE8F0831F46EFE778
:107AD00038F8024F0CF1100C44EA0545BCF1070FD1
:107AE00002DC09F1FF39ECE70678ACB2F60742BFD9
:107AF000E4435EFA84FE1FFA8EF4E4B248BFCEF38C
:107B0000072E49B17E1E07F8014CB342DCD0ACF120
:107B1000080C2D0A3746E1E73E4606F8014B96422F
:107B2000F4E70000D0E901329FED0C0A9FED0C7ADA
:107B300002EB43039A4205D30378DB0748BFB1EE5B
:107B4000400A704733F8021D07EE901AF8EEE77A04
:107B5000E0EE077AB0EE670AECE700BF0000000035
:107B600000008047D0E9023293423DBF5A1C826038
:107B700018784FF0FF3070470369272B1DD0222B58
:107B80001BD0752B03D023F01002622A10D142695A
:107B9000272A12D0222A10D0722B09D1622A0ED1A4
:107BA0008069272809D0A0F1220358425841704724
:107BB000622B04D14369722BF1E70120704700204A
:107BC000704710B502690A2A044622D1C3690133FD
:107BD000C3610123236263692361A3696361D4E9FB
:107BE000010398476369A0610D2B07D10A239842CE
:107BF000636103D1D4E901039847A061A36901330C
:107C000006D163695A1C03D00A2B1CBF0A23A36147
:107C100010BD036A092A04BF073323F007030133A9
:107C2000D8E770B504460D4600262269531C01D1E1
:107C3000304670BD0A2A08D115B1A36A002BF7D0CF
:107C40002046FFF7BEFF0126EFE71046FFF720FEB4
:107C500018B12046FFF7B5FFE7E7232A08D12046F1
:107C6000FFF7AFFF23695A1CDFD00A2BF7D1DCE7FF
:107C70005C2ADDD163690A2BDAD12046FFF7A1FF28
:107C8000E7E7D0E90432013B036152F82300704773
:107C90000369C9431944436953F821007047DE283A
:107CA00007D010F0010306D043080CBF01200020CC
:107CB00070470120704718467047FE2807D010F023
:107CC000010306D0430814BF0120002070470120A3
:107CD000704718467047000010F0010204D040F0D1
:107CE0000100086001207047A8B110F003030FD114
:107CF0000279372A0ED183680B6013F00100F1D1AD
:107D00009A0708D11868044BC31A58425841704763
:107D10001046704718467047B47B060010B50368DC
:107D200013B91360184610BD9C0702D010600120E3
:107D3000F9E71C798C42F9D103F108011160586808
:107D4000000AF0E730B5058D04460022954201D8BF
:107D5000002030BDE36A03EBC20043688B42F8D0D9
:107D60000132F3E7838B426A01339BB28383918CA8
:107D7000994238BF93847047F7B51E4659B111F048
:107D8000030511D14F68FCB294420DD13F0A01F1B5
:107D90000804BD4201DB03B0F0BD54F8041B0190A0
:107DA0000135B0470198F4E7334603B0BDE8F04031
:107DB00018470000024B89689722FFF7DDBF00BF1C
:107DC0000D510400024B89686722FFF7D5BF00BF41
:107DD00047FA040031B1026801F00303134304BF02
:107DE0000B680360704770B504460D46104619468F
:107DF000FFF7A8FF037833B96D681A4620462B4673
:107E0000BDE870401847012BF6D02D684288022B40
:107E10002046AC4608BF0023BDE8704018BF0123D0
:107E2000604737B50DF105040B46214602F07F058A
:107E3000D20904F8015DF9D1091B984701AD01464B
:107E40002346AB4205D19DF804201B1BC25403B04E
:107E500030BD13F8012B62F07F0201F8012BF0E72F
:107E60004379026A032B88BF036B114494BF034616
:107E70009B1801621846704710B50C460121FFF7A8
:107E8000EFFF047010BD4279836A032A88BF426AFB
:107E9000194484BFD218036B816294BF03469B18B8
:107EA0001846704710B50C460121FFF7ECFF04702F
:107EB00010BD000013B504460192FFF7F3FF019ACD
:107EC0000349204602B0BDE81040FFF7AABF00BF3B
:107ED000877E020030B4C36815465C8B9A8B038F93
:107EE0001444C28E14445A1C02871A194379042B75
:107EF00004BFC36B43F8225030BCFFF7DBBF28330D
:107F0000D9B2FFF7D7BF38B50D4603211446FFF7A6
:107F1000BAFF4470240A0570847038BD38B54379BF
:107F2000032B81BF846AC369C4F1FF2404F57F0475
:107F300084BF53F82230FD340D464FF003018CBF4F
:107F4000E4180024FFF79FFF4470240A0570847032
:107F500038BD38B54379032B81BF846AC369C4F542
:107F6000FF4453F8223088BF7D340D464FF00301A3
:107F70008CBFE4180024FFF786FF447024120570BC
:107F8000847038BD4379012B09D083681944C368D4
:107F900081605A8C9142C8BF598400238371704715
:107FA00070B501211D4606461446FFF7EBFF45B9A3
:107FB0000F2C06D8A4F15001C9B2BDE87040FFF7FC
:107FC00071BF05F1190122463046C9B2BDE87040C3
:107FD000FFF770BF70B514460E461B340121FFF742
:107FE000D1FF3246E1B2BDE87040FFF78CBF70B5FB
:107FF0004FF0FF311D4606461446FFF7C3FF45B953
:108000000F2C06D8A4F14001C9B2BDE87040FFF7BB
:1080100049BF05F1220122463046C9B2BDE8704091
:10802000FFF748BF70B514460E4624344FF0FF31B9
:10803000FFF7A8FF3246E1B2BDE87040FFF763BF2B
:1080400070B514460E462A340021FFF79BFF3246D6
:10805000E1B2BDE87040FFF756BFF7B5DDE908763D
:10806000C91AD4B243EA07220546A1EB470101929F
:108070005EB10239FFF786FF611C019AC9B228463A
:1080800003B0BDE8F040FFF715BFFFF77BFF019A93
:108090002146F4E713B501910021FFF773FF019A20
:1080A0001D2102B0BDE81040FFF72DBF10B54FF005
:1080B000FF31FFF767FFBDE810402121FFF7F2BE57
:1080C00038B50D460021FFF75DFF4379012B05D040
:1080D000032B9EBFC369826A43F8252038BD13B5C0
:1080E00001910121FFF74EFF019A162102B0BDE870
:1080F0001040FFF708BF10B50121FFF743FFBDE8AF
:1081000010401821FFF7CEBE10B50121FFF73AFF4E
:10811000BDE810403021FFF7C5BE10B54FF0FF316C
:10812000FFF730FFBDE810403221FFF7BBBE10B5AE
:108130000021FFF727FFBDE810403321FFF7B2BE53
:1081400010B50021FFF71EFFBDE810403421FFF7F6
:10815000A9BE13B501910021FFF714FF019A352143
:1081600002B0BDE81040FFF7F4BE10B54FF0FF318C
:10817000FFF708FFBDE810404121FFF793BE38B577
:108180000C1E14BF03210021FFF7FCFE002C18BFBA
:108190004721BDE8384008BF4221FFF783BE10B534
:1081A0000021FFF7EFFEBDE810404421FFF77ABE43
:1081B000302937B50C461AD031291BD101250724A7
:1081C0004FF0FF310190FFF7DDFEA4F12901019886
:1081D000C9B2FFF767FE019875B10021FFF7D2FE23
:1081E0000198D32103B0BDE83040FFF75BBE012505
:1081F0000624E5E70025E3E703B030BD70B5032AA8
:108200000D46144614BFC5F1010101215034FFF79A
:10821000B9FE2A46E1B2BDE87040FFF74BBE10B58B
:108220006FF00101FFF7AEFEBDE810405421FFF7EB
:1082300039BE2DE9F74F05460C46904699461BB1CD
:108240000B7E43F008030B76A4F81E806B6A1B7844
:10825000002B4DD159EA0803A86A4CD10121FFF740
:1082600091FE6269602103B0BDE8F04FFFF732BEB6
:10827000DB6A03EBC70B13F83730033B012B1AD82B
:108280004FF0000A14E0E36A03EBCA0213F83A3035
:10829000042B0BD1DBF804105368994206D1BBF8CC
:1082A0000220A86A0023FFF77BFE01360AF1010ACB
:1082B000238D5345E7DC01376B6A1A8DBA42D7DC50
:1082C000002EC7D059EA0803A86AF5B21AD1C6F140
:1082D00001010190FFF756FE626962210198FFF7E4
:1082E000F9FD0198294603B0BDE8F04FFFF7DABD6C
:1082F00000273E46E0E74FF0FF31FFF743FE62699B
:108300006121B0E7F1430190FFF73CFE6269632110
:10831000E4E70000F8B504460E4611461A4600236D
:1083200085794769837143610D4BFFF725FDA3688C
:10833000A3B9E18A39B1A28A2AB9A06AFFF75EFF20
:10834000A06AFFF7D8FEA38AE28A31462046FFF7EB
:1083500070FF003D18BF0125A5716761F8BD00BF22
:108360005152040007B5CDE900230B4664220021D9
:10837000FFF773FE03B05DF804FB10B54FF0FF315B
:10838000FFF700FE0123BDE8104083715B21FFF77A
:1083900089BD38B50C464942FFF7F4FDC268137E2B
:1083A00043F0040304F15D011376BDE83840C9B21F
:1083B000FFF778BD2DE9F74F10EE104A002C9DF81D
:1083C0003050044624DAB4EE400AF1EE10FA1FD61B
:1083D0002D2504F8015BB1EE400A9FEDC47AF0EE62
:1083E000C07AF4EE477AF1EE10FA02F0200E14DDB6
:1083F0008EF0490323708EF046058EF04E036370B5
:10840000A570E31C00221A70181A03B0BDE8F08FA3
:10841000002DE2D004F8015BDFE7B4EE400AF1EE94
:1084200010FA08D74EF04E028EF0410522706570AA
:10843000E31CA270E6E7002B42F02002B8BF06233F
:10844000672A02D1002B08BF0123251A491B10EE11
:10845000105A002D01F1FF3748D1662A38D15D1C32
:10846000AF424FF00006D8BFCB1E591C6627B4465A
:108470003546652F23EAE37840F0098108F10101D0
:10848000002301934FF02E0BB2EE047A019B8B4236
:10849000C0F20681662A40F03381A94280F28681CB
:1084A00096B10A2195FBF1F301FB135593FBF1F211
:1084B00001FB12324EF0450E3032303584F800E0C8
:1084C0006670A270E570043400232370201A9CE7C4
:1084D0005D1DAF42D8BFCB1F652A17464FF0000184
:1084E00040F0CF802B268C460D46C2E7B5F17E5F6B
:1084F0006FD2DFED7F7ADFF80082DFF800A2B4EE02
:10850000E70AF1EE10FA4FF00006ACBF4FF0310968
:108510004FF030094FF0200C3546B8EC017AB4EE3C
:10852000C07AF1EE10FAC4BF0AEB060B9BED007A9D
:1085300006F10406C4BF654420EE070A182E4FEA70
:108540006C0CEAD110EE106AB6F17E5F27D2B4EE61
:10855000E70AF1EE10FA1DDB002D14BF2D262B26A5
:10856000B7EE000A662A03D0672A28D1042D26DC3C
:10857000672A04BF05F1FF369B195E1CB742D8BFBE
:10858000CB1E84F8009063B9013419461E464FF0A3
:10859000FF3C58E0F2EE047A20EE270A01352D2642
:1085A000E0E72E216170302619460234013D6AD081
:1085B00009B90E46EBE704F8016B0139F6E78F1FA6
:1085C000BB4202DB672A60D0CB1F174600218C46D6
:1085D0004FE70026DFF82481DFF81C914FF0200CD4
:1085E0003546F8EC017AF4EEC07AF1EE10FA9CBF51
:1085F00009EB060ADAED007A06F104069CBF654431
:1086000020EE270A182E4FEA6C0CEAD1FDEEC07A54
:1086100017EE906A092EC2BFDFED367A013520EEE3
:10862000270A662A11D1AF4217DD591901318F424D
:1086300005DC7F1B012FA7F1020308BF0023E91807
:108640000131AC460026662713E7652A05D0672A64
:108650000CD0174600212B26B9E78E1FB34200DB52
:10866000CB1F00212B268C46652702E71E1DB74233
:1086700000DC8B1F9D4201DB6727EBE7691C5B1A5F
:10868000DDE70E462FE72E4681E73B469DE7672F45
:108690007FF4F6AE002BDABF012188464146EFE6B3
:1086A000FDEEC07A04F1010A17EE903A002BA8BF44
:1086B00003F13009019BACBF5FFA89F94FF0300933
:1086C000634584F8009006D1B8F1000F03D004F19F
:1086D000020A84F801B0F8EEE77A019B30EE670AEF
:1086E000013320EE070A01935446CFE6FFFF7F7F58
:1086F000F8FF7F3FCDCCCC3D00480600184806006F
:10870000F1EE047AB4EEE70AF1EE10FA28DB611E0E
:108710004FF030090B782E2B8C4601F1FF31F9D048
:10872000A3F1300ABAF1090F2CD90CF1010C9CF815
:108730000030302B14D19CF801102E292FD1662F38
:108740002DD02D2E8CF800108CF8013025D1013D54
:1087500008BF2B2623469C4523D331238CF80030B9
:10876000672A7FF49DAEB8F1000F3FF499AE23461F
:108770001C46013B14F8012C302AF9D02E2A08BFE0
:108780001C468DE6392B03D001338CF80030CEE740
:10879000604581F80190BDD1C9E70135DAE70134C0
:1087A000D8E713F8011C03F80119D4E7F1EE047AB5
:1087B000B4EEE70AF1EE10FAA9DA71E600F003036D
:1087C000022B05D1034B0340981F18BF01207047AF
:1087D00000207047070080FF50F8210010B10438D6
:1087E00018BF01207047704708B5C307024608D478
:1087F000074B0340062B06D0FFF7E0FF28B91068AF
:1088000008BD0448FCE70448FAE70448F8E700BF5D
:10881000070080FFB47B0600387F06005C79060005
:1088200038B5816804460846FFF7DEFF4369054610
:1088300005209847E168B1EB600F0ADA49002B6A1E
:10884000A068042241F001019847E3680133E36026
:1088500038BD0020FCE708B5FFF7C6FFBDE80840BB
:10886000C088FEF70BBF7047044B0B60044BC1E997
:1088700001300023CB600846704700BF587D0600DA
:108880002188020013B504460192FFF7ADFFC36AC9
:108890003BB1019A20469847B0FA80F0400902B0F7
:1088A00010BD1846FBE7062806BF480040F001004F
:1088B00000207047042803D0052808D00020704706
:1088C0008A68054B0548002A08BF18467047886823
:1088D000400040F0010070476454060070540600E8
:1088E000074BC1E900300023C1E90233054B0268A0
:1088F0009A4202BF4368C3F317238B600846704750
:10890000F80C0600687C0600136870B56BB9446803
:10891000A51C50F825509C4207D055F82360B14261
:1089200004D1023350F82330136070BD0133F2E7F5
:1089300013685BB940F2F123994208D1436823F0F0
:10894000030343F00203A3F1FF431360704740F2B7
:1089500043239942FAD18368F1E70000044B0B608E
:10896000037A0B7143688B600023CB600846704725
:108970006C300600044B0B6001230B7100238860F0
:10898000CB600846704700BF6C30060038B585687C
:108990000B6802460C46AB4201D3002009E01946A1
:1089A000D068FEF745FE591C20B12160D06800EB6D
:1089B000C30038BD0B46EEE7042803D0052809D0D4
:1089C000002070474B68074833F00F03064B08BF81
:1089D000184670474868C0F31B10400040F0010083
:1089E000704700BF705406006454060010B4C46899
:1089F0000023A4465DF8044B604700221146FFF7B0
:108A0000F5BF000038B504461546FFF7EDFE074BED
:108A1000C2689A4218BF2469A36813B90B602B601F
:108A200038BDE3880B60A368F9E700BF5D6603000B
:108A300001F1FF4323F0030307EE903A072805D81E
:108A4000DFE800F0051D04040704101800210846A3
:108A5000704710481049F5EE407AF1EE10FA08BF61
:108A60000146F4E7FDEEE77A17EE901A490041F06F
:108A70000101ECE7F5EEC07AF1EE10FAE7D5F1EE80
:108A8000677A17EE901A21F0030141F00201A1F17B
:108A9000FF41DCE76454060070540600C30706D5A6
:108AA000401000280DDB14BF0120002070478368B0
:108AB00053B1037913F0010F14BF4FF0FF300120C1
:108AC00070474FF0FF30704718467047174B984279
:108AD00010B502460C4623D0154B984223D0C1074F
:108AE00008D5431000EE103AB8EEC00A84ED000A33
:108AF000012010BD830707D101680E4B994203D1B5
:108B00000430FFF70FF8F1E71046FFF757FE002893
:108B1000EFD002F1FF4222F0030300EE103AE5E746
:108B20009FED050AE2E7B7EE000ADFE764540600AE
:108B300070540600B47B060000000000044B0B607C
:108B4000044BC1E901300023CB600846704700BFE9
:108B5000587D0600598B0200D0E9022391688B42B0
:108B60003BBFD26852F823200022013338BFC360D4
:108B700010467047004870476C5406004368184719
:108B8000C268002A05DDD0E90113994206DB002303
:108B90000AE0FCD0D0E901139942F8DD41684B00AE
:108BA0000A4443F0010342601846704710B5D0E90B
:108BB0000142C3680348C1E90223C1E90004084631
:108BC00010BD00BFB08C0600820708D10068064BBC
:108BD000984206D0054BC31A5842584170470020AE
:108BE00070470120704700BF487E06009879060054
:108BF000044B0B60044BC1E901300023CB600846F5
:108C0000704700BF587D06000D8C020038B58268A1
:108C1000C16855680346A94201D3002008E0D06826
:108C2000FFF7DAFD4C1C20B1DC60D36853F821005B
:108C300038BD2146EFE7000010F0030203D10168C0
:108C4000084B994209D010F0010306D13AB90068E7
:108C5000054BC31A584258417047012070471846C7
:108C6000704700BF8C760600B47B060010B5044642
:108C7000FFF7E2FF28B92046FFF7A0FD00F0010052
:108C800010BD0120FAE70000044B0B60044BC1E962
:108C900001300023CB600846704700BF587D0600B6
:108CA000F18C0200884230B513D20378303B092B97
:108CB0000FD8002313600A2510F8014B1368303CCD
:108CC00005FB03438142136003D00378303B092B3B
:108CD000F2D930BD054A0240062A02D1C008FEF78B
:108CE000D2BC82680A60C068704700BF070080FF7E
:108CF00013B5044601A98068FFF7ECFFE268019B09
:108D00009A423FBF835C5B0043F0010001322CBFFD
:108D10000020E26002B010BD73B50546084601A907
:108D2000FFF7D8FF019B064613B3134B9D4221D09A
:108D3000124B9D424FF0000405D1224613E0305DF6
:108D4000A847A8B10134019BA342F8D80C4802B04F
:108D500070BD315D0846FEF7A5FD18B10846A8476D
:108D6000024628B10134019BA342F2D8002AEDD17A
:108D70000448ECE70024E0E7CD780200E178020047
:108D8000705406006454060001460148FFF7C4BF52
:108D90009178020001460148FFF7BEBFA5780200A6
:108DA00001460148FFF7B8BFB97802000146014803
:108DB000FFF7B2BFCD78020001460148FFF7ACBF14
:108DC000E1780200012A13B50C460AD101A9FFF788
:108DD00081FF019B636042232060A360002002B0FA
:108DE00010BD0023C1E900334FF0FF338B60012039
:108DF000F5E70000044B0B60044BC1E90130002390
:108E0000CB600846704700BF587D0600150305007B
:108E100013B50446084601A9FFF75CFF042C04D0F3
:108E2000052C09D0002002B010BD019A0648074B5E
:108E3000002A08BF1846F6E70199FEF719FD400021
:108E400040F00100EFE700BF7054060064540600D4
:108E5000D0E9022351688B4237BF991C002252F897
:108E60002120013338BFC36010467047044B0B60AC
:108E7000044BC1E901300023CB600846704700BFB6
:108E8000587D0600518E0200F8B50E46114C12496D
:108E9000124B88421AD0C268A24203D0306001242B
:108EA0002046F8BD406B98B102689A42F1D14768FC
:108EB00000F1080505EB87070024BD42F0D255F804
:108EC000040B3146FFF7E0FF0444F6E70024E7E730
:108ED0000446E5E789BF0400E07C0600EC7F06005D
:108EE000F0B50C4685B054F8046B01920022039251
:108EF000054603A93068FFF7C7FF0398019BC768C1
:108F00002246691EB8473061014805B0F0BD00BF78
:108F10006C5406002DE9F041134E144F0D46A84243
:108F20001CD010F003031BD10268B2421AD1406B6F
:108F300090B10368BB42F2D1044654F8043F00EB01
:108F4000830000F1040854F8040FA045E7D929462E
:108F5000FFF7E0FF0028F6D0BDE8F0810120FBE735
:108F60000020F9E71846F7E728800600EC7F0600A6
:108F7000830707D10268064B9A4203D1C268054BAA
:108F80009A4202D00449FFF7C5BF0120704700BFD5
:108F9000288006005D660300D06E060008B5FFF766
:108FA00023FCBDE80840FFF7E3BF38B504460D4693
:108FB000FFF7F4FF18B12046FFF716FC04462946D8
:108FC0002046BDE83840FFF7A5BF70B504460D4602
:108FD000FFF70AFC0646FFF79DFF20B1AE4200D026
:108FE0002469204670BD0446FBE7000010B5044626
:108FF00008460A49FFF7E9FF042C03D0052C08D0E6
:10900000002010BD8268064B0648002A08BF18469B
:10901000F7E78068400040F00100F2E7F07B0600CF
:1090200064540600705406000C4970B5FFF7CDFF7C
:10903000836803EBD37149109B0000229142A3F196
:10904000040301DC064870BDC468E65854F8225099
:1090500044F82260C4680132E550EFE7F07B060077
:109060006C54060010B50446FFF7BEFB0422036AE9
:109070002046BDE81040184713B504460192FFF79B
:10908000B3FB019A036A204602B0BDE810401847BE
:1090900010B50446FFF7A8FB0022036A2046BDE88E
:1090A0001040184713B504460191FFF79DFB019A44
:1090B000836921462E2002B0BDE81040184710B544
:1090C00004460846FFF790FB006B18B10388A342E3
:1090D00018BF002010BD014640F2D920FFF7EFBFB6
:1090E0002DE9F0471E4681468A461546FFF7F3FFF5
:1090F0009DF82070D0E9018317F0020F4FF00004B3
:1091000018BF9846346007F001076DB133462A4610
:1091100051464846C04738B1431C08D133680B2B31
:1091200002D10CB1002333602046BDE8F0871FB99F
:1091300082442D1A0444E8E70446F5E7014BD86859
:10914000704700BF804E0120014B9868704700BFF8
:10915000804E0120024B0348002283F80A22704708
:10916000804E01206C540600024B0348012283F814
:109170000A227047804E01206C540600044B054AB9
:1091800093F80A02044B002814BF10461846704793
:10919000804E0120705406006454060000B589B06A
:1091A00001A8FEF7C9F90398400040F0010009B09A
:1091B0005DF804FB00B589B001A8FEF7BDF902987F
:1091C000400040F0010009B05DF804FB034A044888
:1091D000B2F80832013BA2F808327047804E0120F5
:1091E0006C540600034A0448B2F808320133A2F86E
:1091F00008327047804E01206C54060010B502689A
:10920000002312F8011B01F07F04090644EAC3138E
:10921000F7D40260184610BD0138013910F8012F4B
:1092200011F8013F8AB163B97F2A07D80B4B9B5CC9
:1092300013F00C0F0FD15F3A53425341C3F10103B6
:1092400006E09A42EAD000207047B3FA83F35B0944
:1092500003F0010070470123F0E700BF740D060022
:10926000002813DD002908DD6FF0404393FBF1F186
:109270008142ACBF0020012070474FF0404393FB78
:10928000F0F08842D4BF002001207047002905DD9E
:109290004FF0404393FBF1F18142F3E70028EBD01C
:1092A0006FF0404393FBF0F0E2E7782820D86D2878
:1092B00007D8622817D0662817D0612808BF072072
:1092C0007047A0F16E030A2B12D8DFE803F01011EB
:1092D00011110611111108110A000D2070470B2001
:1092E00070475C207047082070470C2070470A20A8
:1092F00070471FB58388C2889A42044610D3172B43
:1093000015D90123009300F1080103AB006818226E
:10931000FFF7E6FE039B80B2A08043B938B1E3803B
:10932000E088431CE3800444207A04B010BD4FF071
:10933000FF30FAE7BFF34F8F0549064BCA6802F4C6
:10934000E0621343CB60BFF34F8F00BFFDE700BF68
:1093500000ED00E00400FA0508B5074B1B78012B6F
:1093600002D9012800D0FEE7044B43EA0020044B59
:109370001860FFF7DFFF00BF76490120AF0000ADA6
:1093800060510120F8B5284DB5F80832002B47D1BF
:10939000002845D0D5F8F810002942D0411A48BF1E
:1093A0000F314FEA211CD5F8F4004FEADC010CF034
:1093B0000704435C0122A24023EA020343544FEA1C
:1093C0009C06D5F8EC40A05D374661460CF00303DF
:1093D0004FF0030E5B000EFA03F320EA0303E3559C
:1093E0000131D5F8EC408F0801F00303E05D5A002D
:1093F00040FA02F202F00302022AEBD0A1EB0C01C8
:10940000082928BF0821813105EB81014B68B3424F
:10941000D5F82C3288BF4E60B34238BFC5F82C62F5
:10942000F8BD0820FFF798FF804E012008B5022004
:10943000FFF792FF08B50120FFF78EFF2DE9F04FEF
:1094400000228578DFF8A4C0DFF8A4E007241646E0
:109450001746038803F1FF38424505DB0B440846F5
:1094600003F8017CBDE8F08F4FF00009CA46C846FA
:109470004B465B0015F0800F08F1010818BF43F060
:1094800001035FFA88F884B9741CE6B250FA84F4D8
:10949000A5780724BAF1000F01D053450AD31CF870
:1094A00008B00BEB4A0AD944E3E76D00013CEDB28A
:1094B000E4B2EFE74B44A3EB0A0301EB02081EF80A
:1094C00003307F2B04DC8B5401231A4492B2C0E793
:1094D0004FEAA31903F03F0363F07F0369F03F09EC
:1094E00001F8029088F801300223EEE7E84A06000E
:1094F0002ACE0600034B1B68DB0700D500BE002008
:10950000704700BFF0ED00E0084B03EB411310B4CF
:109510001C691CB95DF8044BFFF7ECBF5969044B9B
:109520001961234611465DF8044B184750010600A7
:10953000D42E01200120704708B50B7803F060039A
:10954000202B0FD1084B8A88187890420AD14A788C
:10955000202A05D1054A1AB1991D0020AFF30080D9
:10956000012000E0002008BD2426012000000000AA
:10957000024B1B68DB0700D500BE7047F0ED00E032
:10958000002070474DDF70474EDF70474FDF704758
:1095900050DF704712DF704748B9064BD3F8D80048
:1095A00030B10346C0680028FBD19868704700209E
:1095B000704700BF804E0120012808B50BD8FFF787
:1095C000EBFF38B1836943B1808800F03000203868
:1095D00018BF012008BD0020FCE71846FAE7807A92
:1095E000400040F001007047C07A400040F00100A8
:1095F0007047FEE761DF70474BDF704730B5084AC0
:1096000052F8D03F3BB19C6884421C6804D15D682D
:109610008D4201D1146030BD1A462346F2E700BFE7
:10962000804E0120B1DF7047B2DF704730B5124D78
:1096300004460020E8B14378FF2B18D0C3880333D9
:1096400023F0030308331844A84210D84378002BB2
:10965000F0D043788B42EDD1FF2907D0037803F097
:109660000103A342E6D143889342E3D130BD0020F9
:10967000FCE70248EDE700BFFB1F0F0004A00E004F
:1096800042884378007843EA022340EA0320704787
:109690000B0A017043700B0C090E8370C170704788
:1096A000036A0239023B8B4283BFC389406B01FBD3
:1096B000030000207047836A02680433D289490A94
:1096C000B1FBF2F1186830B1814202D3091A0833B4
:1096D000F8E758680844704700F10B010022D301F5
:1096E00043EA520310F8012B52FA83F38842DAB2AC
:1096F000F5D110467047CA7E8B7E032843EA0223C9
:1097000001BF487D0A7D42EA002243EA024318462F
:109710007047C2F307238A76CB760378032B01BF09
:10972000120C0A75120A4A757047000010B50749F5
:10973000002331F8024B84429AB203D00133802BCC
:10974000F7D11A4602F18000C0B210BD50000600E9
:1097500070B51E4B1E4AB0F5805F28BF1346191D19
:1097600031F8043C0A46ABB1984213D331F8024CAD
:10977000250AE6B253FA84F4A04221DA082D09D86A
:10978000DFE805F005090F11131517191B00C01AA2
:1097900031F8100070BDC31A03F00103C01A80B283
:1097A000F8E71038FBE72038F9E73038F7E71A38E0
:1097B000F5E70830F3E75038F1E7A0F5E350EEE7BE
:1097C0000431002DCCD102EB4603C8E7862B0600FE
:1097D000782D0600830705D16422B0FBF2F302FB6B
:1097E00013034BB94FF4C872B0FBF2F302FB130042
:1097F000B0FA80F04009704701207047084B4A1EBC
:1098000010B533F8114033F812300229A4EB0304E9
:1098100003D1FFF7DFFF00B10134204610BD00BFC8
:10982000402E06004B4BA0F59E00A0F5D05070B521
:1098300090FBF3F403FB14000028BCBF00F5A83034
:1098400004F1FF344FF03C02B8BF00F5C0704FF494
:109850006163B0FBF3F30B71B0FBF2F302FB130097
:10986000B3FBF2F502FB1535A31C072293FBF2F2C2
:10987000C2EBC2029B1A48BF0733002CB8BF04F5E5
:109880000E34CB71BABF04F2B1244FF0FF33002382
:10989000887148F6AC623048B4FBF2F2042A08BF83
:1098A000032200FB024440F2B5562C4894FBF6F626
:1098B000192E08BF182600FB06444D7140F26D15A5
:1098C00094FBF5F5042D08BF03256FF4B67000FB7B
:1098D00005409C00234402EB820203EB830302EB6E
:1098E00082021B0103EB820303EB86032B449BB232
:1098F00003F5FA621A4D0A80002215F9014B8442E1
:1099000024DDD2B2941CE4B20B2C8ABF0A3A8C70CC
:109910008A708A78134C02F10102D2B202F1FF354B
:1099200088BF03F2D17300F1010034F8154088BFFD
:109930000B80C3B2022A0888CB708A701C4403D9FA
:10994000FFF748FF00B101340C8170BD001B0132EC
:10995000D3E700BF805101005471FFFF4BFAFFFFB6
:10996000342E0600402E0600002910B514680CDACB
:1099700021440368002BBCBF1B19036003688B42A2
:10998000D4BFC91A0021116010BDA14228BF2146D1
:10999000EFE701291DBF16224FF0FF301A600020AB
:1099A00070470000004870476C540600064B1B6867
:1099B000082B06D1054B1B68032B02D8044AD05C48
:1099C00070470020704700BF3001001034010010C4
:1099D00028FF050041DF704729DF704728DF704707
:1099E00007B500230DF107008DF80730FFF7D2FD12
:1099F0009DF80700003818BF012003B05DF804FB94
:109A000010B5FFF7EDFF054C18B9207004E0FFF723
:109A1000E1FF2378012BFAD0207810BD39510120C5
:109A2000074B10B501241C70FFF7D6FF28B9FFF7CC
:109A3000E7FF023818BF012010BD0020FCE700BF7F
:109A400039510120F0B508B3204E00213346354688
:109A5000984204D00131082903F10803F8D11C4AC7
:109A6000046817684368BC4223F00303234415D1FC
:109A70004C1C05EBC10513600021072C02DC55F8D6
:109A8000086F26B101B1136000230360F0BD69685F
:109A900021F003010B4401340121EEE70D4A176860
:109AA0009F42F1D105EBC10314600021B34202D003
:109AB00053F8085D1DB10029E6D01460E4E7596849
:109AC00021F00301641A0121F0E700BF7446012070
:109AD000884A01209C4A012010B5084C206858B1E2
:109AE000FFF7B0FF064B93F85010002262F3C3015A
:109AF000226083F850105A6210BD00BF50510120FF
:109B0000F42201202DE9F0431A4B1B4CD3F800C07E
:109B1000D4F800E0AEEB0C0282420646994611DB17
:109B200082070FD1154F00290BBF01204FF0FF30E6
:109B300000230723B84657F833207AB11D18EBB23B
:109B4000072BF8D9002007E0AEEB020247F83320DC
:109B5000226008EBC3035E60BDE8F08307EBC3003F
:109B600026F003020029EFD1624447F833C0C9F858
:109B70000020EEE79C4A0120884A0120744601201B
:109B8000054B064A1B681068834203D00021C01AA7
:109B9000FFF7B8BF002070479C4A0120884A012087
:109BA000064B1868082802D104331B6823B9A0F1BA
:109BB0000D03584258417047012070473001001092
:109BC00042DF704743DF704744DF704707B5FFF758
:109BD00007FF48B101A8FFF7F7FF0198003818BF49
:109BE000012003B05DF804FB4FF08043D3F80C0470
:109BF00000F00110A0F1011358425841F1E70000B4
:109C00004309012200F01F0002FA00F02033024A4B
:109C100042F82300704700BF00E100E00028ACBF1D
:109C200000F16040064B4FEA4111B4BF00F00F0055
:109C300000F56140C9B2B4BF195480F800137047F1
:109C400014ED00E003681F2B83BF03F01F030360C4
:109C500001484FF0A04070470003005007B5019045
:109C600001A8FFF7EFFF019B03F5E073032240F823
:109C7000232003B05DF804FB07B5019001A8FFF7AE
:109C8000E1FF019B03F5E073022240F8232003B0BB
:109C90005DF804FB07B5019001A8FFF7D3FF019A17
:109CA00001239340C0F8083503B05DF804FB07B505
:109CB000019001A8FFF7C6FF019A01239340C0F865
:109CC0000C3503B05DF804FB10B5014690F8200098
:109CD000FF2805D08B7F1BB9CB7F5BB1FFF7E7FF78
:109CE000002308464B770B72BDE8104050F8083B44
:109CF00049681847FFF7CEFFF2E7000038B504794E
:109D00001D4924236343CA180546127F92B3CB58DA
:109D100023B1006840F30730FFF772FF2423634349
:109D2000CA18CB582D687BB1144BC5F80833537F44
:109D300053B101236B61D5F80431002BFBD02423F0
:109D400003FB041300225A77242303FB041393F824
:109D50002100FF2801D0FFF78FFF0023C5F8003551
:109D6000074B9D4204BF01225A60242303FB0411C8
:109D700000230B7738BD00BFD04C012052010800F2
:109D800000F002400023435082B043580193019BEE
:109D900002B070470B7B032B2DD8DFE803F0252999
:109DA0001D028A68154B9A4204D1D0F84C350A69D5
:109DB0009A4209D18A6840F202239A421BD1D0F814
:109DC0004C354A699A4216D000230622C0F8003565
:109DD000C0F8002518467047D0F84C350A699A42F9
:109DE000F2D1D0F83C35ECE7D0F84C350A69E9E718
:109DF000D0F83C35FAE70120704700BF00020400AC
:109E00002DE9F8439846002380F82E30D36803F0FC
:109E10006043B3F1005F06460C46154603D0824FFF
:109E20003846BDE8F883814BC1F8083390F82F30ED
:109E300003F0FF0923B183687D4FC1F80433EFE7D6
:109E4000012380F82F30944600F10C07BCE80F0086
:109E50000FC7DCF800303B6086F830906B78C4F8B0
:109E600088354FF482712046FFF78CFF4FF49271D2
:109E7000FFF788FFC4F85095C4F840952B78032B62
:109E800000F2B180DFE803F07A9C5E022B6903F0F8
:109E90006043B3F1005FC2D14FF48073C4F8003265
:109EA0006B68EA68C4F844254FF4A871C4F84835D3
:109EB000FFF768FF4FF4B071FFF764FF4FF4A47130
:109EC000FFF760FF01232362A360D4F85031002B19
:109ED000FBD04FF4A8712046FFF754FFAB682A6906
:109EE000C4F84425C4F84835524BB3604FF482732C
:109EF0000822514F297803291CBF0121A150326843
:109F0000002A75D1012223441968002974D0D4F89D
:109F1000C434C4F8C434002286F82F20002B79D032
:109F2000464A474F13F0010F18BF174613F0020FB0
:109F300002F1010218BF174613F0040F414B18BF7E
:109F40001F466DE76B68EA68C4F84425C4F84835D5
:109F50002B6903F06042B2F1005F7FF460AFAA6842
:109F6000C4F834354FF48453C4F83825C4F80032AB
:109F700040F20223B36001232362B7E76B68EA680B
:109F8000C4F84425C4F84835B8F1000F0ED04FF49A
:109F90008073C4F80032274BB3604FF4A471FFF70D
:109FA000F1FE4FF4A47301222262A1E74FF4007383
:109FB000C4F8003240F20223B3604FF48273F2E738
:109FC0006B68EA68C4F83425C4F838354FF4805318
:109FD000C4F8003240F20223B3600123236200225E
:109FE0004FF4827385E7184F4FF48273082281E79C
:109FF000B368C4F8043313E7D4F82411002983D0DC
:10A000004FF492712046FFF7BDFE4FF48273226237
:10A01000626178E731462046FFF7BCFE084B002816
:10A0200008BF1F46FCE600BF0A00AD0B02029C0100
:10A030000B00AD0B000204000000AD0B0000AE0BE6
:10A040000100AD0B0200AE0B0400AD0BF0B5D0F873
:10A05000243187B004460D46ABB14FF49271FFF73F
:10A0600091FED0F8043173B9AB68C0F8083302230D
:10A07000AB60AB68C0F8043301230362436185F829
:10A080002E3007B0F0BDD4F804316BB34FF48271B9
:10A09000204605F10C07FFF775FE0FCF01AE0FC686
:10A0A0003B68336095F82E303BB929462046FFF7D0
:10A0B00071FE80F0010085F82E004FF4B07120464B
:10A0C000FFF760FE4FF4AE71FFF75CFE95F830309D
:10A0D00013B195F82E30CBB10023C4F80032AB6039
:10A0E000224BC4F8083311E04FF4A4712046FFF767
:10A0F00049FE2B7BEBB905F10C070FCF01AE0FC664
:10A100003B68336095F83030002BE6D0D4F8C43487
:10A11000C4F8C4349A071ED501238DF8003095F891
:10A1200030300BB985F82F30D5E9003168469847B3
:10A13000A7E74FF40073C4F8003240F20223AB608B
:10A1400003F1CE73C4F80833AB68C4F804330123B9
:10A15000A360236295E713F0050F01D00223DCE72B
:10A1600095F82E30002BD8D00423D6E702029C01AC
:10A1700003790B490268342000FB031309490020CE
:10A180009860C2F80813D2F8001221F4BC51C2F84A
:10A190000012C2F80005012283F82D20704700BF8D
:10A1A000304D012002029C0170B50679144D342314
:10A1B0007343EA18044692F82D20FAB1EB5823B104
:10A1C000006840F30730FFF71BFD2046FFF7D0FF84
:10A1D000342303FB065393F832304BB92368D3F88A
:10A1E0000805FFF749FD2368D3F80C05FFF744FD88
:10A1F000342303FB0655002385F82D3070BD00BFC6
:10A20000304D012001490248FFF720BF304D0120A9
:10A210000030004002494FF04020FFF717BF00BF59
:10A22000644D01200023435082B043580193019BA9
:10A2300002B070471FB50123CDE901218DF8003030
:10A24000D0E900136846984705B05DF804FB0000AC
:10A250002DE9F0412F4E0579242303FB05630446C5
:10A2600093F82020002A52D05B6843B103682A4A41
:10A27000C3F80823006840F30730FFF7C1FC2268E9
:10A28000D2F8003223F02003C2F800322368012202
:10A290005A6020684FF4AC71FFF7C4FF2368DA609E
:10A2A0002368D3F85821002AFBD00022C3F80025E8
:10A2B00023684FF0FF32D3F80C05D3F81485D3F898
:10A2C0000815D3F81075C3F80C25C3F814252368B6
:10A2D0009042C3F80825C3F8102501D0FFF7CCFC45
:10A2E000B8F1FF3F02D04046FFF7C6FC7A1C02D00F
:10A2F0003846FFF7C1FC4B1C02D00846FFF7BCFCF8
:10A30000242303FB0565002385F820306B60BDE83E
:10A31000F08100BF984D01201003420007B5019065
:10A3200001A8FFF78FFC019B00EB8300D0F80037FA
:10A3300023F4403343EA0141C0F8001703B05DF84D
:10A3400004FB07B5019001A8FFF77CFC019BD0F846
:10A350001005D84000F0010003B05DF804FB0000D8
:10A36000054B4FF0FF32072843F8202084BFC01868
:10A3700080F84C20704700BFE04D01200E4B034495
:10A3800093F92420072A02DD0021FFF7C7BFD3B2CB
:10A39000072B10D8930003F1804303F5C043D3F893
:10A3A000101521F00101C3F81015012303FA02F280
:10A3B000024BC3F808237047E04D012000600040C5
:10A3C00010B50E4A537903F0FF01A3B90C4B196085
:10A3D000116821B1012454710A4AC2F8044300F102
:10A3E000804000F524300122026011B91A68002A69
:10A3F000FCD0054800E0054810BD00BF484E0120D4
:10A4000000910240009002400000AD0B0B00AD0B2C
:10A41000054A136833B1054B0020587110601A6863
:10A4200099681047704700BF00910240484E0120D4
:10A430006DDF704772DF704773DF704774DF7047FE
:10A4400075DF704778DF70477ADF70477BDF7047D2
:10A450007CDF70477DDF70478ADF70478BDF704796
:10A460008CDF70478FDF704790DF7047A5DF704744
:10A4700060DF704769DF704767DF704710DF704744
:10A4800011DF70470388102B03D01B2B03D0002053
:10A49000704783880B8001208870704708B50A20B8
:10A4A000FEF75AFF21290DD005D811290AD012290B
:10A4B00008D039B17047312904D0412902D022296E
:10A4C00000D0704701707047A3DF7047ABDF704763
:10A4D000ADDF7047AEDF704770B5EFF3108672B630
:10A4E0000D4A94680123A4B993600C4B0C4DD3F82A
:10A4F000801029401160C3F88050D3F88410516057
:10A500004FF0FF32C3F88420047006B962B6002011
:10A5100070BD0370F9E700BFD050012000E100E0FA
:10A52000FC06FFBDC38802899A420BD05A1C92B226
:10A530000168C280CB5C818891429CBF0022C280AE
:10A54000184670474FF0FF30704710B50289848875
:10A55000531C9C4298BF0023C4889C421DBF0468C2
:10A56000A15403814FF0FF3018BF002010BDC288F6
:10A57000038982B09B1A0193019B002BBFBF019AF4
:10A5800083889B180193019880B202B07047000045
:10A5900010B5084B9A685AB150B9EFF3108172B6F2
:10A5A000054A1C6814605C685460986001B962B622
:10A5B000002010BDD050012000E100E0F7B50446B6
:10A5C0000DF107000F461646FFF786FF00250C34F5
:10A5D000AE4205D89DF80700FFF7DAFF03B0F0BDE3
:10A5E000795D2046FFF7B1FF0135F1E7034610B56D
:10A5F0001A88392A08460DD0502A1AD14A68D988B3
:10A60000928A914204D11A8A03F11201FFF7D6FF10
:10A6100001200FE01C7B012CFAD14A685989928AEB
:10A62000914204D1DA8903F11001FFF7C7FF2046F8
:10A6300000E0002010BD00004368014613B102484D
:10A64000FEF7DCBF704700BFEDA5020076DF704764
:10A650007EDF70477FDF704786DF70479BDF704784
:10A660009DDF70479EDF7047B5DF7047406878B167
:10A67000406868B1837953B1C06848B1406838B167
:10A6800000884FF6FF73C01A18BF012070470120E1
:10A69000704718B143680BB1188870474FF6FF70C8
:10A6A0007047A4DF704770B505460C468E18B4425B
:10A6B00000D170BD21782846FFF747FF002806DA51
:10A6C0002846FFF72FFF21782846FFF73EFF013489
:10A6D000EDE770B506460C468D18AC4200D170BD52
:10A6E0003046FFF71FFF04F8010BF6E7F0B5838B48
:10A6F000002187B0044680F82310002B3CD062680C
:10A7000094F82250978A94F82020C08B94F8216006
:10A710000432F5B104EB8202CDF8091052688DF8CD
:10A720000D1002A98DF80860ADF80A70ADF80E3072
:10A730000492FFF7C9FE50B994F82030A08301338A
:10A7400003F0010384F82030012384F8233007B09C
:10A75000F0BD04EB8202ADF806300DF10603049360
:10A7600002A95368ADF808708DF80A60ADF80C5076
:10A770000593FFF7AFFEDEE71846E8E7F0B585B0D2
:10A780008389ADF8062002329A4205460E4620D84B
:10A790000DF10D00FFF7A0FE05F108042046A98980
:10A7A000FFF7E5FEBDF80630081A023398424FF075
:10A7B000020210DB0DF106012046FFF774FF204670
:10A7C0009DF806203146FFF76EFF9DF80D00FFF75C
:10A7D000DFFE05B0F0BD0DF10E012046FFF779FF59
:10A7E0000027BDF80E20BBB29A42D7D92046FFF70A
:10A7F00099FE0137F5E738B50446CD8BA3889D4215
:10A80000084606D12388392B05D023F00403382BC2
:10A8100015D0002005E04B6862899B8A9A4201D0DE
:10A82000012038BDE28904F11001FFF7A7FF237B67
:10A83000022BF5D161892846FFF733FFF0E7FFF7D8
:10A8400055FFEDE738B5034608461A88502A03D06D
:10A85000572A24D0002038BD4468D988A58A9A8810
:10A860008D420FD1C18B4FF6FF74A14207D1C28335
:10A870001A8A03F11201FFF781FF0120EBE79142F1
:10A88000E8D1F5E7648C8C42F7D1C48B4FF6FF71A9
:10A890008C42F2D15B8ADB07EFD5C283EDE7FFF78D
:10A8A00025FFD7E7A8DF7047AADF704762DF704750
:10A8B00064DF7047A1DF7047ACDF7047012070474D
:10A8C0001020704790F8203033B98268D2F8041114
:10A8D00011B18377C2F80431807F70470C4B9842E6
:10A8E00011D00AD8A3F57F43F73B98420DD001332E
:10A8F00098420CBF102000207047064B98420CBFB6
:10A90000052000207047132070470520704700BFC6
:10A910000100AE0B0200AE0BFF280CD04109064A25
:10A92000012300F01F0003FA00F052F8213023EA5F
:10A93000000342F8213070476C49012038B5074DBB
:10A940004368AB42044607D01879FFF795F963686E
:10A950001879FFF7E1FF656038BD00BF6C54060051
:10A9600070B50E4B0122002604465A60C3F80065FC
:10A97000FF2590F82100FFF7CFFF94F8220084F81C
:10A980002150FFF7C9FF94F8230084F82250FFF705
:10A99000C3FF034B84F823501E6070BD005002407B
:10A9A0008C4A012010B5837AFF2B04460ED04068F4
:10A9B000FFF7FAFBA07AFFF7AFFF607AFFF7ACFF73
:10A9C000FF23A3726372636800221A7210BD10B570
:10A9D000437AFF2B04460DD04068FFF78FF9607A69
:10A9E000FFF79AFFA07AFFF797FFE07ABDE81040E3
:10A9F000FFF792BF10BD10B504464068FFF728FC72
:10AA0000607FFFF789FFA07FFFF786FFFF23637753
:10AA1000A3772069FEF7B6FC00236361238310BD92
:10AA20004109064A012300F01F0003FA00F052F822
:10AA30002130184342F82100704700BFBC5001206C
:10AA400003790649580903F01F020123934051F886
:10AA50002020134341F82030704700BF6C4901208B
:10AA60004CDF704720B1034B800143F001031847CE
:10AA7000704700BF602F060010B5094C2046FEF756
:10AA800089FD237823B1BDE810400648FFF724BDB7
:10AA900072B6BFF35F8F044A13680133136010BDB1
:10AAA0003A510120904A0120B450012010B5124BB8
:10AAB0001B788BB1114B9A686AB1114A127852B95E
:10AAC000EFF3108072B60F491C680C605C684C6034
:10AAD0009A6000B962B610BD0B4B1A6812B9022019
:10AAE000FEF73AFC1A68013A1A601B68002BF2D193
:10AAF000BFF35F8FEEE700BF3A510120D050012035
:10AB0000904A012000E100E0B450012038B5FFF781
:10AB1000B3FF044BD3E90045FFF7C8FF20462946A1
:10AB200038BD00BF4851012030DF704731DF70472A
:10AB3000184B53F820300022022110B5C3F800252D
:10AB4000C3F80425C3F810154FF4FA41C3F81425CF
:10AB5000C3F80C25C3F808150F4901EBC004C3F86E
:10AB600020450424C3F82445C3F82825C3F82C2520
:10AB7000C3F84025C3F84425C3F84825C3F84C253D
:10AB80004FF4004321F8303001EBC0004380838054
:10AB9000C38010BD5C8C0600F050012001F5AC7143
:10ABA0004FF0FF3340F82130002303F5AC7250F82A
:10ABB0002220013205D10133042BF6D10023C0F845
:10ABC0000035704710B5436804467BB1007AFFF743
:10ABD00053F8617A60680023636001F07F01FFF73A
:10ABE000DDFF207AFFF798FEFF23237210BD30B5FA
:10ABF00043684181D3F82055447AD3F8082504F0FE
:10AC00007F0451434FF6FF73B1FBF3F36FEA434305
:10AC10006FEA534325F81430436801229A6030BD2F
:10AC20002DE9F84F002516469DF828B004460F463A
:10AC30002A469A46002B7CD04949A946012347F66B
:10AC4000FB70B1FBF3F8B8FBFAF8A8F1040C8445EB
:10AC500068D8DFF814C100215CF8040BD0F8003587
:10AC600013F00F036FD0BBF1000F67D1D0F8083598
:10AC7000984563D1D0F80C354B455FD15B4603F561
:10AC8000AC7E50F82EE0BEF1FF3F54D15AB2012500
:10AC90006060002861D0637A62F3060363723B79D7
:10ACA00023723846FFF7CCFE637A207AC4F80CA0F2
:10ACB0006BF3C7136372FEF7D1FF63680022C3F81A
:10ACC0000025DDB96368274A93420CD002F5A04203
:10ACD00093423BD002F58052934239D002F5304284
:10ACE000934237D10325E8B2FFF722FF63680022C1
:10ACF000C3F80C95C3F80425C3F80885637A626825
:10AD0000397903F07F0303F5AC73204642F8231032
:10AD100063680122C3F800253146FFF768FF002071
:10AD2000BDE8F88F09F10109B9F1080F4FEA4303B3
:10AD300087D10220F4E70133042BA0D1013104298B
:10AD40008AD10020A4E71A461D46A1E70125CAE7DB
:10AD50000225C8E74FF0FF35C5E70420E0E700BF54
:10AD60000024F40000C001405C8C060003685B68AE
:10AD70004FF0FF32C3F860250368187AFEF797BFDB
:10AD800010B5174B53F82020FAB11079FFF7D9FA14
:10AD9000C1B250794C00FFF7D4FAE4B24140937944
:10ADA00054FA81F1C9B2CB1A03F00303012B0DD180
:10ADB000D3790133D37192F907309171032B0ADDF6
:10ADC0009368013393600023D37110BD032BF2D13C
:10ADD000D379013BEEE70333F7DA9368013BF1E700
:10ADE0006C440120052801BF024A136803F50013D3
:10ADF00013607047345101201FB5134BD3F804057D
:10AE0000124B1B6801A903EBD000FEF70BFD9DF868
:10AE100007309DF806001B0443EA40539DF80800E4
:10AE200043EAC0239DF8090043EA40139DF80A0055
:10AE300043EA5003BDF80400A0F2BC7043EA40604E
:10AE400005B05DF804FB00BF004002403451012012
:10AE5000807D400040F00100704700008068024B98
:10AE6000002808BF184670476C54060008B5FFF765
:10AE7000E3FB014808BD00BF6C54060043683BB1CA
:10AE800093F85A200348044B022A08BF184670471B
:10AE90000048704764540600705406008068024BF6
:10AEA000002808BF184670476C5406004068704779
:10AEB00008B54368014613B10248FEF79FFB0248FC
:10AEC00008BD00BFF7A702006C5406008079034A52
:10AED000034B002814BF10461846704770540600F4
:10AEE00064540600C079034A034B002814BF10467F
:10AEF0001846704770540600645406008068024B80
:10AF0000002808BF184670476C540600C30747BFA7
:10AF1000401007EE900A00F1FF4020F003034CBF01
:10AF2000F8EEE77A07EE903A9FED337AF4EEC77ABF
:10AF3000F1EE10FA82B00EDDDFED306A67EEA66A40
:10AF4000FCEEE66A16EE903A1B0206EE903AF8EE38
:10AF5000666A77EEE67ADFED2A5AF4EEE57AF1EEEC
:10AF600010FAF0EE086A13D567EEA67A37EE677A24
:10AF7000FCEEE77ABCEEC77A8DED017A9DF80430DD
:10AF8000CDED017A9DF80400000440EA03201AE0A8
:10AF90009FED1C6AF4EEC67AF1EE10FA18D577EE42
:10AFA000E57A67EEA67A37EE677AFCEEE77ABCEED2
:10AFB000C77A8DED017A9DF80430CDED017A9DF8C8
:10AFC000040040EA0340400040F0010002B0704736
:10AFD00077EEC67A67EEA67AFCEEE76A77EE677AD6
:10AFE000CDED016AFCEEE77A9DF80430CDED017AF3
:10AFF0009DF80400C9E700BF00007F430000803BCC
:10B000000000AA4200002A4308B5FFF797FC014858
:10B0100008BD00BF6C54060008B50868FFF78EFC39
:10B02000004808BD6C54060008B5086890F8233045
:10B03000FF2B01D0FFF794FC004808BD6C540600BC
:10B0400038B5084B0C681B680025C3F800552079FB
:10B05000FFF762FC60792571FFF75EFC65710248BD
:10B0600038BD00BF442201206C54060008B5FFF72C
:10B0700099FC014808BD00BF6C54060008B508687B
:10B08000FFF790FC004808BD6C54060008B5FFF7B8
:10B090009EFC014808BD00BF6C54060008B5086856
:10B0A000FFF795FC004808BD6C54060008B5086819
:10B0B000837FFF2B01D0FFF79EFC014808BD00BF36
:10B0C0006C540600064BD3F8B83093F8250093F87B
:10B0D00024204000D2B283F8252040F001007047C0
:10B0E000804E0120F0B5134D3124013C14F0FF04D3
:10B0F00011D1114D3124013C14F0FF0419D02E461A
:10B100006F68B84205F10805F5D140F28F2008605C
:10B1100040F2C32109E02E466F68874205F1080519
:10B12000E3D1002008604FF4C77111603268D20883
:10B130001A60F0BD10240600804D060008B5FFF728
:10B14000B5FC014808BD00BF6C54060008B5FFF708
:10B1500093FC014808BD00BF6C54060000487047CE
:10B16000F083060008B50868FFF72CFD004808BD0D
:10B170006C54060008B5FFF725FD014808BD00BF67
:10B180006C540600024BC3F8B4000248704700BF7D
:10B19000804E01206C540600024B034800221A70B6
:10B1A000704700BFB84601206C54060008B5FFF791
:10B1B000ADFC07EE901AB8EE677A07EE900ADFED65
:10B1C000096AF8EE677AE7EE267A9FED077AC7EE0E
:10B1D000877A17EE900A20F0030040F00200A0F1F9
:10B1E000FF4008BD0000804F00007A44806870472F
:10B1F000C06870470079034A034B002814BF10460B
:10B200001846704770540600645406004079034A9B
:10B21000034B002814BF10461846704770540600B0
:10B2200064540600F7B587689DF820609DF82440B7
:10B23000042F04D1857C15B1E40844F0E004456A8C
:10B2400079435DB1042F08BF077C0D4408BFEC555E
:10B25000477BEA55877BEB55C77BEE55056A29444A
:10B260008568042D11D1857C6DB907EE904A90ED6B
:10B27000067AF8EEE77A67EE877AFCEEE77ACDEDAC
:10B28000017A9DF80440057C4C5507EE902A90ED1C
:10B29000067A447BF8EEE77A67EE877AFCEEE77A87
:10B2A00017EE902A07EE903A0A55F8EEE77A90EDFD
:10B2B000067A827B67EE877AFCEEE77A17EE903AA1
:10B2C00007EE906A8B54F8EEE77A90ED067AC27B2F
:10B2D00067EE877AFCEEE77A17EE903A8B5403B06C
:10B2E000F0BD000000234360004870476C54060026
:10B2F00000697047007B7047807B7047704730B5AE
:10B30000039C85682560446849B1857BB2FBF5F1F3
:10B3100005FB1122017BD2B2C90802FB01441C606B
:10B32000002030BD10B501241470427B1A70029BBE
:10B3300082681A6001B1847B039B1C7010BD000001
:10B340000B68024800225A60DA6070476C540600AD
:10B35000806A7047807E704790F82400704710B56F
:10B3600000241470827E082A94BF002201221A70E1
:10B37000029B4FF400721A6021B190F82430039AB6
:10B38000137010BD0123FAE70023C0E9013301481F
:10B39000704700BF6C54060040697047C07C70471E
:10B3A000007C704710B500241470827C1A70029BD8
:10B3B000C2681A6019B1C37C039A137010BD0123CF
:10B3C000FAE7008B07EE900AFBEEE87A17EE900A98
:10B3D00020F0030040F00200A0F1FF4070470000A1
:10B3E0008068034A034B002814BF10461846704774
:10B3F0007054060064540600002210B5144690F8FC
:10B400002410D3B2994200D810BD00EB830301325F
:10B41000DB6A9C60F3E7406A704790F82D00704744
:10B4200010B50024147001221A70029B046A1C607B
:10B4300009B190F82D20039B1A7010BD10B50D4B6B
:10B4400082689A42044614D00430FFF777FA94F8E1
:10B4500020309A0703D504F10C00FFF76FFA94F837
:10B460002030DB0705D504F11400BDE81040FFF7DC
:10B4700065BA10BD6C54060008B50868FFF7DEFF1A
:10B48000004808BD6C54060008B5FFF7D7FF014817
:10B4900008BD00BF6C54060030B5838899422CDA91
:10B4A00000292ADBC3889A4227DA002A25DB838910
:10B4B00084685A43837BDD080FD1C57B41FA05F5CB
:10B4C0002A440569008C294001FB0333C3F12001A4
:10B4D00054F82230CB40184030BD012D04EB8202DD
:10B4E00001D1505CF8E7022D02D132F81100F3E7E8
:10B4F000042D02D152F82100EEE70020ECE7000015
:10B50000C1EB0141084480EA50310C4B9FED0C7AAD
:10B5100001FB01F04EF64D4202FB0030094B01FBEE
:10B52000003020F0004307EE903AFAEEE07A67EE42
:10B53000877AFCEEE77A17EE900A70471F07310111
:10B5400000007F430DDD0852C20CC0F3C403400964
:10B5500043EAC22300F4FC60184340BA80B270474B
:10B56000020C13235343C2B2FF213632B3FBF1F373
:10B57000B2FBF1F2C0F307201344B6225043B0FBF4
:10B58000F1F01844C0B27047C2B2030C934219469E
:10B5900010B538BF1146C0F30724A14238BF214679
:10B5A0009342184628BF1046A04294BF081A081BB1
:10B5B00010F0FF0010D0C9B28B420ED1A21AF023B6
:10B5C0002824624392FBF0F292FBF3F003FB10207D
:10B5D000002800DAF030C0B210BD8C4207D1D21A78
:10B5E00002EB40022823534393FBF0F0F0E78A423A
:10B5F00003D11A1B02EB8002F4E70020EBE7000006
:10B600000079034A034B002814BF104618467047C0
:10B61000705406006454060010B50446FFF776FA2D
:10B620002369226FC11A91429ABF9B18181A0020F1
:10B6300010BDC088400040F0010070478088400085
:10B6400040F0010070470000042806D0052806D10C
:10B650008868400040F001007047024870470020B1
:10B66000704700BF7054060090F95030816A30B5C1
:10B67000002BB4BFB0F91240B0F91040B0F90C3053
:10B68000858923449CB28B7BC3B191F905204B88FB
:10B6900012FB05F21A4412B2A0F8462091F90530C7
:10B6A000498813FB04F30B441BB29A42D2BFA0F8A3
:10B6B0004A30A0F84A20A0F8463030BD91F9042065
:10B6C0000B8812FB05F21A4412B2A0F8442091F93B
:10B6D0000430098813FB04F30B441BB29A42D2BF17
:10B6E000A0F84830A0F84820A0F84430E5E790F9E9
:10B6F0005030816A30B5002BB4BFB0F91040B0F9BA
:10B700001240B0F90E30C58923449CB28B7BC3B183
:10B7100091F904200B8812FB05F21A4412B2A0F82A
:10B72000442091F90430098813FB04F30B441BB245
:10B730009A42D2BFA0F84830A0F84820A0F8443080
:10B7400030BD91F905204B8812FB05F21A4412B264
:10B75000A0F8462091F90530498813FB04F30B4407
:10B760001BB29A42D2BFA0F84A30A0F84A20A0F8F3
:10B770004630E5E72DE9F04190F82E309A0704466F
:10B7800022D4BDE8F081636853F83500830710D1F7
:10B790000368B34212D190F85030C0F8288023F0EB
:10B7A000140343F0140380F85030FFF75DFFFFF7F8
:10B7B0009EFF0135638D9D42E5D3E2E7BB42F8D1A0
:10B7C000414600F00BF8F4E7024E034F002500F16C
:10B7D0000808EFE7883C0600643806000A1E90F867
:10B7E0002E3018BF012262F3410380F82E309B07F0
:10B7F00030B428D58C7BB0F92420B0F9263014B1B0
:10B8000014461A4623460C8891F9045005FB02425F
:10B8100002814A8891F9054004FB032343810B7997
:10B8200090F8282013FB02F303734B7913FB02F308
:10B8300043738B7B83750B7B03754B7B43758B79D4
:10B8400013FB02F3837330BCFFF794BFB1F90030F0
:10B85000B0F900209A42C8BF0380B1F90230B0F9B4
:10B8600002209A42C8BF4380B1F90430B0F90420E5
:10B870009A42B8BF8380B1F90630B0F906209A42E7
:10B88000B8BFC380704710B5B0F900301380B1F96C
:10B890000040A342B8BF23461380B0F90430938020
:10B8A000B1F90440A342A8BF2346B2F900409380F7
:10B8B0009C4218DAB0F902305380B1F90240A34239
:10B8C000B8BF23465380B0F90600D080B1F90630E6
:10B8D0009842A8BF1846B2F90230D0808342ACBF6C
:10B8E0000020012010BD0020FCE7028883889B1AFD
:10B8F000C2884088101A9BB280B2584370474FF4F8
:10B90000B473F0B591FBF3F505FB1311002501238A
:10B91000B0F84220066CB0F84040A0F844104562F0
:10B9200080F82A30058680F8325021B1B42920D120
:10B9300040F201130386002390F832C04363C363CF
:10B9400040F20113038590F8301090F8313025B2A1
:10B9500017B2BCF1000F16D00787458719B1828452
:10B96000FF2280F828201BB1C484FF2380F82930EF
:10B97000F0BDB1F5877F80F832300CBF80F83130F0
:10B9800080F83030D7E7866319B1FF21848480F8CE
:10B990002810002BECD0C284E7E7000038B505463C
:10B9A00043680C4619BB174A92F82E10C1F34000A9
:10B9B00089071BD5934222D138BD33B193F82E208D
:10B9C0006FF3410283F82E2054B105F12401204683
:10B9D000FFF704FF94F82E3043F0020384F82E3072
:10B9E00001236C6085F858300120E5E714469C423D
:10B9F000FAD094F82E209207DFD50020DCE7002B48
:10BA0000DCD1D9E78C210120836900681847036ADB
:10BA1000006818472DE9F04F8DB004460593BDF836
:10BA200058300693199B07925A88029290F84A2040
:10BA3000B3F800A0B3F80490DB889DF85C809DF813
:10BA400060600393072A0D460ED80823B3FBF2F279
:10BA500090F84B30534390F85020002A00F0B78004
:10BA6000BAFBF3FAB9FBF3F92046FFF7CDFF002E3E
:10BA700008BF46468DF828500125B8F1000F40F068
:10BA8000AF800095E76920680AAB42464146B84757
:10BA9000AB464546AA1C0492B4F84620B4F954308B
:10BAA000FF2A00F2A080DAB25AFA83FA0CAB2B44D8
:10BAB00003F808AC531E99446A1C0CAB134403F8FA
:10BAC000089C05F102090AAB2068E769CDF80090EF
:10BAD00032465946B8472046FFF799FF059BB3F514
:10BAE000807F1BD04FF0010A20468DF82730FFF7EA
:10BAF0008BFF2068E769CDF800A00DF127033246DF
:10BB00000021B847C9F3470320680093E7690AABEF
:10BB100032465146B8472046FFF779FF2046FFF7E7
:10BB200073FF079B8DF82830B8F1000F07D1012370
:10BB300000932068E7690AAB42464146B847B4F82B
:10BB40004820B4F95630FF2A0CAA0CA902EB0500D4
:10BB500005F101020A44114663D8029DDAB255FA92
:10BB600083F300F8083C531E039A134401F8083C81
:10BB7000049B2068009332460AAB5946E569A84702
:10BB80002046FFF744FF069BB3F5807F1CD04FF0A3
:10BB9000010820468DF82730FFF736FFE569206859
:10BBA000CDF800800DF1270332460021A847049B01
:10BBB0002068E569C3F34703009332460AAB414668
:10BBC000A8472046FFF723FF0DB0BDE8F08F029A8B
:10BBD000B2FBF3F20292039AB2FBF3F3039343E74F
:10BBE0004FF0000B56E79AB21AFA83FA531E0CAACA
:10BBF0002A44CAF3072102F8081C691C0CAA0A444B
:10BC0000A81C02F808AC0CAA4B440244C3F3072159
:10BC100002F8081C0CAA2A4405F1040902F8053CA4
:10BC200051E7029F9AB217FA83F3C3F3072C039FDD
:10BC300000F808CC013A01F8083CA91C0CAB0B44F5
:10BC40001744C7F3072103F8081C2B1D04930CAB02
:10BC50001D4405F8057C8BE738B50546343014469D
:10BC6000FFF711FE10B395F84A20072A1ED80823C3
:10BC7000B3FBF2F395F84B2095F8505013FB02F309
:10BC8000DBB2A5B1B4F9002092FBF3F103FB112163
:10BC900009B1521A2280B4F9042092FBF3F103FB9C
:10BCA000112119B113445B1AA380284638BDB4F999
:10BCB000022092FBF3F103FB112109B1521A6280B9
:10BCC000B4F9062092FBF3F103FB11210029EDD01A
:10BCD00013445B1AE380E9E740687047A1F1200351
:10BCE0005E2B2DE9F0410E4602D8D8B2BDE8F081B6
:10BCF000C568078A4FF000082F44BD425FFA88F4F8
:10BD000001D3FF20F2E72846FBF78CFD01462846C9
:10BD1000FBF7A5FD8E42054608F10108EDD104F1BF
:10BD20005F00C0B2E2E70268034610783E2805D8FB
:10BD30003B2805D8212806D0402070474028FBD159
:10BD400001321A6070473E20FAE7000010B50C6817
:10BD5000606818B1FEF7F2FD00236360004810BD73
:10BD60006C54060010EE103A23F00043B3F1485F24
:10BD700004DAFDEEC07A17EE903A5BB320EE007A5B
:10BD8000DFED157A9FED156AA7EE276ADFED147ACD
:10BD9000E6EE077A9FED136AA7EE876ADFED127A67
:10BDA00060EE076AE6EE077A30B99FED106AA7EEFB
:10BDB000276AA6EE260A704767EEE67AB6EE006AB4
:10BDC000E0EE867AD7EE870ADFED097AE6EEA70A7B
:10BDD00030EE600A704700BFD3C92E2F342FD7B280
:10BDE0001BEF3836010D50B98988083CABAA2ABE32
:10BDF000ABAA2A3E10EE103A23F00043B3F1485F9D
:10BE0000B7EE006A05DAFDEEC07A17EE902A002A36
:10BE10003DD060EE005ADFED1F7A9FED1F7ADFED17
:10BE20001F6A1F4AA5EEA77A9342DFED1E7AE7EE5E
:10BE3000257A9FED1D7AA7EEA57ADFED1C7AE7EE55
:10BE4000257AB0EE667AA7EEA57AF6EE006A65EE80
:10BE5000A67A67EE256A20EEC07AA5EEA67A04DC03
:10BE600037EEC77A36EE470A7047114A9342DABF77
:10BE700003F17F4306EE903AF5EE026A77EEE67A3A
:10BE800036EE660A77EEC77A30EE670A7047B0EE94
:10BE9000460A70474ED747ADF6740F31ABAA2A3D1C
:10BEA0009999993E7CF293B4010DD037610BB6BAE3
:10BEB0000000483F10EE103A23F00042B2F1465F16
:10BEC00016DAFDEEC07A17EE901A39BB431C134305
:10BED00006D1F0EEC07AB7EE007A87EE270A7047F7
:10BEE000012800F0A080FFEE007A87EE800A7047FC
:10BEF0004D498A4212DBDFED4D7A002BB8BFB1EE1F
:10BF0000400A37EEC00ADFED4A7AB8BFF1EE600AA8
:10BF100077EEE00A30EE800ADFED460A9FED466AD2
:10BF2000DFED466ADFED465A3F4920EE007A8A424D
:10BF300067EE077AE7EE866A9FED426AA6EEA76A89
:10BF4000DFED416AE6EE276A9FED406AA6EEA76A3A
:10BF5000DFED3F6AE6EE276A9FED3E6AA7EEA56A2F
:10BF6000DFED3D5AE6EE275A9FED3C6AA5EEA76A43
:10BF7000DFED3B5AE6EE275A9FED3A6AA5EEA76A37
:10BF8000F0EE467AE7EE876A20EE076AF0EE667A10
:10BF9000F0EE606AE7EE866ADFED337AE6EE870A56
:10BFA000E6EE270A30EE207A1DDB07EE900AF8EE67
:10BFB000E77A27EE076A37EE277A9B17C6EE076AFD
:10BFC00003F00203C3F10103B0EE007A76EEE00A5B
:10BFD00070EE600A00EE103AE0EEC77AB8EEC00AE2
:10BFE00020EE270A704701281BD0FFEE007AC7EE2B
:10BFF000876A1E4B17EE102A1A4006EE102A16EE1C
:10C00000902A36EE400A134070EEC00A00EE103A55
:10C01000F7EE007AE6EE007AE0EE807AA7EEA60A66
:10C020007047B0EE470A704740A12C3FDA0F493FF6
:10C0300068212233000000005FAE9BB745F4A338AF
:10C040008453D937C8261A3A16696B3BA427B33CE8
:10C050008988083E7AC09538B937813948DEBE3ABA
:10C060001F37113CD10D5D3DABAAAA3E00F0FFFF8A
:10C07000DFED0A7A9FED0A7ADFED0A6AA0EE277AF1
:10C08000DFED097AE7EE007AB7EE007AA0EE267AC5
:10C0900067EE807A87EE870A704700BF6BD30DBCCE
:10C0A000BA132FBDAEE534BF75AA2A3EF0B501F034
:10C0B0001F014368C1F11F0523FA05F58B4043605A
:10C0C00083685E1A002E4FEA550586602CDAC26836
:10C0D000032AA1EB030129DD04682746631C0360E2
:10C0E00017F8023B1B06C0E90073677843EA074371
:10C0F000E71C43600760A77843EA0723271D4360D6
:10C100000760E47823434360043A20238360C260DD
:10C11000436806F1200223FA02F21543826803FA0B
:10C1200001F11644866041602846F0BD002343605B
:10C13000144647684CB9C2F10303DB0007FA03F366
:10C14000D200C0E902244360E2E7036803F1010C76
:10C15000C0F800C01B783B431B02013C4360E8E78A
:10C16000F0B510B94FF0FF30F0BD0368002BF9D0E7
:10C170000A78FF2AF6D14C7804F0E002E02AF1D1E7
:10C18000E20814F0180F1ABFD24302F00102022293
:10C190001A704C78C4F34104C4F104045C604D7817
:10C1A000ED4305F001059D608F783F09DF608E78D3
:10C1B000C6F381061E618D78C5F340055D618D78FB
:10C1C00005F001059D61CD78AD091D7791F803C09B
:10C1D000CCF3011CC3F820C091F803C0CCF3C00C11
:10C1E000C3F824C091F803C0CCF3800CC3F828C076
:10C1F00091F803C0032E0CF0030CC3F82CC0B1D08F
:10C20000042CAFD00F2FADD0DE2454434A2212FBB2
:10C210000642384E012D16445E6303D00022032DE2
:10C220001A6262D00222C0F8BC271A781C6902EB9D
:10C2300042022244304C54F82220C0F8C0271A7819
:10C24000002A0CBF02250125C0F8C4571A785C6883
:10C2500002EB4202013C2244284C34F9122092FBAA
:10C26000F5F2C0F8C8275A68C0F8D0271C7880F8C3
:10C27000D447DE68002E30D05A68013AC2EB02156E
:10C280002D2202FB045434441D4D35F814404FF464
:10C290007A7514FB05F4C0F8B8471D691C78C5EB26
:10C2A000051502FB0452DD682A44164D35F91220AB
:10C2B0001D7F6400032D18BF0134134D35F9144060
:10C2C0005D69121B9C68002C18BF0224043A121BE3
:10C2D000002D18BF0132C0F8CC279A683AB18A887D
:10C2E00052BA92B21A6306203EE701229BE71A6314
:10C2F000042039E792FA06005CFA060080FA06008C
:10C30000E8CF060038FD06002CFD06002DE9F04FB1
:10C3100087B0CDE90323109B052B8C4600F30783E0
:10C32000C3F1060E00F17C01031F53F8042F42FAFB
:10C330000EF299421A60F8D1C56F0368D0E90F1464
:10C340005A195B1B7D4D85FB03630D195B00091BAF
:10C350007B4C84FB0161541904604901794C521BE8
:10C3600084FB02525200C2635A1802645B1A84FBB7
:10C3700003235B00856FC3674368816B446C5A1964
:10C380005B1B714D85FB03630D195B00091B6F4C33
:10C3900084FB016154194460C9006D4C521B84FB3D
:10C3A0000252520082635A1842645B1A84FB0323D0
:10C3B0005B00456F83678368416B846C5A195B1B14
:10C3C000644D85FB03630D195B00091B624C84FB04
:10C3D000016154198460C900604C521B84FB0252F5
:10C3E000520042635A1882645B1A84FB03235B0089
:10C3F000056F4367C368016BC46C5A195B1B584DCA
:10C4000085FB03630D195B00091B564C84FB01611E
:10C410005419C4608900544C521B84FB02525200D0
:10C4200002635A18C2645B1A84FB03235B00C56E67
:10C4300003670369C16A046D5A195B1B4B4D85FB89
:10C4400003630D195B00091B494C84FB01615419FE
:10C4500004618900474C521B84FB02525200C262A5
:10C460005A1802655B1A84FB03235B00856EC36662
:10C470004369816A446D5A195B1B3F4D85FB036319
:10C480000D195B00091B3D4C84FB0161541944618B
:10C4900049003B4C521B84FB0252920082625A18A4
:10C4A00042655B1A84FB03239B00456E83668369A8
:10C4B000416A846D5A195B1B324D85FB03630D196C
:10C4C0005B00091B304C84FB0161541984614900F5
:10C4D0002E4C521B84FB0252920042625A18826513
:10C4E0005B1A84FB03239B00056E4366C369016AE4
:10C4F000C46D5A195B1B264D85FB03630D195B0048
:10C50000091B244C84FB01615419C4614900224C6D
:10C51000521B84FB0252120102625A18C2655B1A56
:10C5200084FB03231B0103661C4FDFF874B000F18A
:10C53000A00300F12002059334E000BF51C2134074
:10C54000FB22855172464F40BD45B340CF200B6D55
:10C55000103CE1426D2DFA419057D941449F9148DA
:10C560002134F943968DFC5E630ECB52C41BCC463E
:10C57000971AD84A2E40E264F09C9D4AB31D7D7CF8
:10C58000A924E2431137AE4F26CF6F6BC1923C6EA8
:10C59000A71E6056EBF64C5F044E9E515C2E0600C3
:10C5A0009A79825A52F8203C52F8044C3E6E19197E
:10C5B00052E905851B1B86FB034308EB05067C6ED1
:10C5C0005B00A8EB050884FB08584FEAC804BD6E61
:10C5D00001EB0608891B85FB01611E1949000091CA
:10C5E00001961B1B85FB03435B0052F8089C0293DA
:10C5F00052F81C3C52F8185C52F80C6CF96E03EBC4
:10C600000904A3EB090381FB039305EB0609396FCA
:10C610005B00AD1B81FB05A504EB0906D7F874A0F0
:10C620006D00A4EB09048AFB049403EB0509A40044
:10C630005B1B8AFB03539B00A8EB06058BFB05A540
:10C640000099A1EB040A8BFB0A1A4FEA4A0142F84F
:10C65000141C0099214401EB4A0142F8181C01996D
:10C6600046446D0042F8206C42F81C5CA1EB0901C5
:10C670008BFB0141029C029D1C444900EB1A8BFB81
:10C680000353019E04EB43045D00B14401EB4303FB
:10C6900042F80C3C09EB0406059B42F8106C0C4474
:10C6A00042E902452032934207F118077FF47AAF3E
:10C6B000DDE903329C1A002A04F0070404F58064C3
:10C6C00014BF4FF000084FF4885808EB84050CEBBA
:10C6D000050703683B624CF80530039B466814BFAE
:10C6E0004FF48852002202EB83020CEB02031E621D
:10C6F0004CF80260466E426F3244466C1644C3F8F2
:10C700002061C3F80061416B466A0E44C3F82062A1
:10C71000C3F80062416D0A44C3F82023C3F8002324
:10C72000466FC26E32444669C3F82064C3F80064A1
:10C73000466D1644C3F82065C3F80065C16A466BB0
:10C740000E44C3F82066C3F80066C16C0A44C3F8FF
:10C750002027C3F80027C66EC26F3244C668C3F8EC
:10C760002068C3F80068C66C1644C3F82069C3F893
:10C770000069C16BC66A0E44C3F8206AC3F8006A38
:10C78000C16D0A44C3F8202BC3F8002BC269C66FE1
:10C79000C3F8202CC3F8002CC26D3244C3F8202DFE
:10C7A000C3F8002DC26BC3F8202EA5F57C61C3F839
:10C7B000002EC3F8206F0CEB0102C3F8006F446831
:10C7C00014624CF80140446E816F466C21440E4463
:10C7D000C2F82061C2F80061466A846B3444C2F832
:10C7E0002042C2F80042866D3144C2F82013C2F8DC
:10C7F00000138169C2F82014C2F80014846F816E9E
:10C80000866D21440E44C2F82065C2F80065866B2F
:10C81000846A3444C2F82046C2F80046866C31442B
:10C82000C2F82017C2F800178168C2F82018C2F8B1
:10C830000018846E016F866C21440E44C2F8206992
:10C84000C2F80069866A046B3444C2F8204AC2F810
:10C85000004A066D3144C2F8201BC2F8001B016972
:10C86000C2F8201CC2F8001C046F016E066D214442
:10C870000E44C2F8206DC2F8006D046A066B3444A1
:10C88000C2F8204EC2F8004E046C2144C2F8201FAA
:10C89000C2F8001FBEF1000F46D05CF80510CEF1C3
:10C8A0001F044FF0004041FA04F820FA0EF0CE17B2
:10C8B000B8EBE17F00F1FF3018BF80EA060101FA12
:10C8C0000EF139624CF8051003F1200503F5815390
:10C8D00055F8201C41FA04F7B7EBE17F4FEAE17607
:10C8E00018BF80EA060101FA0EF1296045F8201C04
:10C8F00005F58075AB42EBD102F1200102F58152C2
:10C9000051F8203C43FA04F6B6EBE37F4FEAE375B7
:10C9100018BF80EA050303FA0EF30B6041F8203CD0
:10C9200001F580718A42EBD107B0BDE8F08F4FF07E
:10C93000000E01E538B10023002801DA18467047DF
:10C9400001334000F8E72023F8E700002DE9F04F1D
:10C950000446594D5948DFF89091884603F0030189
:10C960009B1089B01F2B05EB81159C4650F82110B8
:10C970000291A8BF4FF01F0C1C2B1946A8BF1C2109
:10C980006E68033121EAE1710E410596AE680E41F1
:10C990000696EE68002046FA01F104EB820204904C
:10C9A00007910392019054F8046B454A164226F011
:10C9B000004114D108AA02EB810151F8102C019911
:10C9C000002E41EA0201B8BF524248F8042B039AF4
:10C9D0000191A242E7D1019809B0BDE8F08F394A30
:10C9E00016420AD1002B55F82110BABFCCF1000233
:10C9F00001FA02F241FA0CF2E1E7334A164214D18D
:10CA00001039324A029F52F8212082FB0717ACF1FD
:10CA1000030100294DDA49426FF0004242FA01FE5B
:10CA2000BE45CCDB07FA01F2C9E74A04B2F1006F58
:10CA3000B6BF4A0500210421B2F1005FBCBF9200DD
:10CA40000231234F2348B2F1804FBCBF5200013165
:10CA5000BA42214FC8BF38468346204F2048D4BF32
:10CA6000BE4686469246584680FB0ABADEF80470F7
:10CA70005744924687FB0ABADEF80870574492463C
:10CA800087FB0ABADEF80C70574487FB02A2DEF877
:10CA900010703A4459F8217082FB07E74FEAC70E3D
:10CAA000029F8EFB07270F4A52F82110ACEB0101C1
:10CAB000AFE747FA01F282E7808806007087060038
:10CAC000FCFFFF7FF0FFFF7FC0FFFF7FC0870600F6
:10CAD0009979825AA9BDA029632185105087060043
:10CAE0003C87060080870600A08706002DE9F74FE7
:10CAF0000368816982680469066AD0F80CC05B1A11
:10CB00000193C1694369591A131BA3EB060B02EB8E
:10CB1000040E364B83FB0C5C45684769EF1BC56907
:10CB20007F1B83FB0757324DF04685FB0838314B9E
:10CB3000324483FB0292361B85FB0646744683FB18
:10CB40000454DFF8B4A08E468AFB0E3E4368C569E4
:10CB5000DFF8A8902B4489FB035345680093436991
:10CB60001D448AFB053589FB01A103689946836949
:10CB700009EB630A019B0AEB4C09AAEB4C0C03EB93
:10CB80006B0A009B520002EB48025B00490003EB7A
:10CB90004E0EC1EB450509EB020171446400C4EB84
:10CBA000460601600AEB470141600CEB060194194F
:10CBB0002944A5EB0E038160ACEB0401C91AC160E6
:10CBC0000199A9EB04044E446244A1EB0B011C44FF
:10CBD000751BAAEB4707A2EB0E0201614461856158
:10CBE000C761026203B0BDE8F08F00BFA1EBD96E50
:10CBF0008BBE0D627E1A3A1649DD4652322E0E7EEB
:10CC00002DE9F0410568C4688269436A066BC06B10
:10CC1000DFF87CC0361A9B1BD21AA41A1B1A2D1BD4
:10CC2000E41A6D1064108CFB027205EB6607AD1BF5
:10CC300007EB4206A7EB42078CFB032304EB6002E1
:10CC40004FEA430CDFF84CE002EB43038EFB038317
:10CC5000201A9B000C4C84FB00E00C4C8000A2EBE3
:10CC60000C0284FB02C2F4180C602C184C60281AC9
:10CC700007EB8204F31AA7EB82028C60CA6008619A
:10CC80004B61BDE8F08100BF9A79825A83FB202175
:10CC9000A1EBD96E1D75A37B022A2DE9F0415AD173
:10CCA0003B4B826883FB02423A4E846986FB045404
:10CCB00022440A60384C426884FB0252374FC569EF
:10CCC00087FB05C52A444A60026883FB0252056A55
:10CCD00086FB05752A448A60314F026887FB025241
:10CCE000304D066A85FB06C63244CA604FF0604686
:10CCF000426886FB02C2D0F81CC086FB0CEC624482
:10CD00000A61826885FB02C2D0F818C087FB0CEC70
:10CD100062444A61426983FB02C28A61026984FB00
:10CD200002C2CA61C26883FB02420A62C36887FB0F
:10CD300003234B62036986FB03238B62436985FBF4
:10CD40000323CB620023C1E91033C1E90E33C1E9EB
:10CD50000C33BDE8F081144B902404FB023202F145
:10CD6000480C01F144058C3200F1240E50F8043BCC
:10CD700052F804695CF8047B1C4687FB048441F884
:10CD8000044B86FB0343864545F80439EED1E0E7C2
:10CD9000D8E3CEB8281C310733C3BEB2CD3C410D19
:10CDA0009A615FC9669EA0F69CF306002DE9F047E4
:10CDB00002F001028BBB6AB3D0F88020D0F88072F9
:10CDC000D0F88063D0F88054D0F88045D0F8801631
:10CDD0005242C0F88020D0F880215242C0F8802111
:10CDE000D0F880275242C0F88027D0F880287F42B0
:10CDF000524276426D4264424942C0F88028C0F8EF
:10CE00008072C0F88063C0F88054C0F88045C0F8D4
:10CE100080161A461046BDE8F0874FF00044DC400B
:10CE2000013C00F51067C3F11F06002A3DD0002227
:10CE300094469646056845FA06F94FEAE578B9EB57
:10CE4000E57F18BF88EA04059D400560E04685EA55
:10CE5000E578A8EBE578D0F880506D4245FA06FAFF
:10CE60004FEAE579BAEBE57F18BF89EA04059D40F2
:10CE7000C0F88050F14685EAE579A9EBE5790D68BF
:10CE800048EA090845FA06F9B9EBE57F42EA0802E3
:10CE90004FEAE57818BF84EA080500F580709D40E8
:10CEA000B84241F8045BC5D1B4E79446964605689C
:10CEB00045FA06F94FEAE578B9EBE57F18BF84EA51
:10CEC00008059D400560E04685EAE578A8EBE57831
:10CED000D0F8805045FA06FA4FEAE579BAEBE57FDB
:10CEE00018BF84EA09059D40C0F88050F14685EAE4
:10CEF000E579A9EBE5790D6848EA090845FA06F9EC
:10CF0000B9EBE57F42EA08024FEAE57818BF84EA08
:10CF1000080500F580709D40874241F8045BC6D14A
:10CF200078E730B570B930BD21F813500133D0F82F
:10CF3000C827D0F8C4475443D0F8BC276243934273
:10CF4000F2DBF0E700231D46F1E70346013900203C
:10CF5000814202DC4FF0FF30704713F8012BFF2AAB
:10CF600004D11A7802F0E002E02AF5D00130EFE7B0
:10CF70002DE9F04F87B000264FF0007C00900A6842
:10CF8000CB6D64463546C2FB06456FF0730EC3FB9E
:10CF90000E45D1F8DC70D1F8800062463346C0FB04
:10CFA0000623C7FB0E234FF4557A4868C0FB0A4599
:10CFB000834F886DC0FB0745D1F88400C0FB0A236E
:10CFC000D1F8D800C0FB072341F6D4798868C0FBAC
:10CFD00009457C4F486DC0FB0745D1F88800C0FB70
:10CFE0000923D1F8D400C0FB072346F2B86EC86805
:10CFF000C0FB0E45744F086DC0FB0745D1F88C008F
:10D00000C0FB0E23D1F8D000C0FB07236F4F086987
:10D01000C0FB07456E4FA046AB46CC6CC4FB078BEC
:10D020006A48D1F89050D1F8CC40C5FB0023C4FB2E
:10D0300007238F6C486944465D46C0FB0E4545F2A8
:10D040008408C7FB0845D1F8C870D1F89400C0FB2C
:10D050000E23C7FB08234F6C8869C0FB094540F2CB
:10D060002C7EC7FB0E45D1F8C470D1F89800C0FBE8
:10D070000923C7FB0E230F6CC869C0FB0A454FF09C
:10D08000740EC7FB0E45D1F8C070D1F89C00C0FBF0
:10D090000A23C7FB0E234FEA946444EA85140098E0
:10D0A00004804FEA926242EA831201F58053428083
:10D0B0001B684FF4D07465463246C3FB045201F539
:10D0C00084536746D3F800E03346CEFB047341F245
:10D0D000040451F804E041F67C04CEFB045241F212
:10D0E000840E51F80EE0CEFB047341F2080451F8AF
:10D0F00004E049F2FC74CEFB045241F2880E51F870
:10D100000EE0CEFB047341F20C0451F804E0314C04
:10D11000CEFB045241F28C0E51F80EE0CEFB0473AC
:10D1200041F2100451F804E02B4CCEFB045241F2C2
:10D13000900E51F80EE0CEFB047341F2140451F846
:10D1400004E06FF0B304CEFB045241F2940E51F8A8
:10D150000EE0CEFB047341F218044FF4127E51F836
:10D1600004801446C8FB0E5441F2980251F8028024
:10D170003A46C8FB0E2341F21C0751F807E06FF056
:10D180001307CEFB075441F29C0E51F80EE0CEFB84
:10D1900007234FEA956545EA8415A0F840504FEA09
:10D1A000926242EA8312034608330193CDE902C634
:10D1B00003464433DFF824E0A0F8422005930FE053
:10D1C000D4F8FFFF7CAFFFFF3CB6FDFF789404006E
:10D1D000C44902004CE803002464FFFFDCF50600AC
:10D1E000DEE91089DDE9024CD1F80001D1F85C31AB
:10D1F000C0FB084CDDE90226C0FB0926C9F1000A84
:10D20000C3FB0A4CC3FB0826DDE90207D1F880B155
:10D210000492CBFB0807DDE90235CBFB0935D1F8D9
:10D22000DC21C2FB0A07C2FB0835DEE912B8D1F8DF
:10D2300004A1D1F85891CAFB0B4C049ACAFB0826EA
:10D24000C8F1000AC9FB0A4CC9FB0B260492D1F8AD
:10D25000D891D1F88421C2FB0B07C2FB0835C9FB6A
:10D260000A07C9FB0B35DEE914B8D1F808A1D1F8DB
:10D270005491CAFB0B4C049ACAFB0826C8F1000A59
:10D28000C9FB0A4CC9FB0B260492D1F8D491D1F802
:10D290008821C2FB0B07C2FB0835C9FB0A07C9FB83
:10D2A0000B35DEE916B8D1F80CA1D1F85091CAFBC4
:10D2B0000B4C049ACAFB0826C8F1000AC9FB0A4CA9
:10D2C000C9FB0B260492D1F8D091D1F88C21C2FB76
:10D2D0000B07C2FB0835C9FB0A07C9FB0B35DEE9A2
:10D2E00018B8D1F810A1D1F84C91CAFB0B4C049A94
:10D2F000CAFB0826C8F1000AC9FB0A4CC9FB0B2669
:10D300000492D1F8CC91D1F89021C2FB0B07C2FB5B
:10D310000835C9FB0A07C9FB0B35DEE91AB8D1F895
:10D3200014A1D1F84891CAFB0B4C049ACAFB0826F9
:10D33000C8F1000AC9FB0A4CC9FB0B260492D1F8BC
:10D34000C891D1F89421C2FB0B07C2FB0835C9FB79
:10D350000A07C9FB0B35DEE91CB8D1F818A1D1F8D2
:10D360004491CAFB0B4C049ACAFB0826C8F1000A78
:10D37000C9FB0A4CC9FB0B260492D1F8C491D1F821
:10D380009821C2FB0B07C2FB0835C9FB0A07C9FB82
:10D390000B35DEE91EB8D1F81CA1D1F84091CAFBCB
:10D3A0000B4C049ACAFB0826C8F1000AC9FB0A4CB8
:10D3B000C9FB0B260492D1F8C091D1F89C21C2FB85
:10D3C0000B07C2FB0835C9FB0A07C9FB0B354FEA3F
:10D3D000946444EA8C14019A22F8044C4FEA906059
:10D3E00040EA871022F8020C049A4FEA926242EA5D
:10D3F00086120098A0F87C204FEA936343EA8513D5
:10D40000A0F87E30019B059A04330193031F00931B
:10D41000019B93420EF1400E01F580717FF4E0AE66
:10D4200007B0BDE8F08F00BF024B03480022C3F8ED
:10D43000B8207047804E01206C54060043788278F3
:10D440001B01120202F4E06203F03003134302787E
:10D4500002F003021343C278120302F48052134312
:10D460000279120402F4E02213434279120502F415
:10D47000801213438279120602F080721343024A2B
:10D48000C2F81835704700BF0070004010B5084A58
:10D49000002388214FF6FF7001FB03F4A45A844255
:10D4A00004D10133052BF7D1024810BD0248FCE737
:10D4B000C0460120645406007054060001F0604329
:10D4C000B3F1005F70B502460E4663D10379324D69
:10D4D000242101FB0351496821B100684FF4047411
:10D4E000C0F80843242000FB03539C6954B1D86959
:10D4F00000283FD021B113684FF40472C3F804230D
:10D50000264836E001219961DE60DC6110684FF445
:10D510008871FCF787FE4FF4A2711068FCF782FE59
:10D5200013680121C3F83465C3F83815136824BBA8
:10D53000196011791368242202FB015252681ABB48
:10D54000D3F81041D3F84421D3F82461144302D115
:10D55000002EF5D02246242303FB0155002310485A
:10D56000AB61104B002E18BF18460733002A18BFB6
:10D57000184670BD1E610124C7E7D3F8001241F0C0
:10D580002001C3F80012D4E74FF404720448C3F832
:10D590000423EEE70448ECE7984D01200B00AD0BA7
:10D5A0000000AD0B0100AD0B0A00AD0B10B5037808
:10D5B000012B0C4602D0022B00D010BD4168027A2C
:10D5C00004F11000FDF76FF8606804F11C01BDE87C
:10D5D0001040FFF773BF000013B5104B10481B68D5
:10D5E00000681A680121D1600E4A128892B20024A4
:10D5F00030F812001A68C2F84041D2F84021019276
:10D60000019A1A684FF48034C2F804431A68C2F8C9
:10D6100040051B68196002B010BD00BF54510120C5
:10D62000E8500120EC500120B0F5A07F08B524D1CE
:10D63000124B13481B6800881B6801225A60114A6C
:10D64000138801339BB2138013889BB2984204D88D
:10D65000BDE80840081DFDF789BB1388DB0708D427
:10D660004B685A681B7AC2F86035BDE80840FFF77E
:10D67000B3BF081DFDF77AFBF7E708BD5451012041
:10D68000EE500120EC50012007B5019001A8FCF7F5
:10D69000D9FA019B03F5E073890040F8231003B029
:10D6A0005DF804FB38B505460C460846FDF7C8F999
:10D6B0006C6020790021FFF7E7FF002038BD0129C9
:10D6C00006D08B1E5942594143681879FFF7DCBFD9
:10D6D0000321F9E710B5436802460C46187900218A
:10D6E000FFF7D2FF21461046BDE81040FFF7E7BF25
:10D6F0002DE9F34105793A4E24236B43F2180C4689
:10D70000517F8046002968D1F3580BB1012353772C
:10D7100094E80F00242707FB056707F10C0C8CE841
:10D720000F0097F82000FF2805D0BB7F1BB9FB7FB7
:10D73000C3B1FCF7AFFA226822B102F06043B3F143
:10D74000005F06D1A36883B103F06043B3F1005FCB
:10D750000BD0242303FB0565224800236B7702B01E
:10D76000BDE8F081FCF7A3FAE5E7D8F8003061687E
:10D77000C3F84425C3F84815D4E90212C3F8341598
:10D78000C3F838250022C3F81821D3F818110191E5
:10D790000199C3F85025C3F8402501221A612422BB
:10D7A0006A43B258AAB9D3F81821002AFBD024231F
:10D7B00003FB056595F82000FF2805D0AB7F1BB95A
:10D7C000EB7F1BB1FCF773FA0748C8E7FCF762FA76
:10D7D000FAE74022C3F80423F6E70448BFE700BF96
:10D7E000D04C01200A00AD0B0000AD0B0B00AD0BBF
:10D7F00000F1804382B01A68002A14BF0120002083
:10D8000004D000221A601B680193019B02B070478C
:10D8100010B54FF08043D3F80443620707D54FF4A7
:10D820008470FFF7E5FF10B11E4B1B689847A306F5
:10D8300008D54FF48A70FFF7DBFF18B11A4B0020B0
:10D840001B689847600608D54FF48C70FFF7D0FF2F
:10D8500018B1154B01201B689847210608D54FF4D5
:10D860008E70FFF7C5FF18B1104B00201B6898475A
:10D87000E20508D54FF49070FFF7BAFF18B10B4BD3
:10D8800001201B689847A3050AD54FF49270FFF753
:10D89000AFFF28B1054BBDE810401B6802201847B8
:10D8A00010BD00BF6C4E0120704E0120744E01204F
:10D8B00040F20110814209D112F001000AD0064B5A
:10D8C000D88980B2003818BF0120704716221A602C
:10D8D0004FF0FF30704700BF5032012040F201107E
:10D8E00081420BD112F004000CD0074B587848B19C
:10D8F0009B78002B0CBF00200420704716221A6072
:10D900004FF0FF30704700BF5032012008B5074B81
:10D91000D3F80630B3F5966F06D14FF080434E2210
:10D92000C3F81C25FBF706FD08BD00BF2426012017
:10D9300010B58478182104F07F030C22E4095943C0
:10D9400002FB0411114A0A440179117201221049A3
:10D9500002FA03F07CB90C3302FA03F3C1F8043382
:10D96000D1F814350343C1F81435BFF36F8FBFF3FB
:10D970004F8F012010BD023302FA03F3C1F80433C4
:10D98000D1F810350343C1F81035EEE7E82E012039
:10D99000007002402DE9F843DDE908890C4616467F
:10D9A0001F460025AE4201DC01200EE06378052B06
:10D9B00004D1E37803F00303BB4208D00D4B186891
:10D9C00010F0010001D000BE0020BDE8F883204621
:10D9D000FFF7AEFF18B9BDE8F843FBF78BBDA3789E
:10D9E000DA0914BF89F8003088F80030237801354F
:10D9F0001C44D7E7F0ED00E0C208054900F007003D
:10DA000001238340885C20EA03008854704700BFEC
:10DA1000354E012038B5144C0546FCF7AFFC6219B1
:10DA200092F9243092F82420072A9FBF0F4A03F569
:10DA3000A273002142F8231004EBD50305F007027E
:10DA400093F85530D340DB0705D52846FCF714F989
:10DA50002846FFF7D1FF2C4494F82400FCF780FC03
:10DA6000FF2384F8243038BDE04D012000600040E1
:10DA700010B504460079FF281AD00E4B61790022B8
:10DA800043F8202043F82120FCF778FC6079FCF76C
:10DA900075FC2079FFF7BEFF6079FFF7BBFF2079A7
:10DAA000FCF73AFF6079FCF737FF4FF6FF73A3806E
:10DAB00010BD00BF6C44012008B5FFF7D9FF014835
:10DAC00008BD00BF6C54060008B50868FFF7D0FF1A
:10DAD000004808BD6C54060037B5204C2518024696
:10DAE00095F92410072913DD214491F84C309B0946
:10DAF000032B09D1FCF725FC40B10321104603B0EC
:10DB0000BDE83040FCF70ABC012BF6D10221F5E755
:10DB1000CBB2072B1FD88A0002F1804202F5C04227
:10DB20009B00D2F8100503F1804303F5C24340F097
:10DB30000100C2F8100500221A601B680193019BC6
:10DB400095F9243054F823302BB1012303FA01F165
:10DB5000034BC3F8041303B030BD00BFE04D0120F8
:10DB60000060004038B50C464942FAF70BFA022132
:10DB7000FAF789F95C230370447038BD73B50C461D
:10DB800001210646FAF7FEF904F110033F2B06D8EF
:10DB9000A4F18001C9B2FAF785F902B070BD142171
:10DBA0000DF10505FAF77EF9294604F07F00E3B28E
:10DBB000E4112A4605F8010D601C0128F5D801344E
:10DBC00003F0400312D11BB97F2305F8013C951ED9
:10DBD000491B3046FAF757F901AC01462B46A342E0
:10DBE00008D15D1B9DF804204255D6E7002BEFD0ED
:10DBF0000023EAE713F8012B62F07F0201F8012B02
:10DC0000EDE700002DE9F84F90F82E30468D934F48
:10DC1000DFF85082DA0748BF0162054648BF00F1CD
:10DC20001801013E731C02D10846BDE8F88F6B68ED
:10DC300053F8364014F0030E11D12368884A9342FA
:10DC400040F0038194F85130B4F938C0B4F93C0085
:10DC50009B0706D0844502D0216404F13801013EBF
:10DC6000E0E794F850305A0733D5844531D0B4F901
:10DC70004430B4F946209C45A8BF9C46B4F94830CE
:10DC8000A4F82CC09842B8BF1846B4F93A302086A0
:10DC90009342A8BF1346E385B4F94A20B4F93E3055
:10DCA0009342B8BF134604F12C0963864846FDF73A
:10DCB0001CFE228A638A5343B0EB430F02D8616390
:10DCC0004946CCE704F138032164E36404F14401DC
:10DCD000C5E76268930724D1DFF88C9113684B4540
:10DCE0001FD1B2F91430B2F91890994519D002F148
:10DCF00014094945D16114D0B4F81690B9F1010F57
:10DD000029D1A385B2F91630E385B2F918302386FC
:10DD1000B2F91A30638694F8503043F0010384F866
:10DD2000503094F850309A071AD4A26812F00309C0
:10DD300004D11368434516D192F80CE094F85030A2
:10DD40006EF3410384F85030DAB29B0701D4844566
:10DD50000BD1E164BAE794F8503043F00203DEE7F8
:10DD60004FF0010EEAE7CE46E8E7D2077FF577AF3E
:10DD7000B4F90C00B4F92C90B4F930C0A36AB4F92A
:10DD80000EB0B4F92E2093F904E0B3F800A081445A
:10DD90008444B4F932005A44584493F80EB01FFA40
:10DDA0008EFE1FFA89F992B21FFA8CFC80B2BBF189
:10DDB000000F2ED01EFB02A2A28593F905E01EFBE8
:10DDC00009F9B3F802E0F144A4F82E9093F9042085
:10DDD00012FB00F01A881044208693F905205B8816
:10DDE00012FB0CFC9C44A4F832C0B4F93230B4F9F4
:10DDF0002E2061639342BCBF6286E385B4F92C2078
:10DE0000B4F930309342BCBF2286A38504F12C01C3
:10DE100025E71EFB09AEA4F82CE093F905E01EFBF4
:10DE200002F2B3F802E07244E28593F9042012FB97
:10DE30000CFC1A889444A4F830C093F905205B8840
:10DE400012FB00F018446086CFE7BB427FF407AFB7
:10DE50002046FFF7D7FE014601E700BF6438060001
:10DE6000883C0600703A0600D03306000048704730
:10DE70006C5406000E4B1A78C2F34000920716D578
:10DE80001A78510712D40B4A507880B100F07F0203
:10DE900003EB420303EBD01320335A78D20705D4A7
:10DEA0005878C0F3400080F00100704700207047B0
:10DEB0006C450120AC2F012070B5084D084E64243C
:10DEC00045F00105336833B94FF42070A847013C91
:10DED000F8D1044870BD0448FCE700BF402F06009D
:10DEE000009102400700AD0B0000AD0BF8B53C4BB4
:10DEF0005B791446054603F0FF02002B6ED1394EC4
:10DF0000326019B34378023B072B1FD8DFE803F0D8
:10DF1000545250114E4C4A04CB791B068A7943EA7D
:10DF200002434A7943EA02230A7913432E4AC2F88C
:10DF30003C36CB781B068A7843EA02434A7843EAA8
:10DF400002230A781343284AC2F83836264F0123A1
:10DF5000C7F80833AB786A781B0343EA02232A78B0
:10DF60001343EA7843EA42332A7943EA82336A79EF
:10DF700043EAC233C7F83436FFF79EFF1B4B984283
:10DF80002DD0002333603CB36978D7F83C26D7F80E
:10DF90003836023907291FD8DFE801F01D1B191791
:10DFA000161412100023B9E70023BAE70023BBE7D9
:10DFB0000023C0E70023C1E70023C2E7110EE1718F
:10DFC000110CA171110A617122711A0EE2701A0C02
:10DFD000A2701A0A62702370054800E00548F8BD77
:10DFE000484E012000910240009002400700AD0B16
:10DFF0000000AD0B0B00AD0B07B5012300228DF81F
:10E0000000008DF80130114640F201136846ADF86A
:10E010000230ADF80420FFF769FF034BC31A5842E2
:10E02000584103B05DF804FB0000AD0B07B540F2AA
:10E030000113ADF80230013200238DF800008DF895
:10E04000012068460A461946ADF80430FFF74EFF36
:10E05000034BC31A5842584103B05DF804FB00BF9C
:10E060000000AD0B07B500238DF80430012201A993
:10E070000520FFF7DBFF18B19DF804309B07F5D1B1
:10E0800003B05DF804FB000070B5124B1B68064638
:10E090000C4615460BB9002070BDFFF7E3FF0028C2
:10E0A000F9D004F06043B3F1005F10D1A2070ED1A4
:10E0B000094B0420C3F80465C3F80845C3F80C55A0
:10E0C000FCF77EF9054BC31A58425841E4E704486F
:10E0D000F8E700BF7C4A0120009002400000AD0B31
:10E0E0000A00AD0B10B50422ADF5027D0DEB020167
:10E0F0000446FFF7C9FF78B101AA042312F8011BF7
:10E10000FF2909D1013B9BB2002BF7D14FF40072DC
:10E1100002A92046FFF7B8FF00200DF5027D10BDD3
:10E1200007B501328DF800008DF8012040F201138F
:10E1300000226846ADF80230ADF80420FFF7D6FEA5
:10E14000034BC31A5842584103B05DF804FB00BFAB
:10E150000000AD0B08B5114A136913B90620FBF78F
:10E16000FBF81968586011611846C468056946696A
:10E170008769D0F81C80D0F82090D0F824A0D0F87F
:10E1800028B0D0F82CD090ED0C8B90ED0E9B90ED3C
:10E1900010ABD0F808E00120704700BF804E01208E
:10E1A00008B50248FAF729FCFFF7D4FF44730600CC
:10E1B00001207047004870476C540600704740F2D9
:10E1C0000110814217BF162202F004001A604FF0BE
:10E1D000FF307047806870470079400040F00100D0
:10E1E00070470000F0B58BB06846F8F709FF0F4B99
:10E1F0000F4D1F680F4C104E2D1A07F5806001213E
:10E200002844FBF77FFC206070B9012105F5C84068
:10E21000FBF778FC4FF4C043206033602368074A63
:10E220001B681A600BB0F0BD3760F7E73C22012095
:10E23000000004203C5101207C490120EF29780195
:10E2400010B50A4C206840B1094B1A68094B1B688D
:10E250009A4203D10368084A1A6010BDFBF7F2FB2B
:10E2600000232360BDE81040FFF7BCBF3C510120F4
:10E270003C2201207C490120EF2978012DE9F04161
:10E28000164FDFF85C8006460C460025738D9D42D4
:10E2900001D3BDE8F081736853F83500820708D1D7
:10E2A0000368BB4207D190F8513064F3410380F812
:10E2B00051300135EAE74345FBD190F82E30C3F3E6
:10E2C000C002A242F5D064F3C30380F82E305B078E
:10E2D000EFD42146FFF7D2FFEBE700BF883C0600F2
:10E2E000643806008088400040F001007047C08814
:10E2F000400040F001007047004870476C54060031
:10E300008088400040F001007047000004288B68BE
:10E3100003D0052808D000207047064A06489BB263
:10E32000002B08BF10467047044800EA430040F045
:10E33000010070476454060070540600FEFF01009F
:10E3400000234360C3600148704700BF6C5406005F
:10E350000B68024800225A60704700BF6C540600E8
:10E360000B6802480022C3E9012270476C54060082
:10E3700008B5FCF7E3FA014808BD00BF6C5406007D
:10E3800008B50868FCF7DAFA004808BD6C540600C6
:10E3900041680A7A2AB901230B72416818460A7249
:10E3A000704700207047436800221A727047416826
:10E3B0000A7A2AB901230B72416818460A7270471B
:10E3C0000020704710B5074B82689A42044608D077
:10E3D0000430FCF7B3FA04F10C00BDE81040FCF780
:10E3E000ADBA10BD6C54060008B50868FFF7EAFF27
:10E3F000004808BD6C54060008B5FFF7E3FF01486C
:10E4000008BD00BF6C5406008268034B9A4202D0DC
:10E410000430FCF793BA70476C54060008B5FFF758
:10E42000F3FF014808BD00BF6C54060008B508683A
:10E43000FFF7EAFF004808BD6C54060008B50868FD
:10E44000044BC2689A4202D00430FFF7DDFF014856
:10E4500008BD00BF6C540600037A1BB90123037288
:10E460000148704701487047705406006454060024
:10E47000044B054801221A70044B03F138029A65D7
:10E48000704700BF155101206C540600804E0120DA
:10E4900043681A7A12B90120187270470020704739
:10E4A00038B505460C46FCF731FBC5E90001024BC7
:10E4B0009B689B09236038BD10E000E0F0B585B093
:10E4C00001A9044602A8FFF7EBFF019D334BC5F5F8
:10E4D0007A700190002153F8042B12B11679A642EC
:10E4E00046D001310829F6D105B0F0BDD2E9066762
:10E4F000029B991B538A548AA4B2A0429BB230D289
:10E50000508AC5F5FA6380B20129A3EB000305D94F
:10E510004FF47A7000FB0133A3F57A734FF6FE7067
:10E520004FF6FF71834288BF0B46D189108A9489C8
:10E5300080B210FA81F1B1FBF4F004FB1011906885
:10E5400020F81130138A91899BB299428BBF138AAC
:10E55000D389013301338BBF9BB29BB21382D3812A
:10E5600014E0C31A4FF47A70414311FA83F3D5E7EC
:10E57000D379002BBAD02046FBF7E3FE003853795D
:10E5800018BF0120834201D00023D371DDE90201CD
:10E59000BDF80430C2E906015382A5E74C440120CE
:10E5A0008968806A0909F9F775BD8379012B14BF61
:10E5B0004FF48070202040F0010070474069FCF764
:10E5C00051BA0000154A38B500210446042352F818
:10E5D000040B844208BF42F8041C013BF7D1A26837
:10E5E000C2F80035A07E08B1FCF796F9E07E08B1CC
:10E5F000FCF792F9A0680021FCF7D0FA002502216F
:10E60000A068FCF7CBFAE068A560FAF7BBFE2069CA
:10E61000E560FAF7B7FE256138BD00BF644601200A
:10E6200008B5086883680BB1FFF7CCFF004808BD48
:10E630006C540600044B054A5B8B05489BB2002BCB
:10E6400018BF1046704700BF2426012070540600F2
:10E650006454060038B50A4D0A4C286838B1FBF7F7
:10E66000F1F900232B600023C4F8C83038BDD4F87A
:10E67000F830002BF7D0D4F8C800FAF783FEF2E7A1
:10E6800040510120804E012010B50368044613B1AB
:10E690004068FAF777FE2046BDE81040FAF772BEF0
:10E6A00010B5037BDB07044602D48068FAF76AFEE4
:10E6B0000023A36010BD0229F8B5044605D0042943
:10E6C00023D001291CD100202CE05668012E10D047
:10E6D000022E10D00020156829182CBF0127002712
:10E6E00066B1002D0ADA884238BF0021A1601160AE
:10E6F000E9E78068EFE741684868ECE7002FF5D06C
:10E7000016221A604FF0FF300CE0456845B12B7BB4
:10E71000DB0702D4A868FAF735FE2846FAF732FE7E
:10E7200000206060F8BD2DE9F04316468BB0B207BB
:10E73000DDF84890074698463DD416F0040F0CBF0C
:10E740000023202300930A46139B202102A8F9F7F7
:10E7500031FEF30504460DD5431C1F2B0AD80AAA27
:10E760001444252204F8202C0AAA1A44002102F895
:10E77000201C1C4616F040051FD09DF808302F2B9A
:10E780004FF000031BD8012202A9CDE90032384620
:10E79000F8F788FF09F1FF390546013C0DF1090141
:10E7A000CDE90089334622463846F8F77BFF2844F6
:10E7B0000BB0BDE8F0832B23C4E702A9F0E702A960
:10E7C0001D46EDE710B5044638B18068FAF7DAFD6A
:10E7D0002046BDE81040FAF7D5BD10BD38B5044657
:10E7E00058B3006808B1FAF7CDFD606800252560D0
:10E7F00008B1FAF7C7FDA068656008B1FAF7C2FD75
:10E80000E0680025A56008B1FAF7BCFD2069E56065
:10E8100008B1FAF7B7FD60690025256108B1FAF77C
:10E82000B1FDA069656108B1FAF7ACFD0023A361F1
:10E830002046BDE83840FAF7A5BD38BD10B50446FE
:10E84000406808B1FFF7CAFF0023C4E90133C4E9F7
:10E850000533A36210BD000008B5FFF7EFFF0148C4
:10E8600008BD00BF6C54060008B50868FFF7E6FF56
:10E87000004808BD6C54060007B5436801291B79A0
:10E88000019301A80CBF07220322FBF7DBF9019BD0
:10E89000120203F5E07342F0030240F8232003B0B4
:10E8A0005DF804FB00F01F0301229A4043099B001E
:10E8B00003F1604303F56143C3F880211A60704798
:10E8C000084BD3F8183182B04BB1074B07480022F0
:10E8D0001A601B680193019B02B0FBF7F5B902B007
:10E8E000704700BF00F0024018F10240F44C0120D4
:10E8F0002DE9F8431D4B1B6807460E46154693B39A
:10E9000000239AB2954202D80120BDE8F883B25C98
:10E91000FF2A03F10103F4D0DFF85480DFF85490AC
:10E920000024FFF79FFBF0B10620FFF765FBD0B195
:10E93000331903F06042B2F1005F14D19A0712D18B
:10E940003A19C8F81025C8F814354FF48073C8F880
:10E9500018350820FBF734FD484504D104F58074D0
:10E96000A542DED8D0E70020CFE700BF7C4A0120D7
:10E97000009002400000AD0B30B5C1B00C464FF422
:10E98000807269460546FFF77FFBA0B14FF48072A5
:10E9900069462046FFF7ACFF68B14FF480726946C4
:10E9A000A818FFF771FB30B14FF480726946A018C8
:10E9B000FFF79EFF00B9002041B030BD43681879D1
:10E9C00009B9FBF774B9FBF765B938B504460D46CC
:10E9D0001146FFF751FF29462046BDE83840FFF7B2
:10E9E000EDBF38B5044604340D46FCF745F8204623
:10E9F00001220021FFF7E9FF002D14BF06203C2073
:10EA0000FCF730F820460021FEF764FE002D14BF0D
:10EA100040200A20FCF726F8BDE83840FCF746B84D
:10EA200001211030FFF7CABF70B51C464B1E59427A
:10EA3000594105460830FFF7C1FF049AD5E90D108A
:10EA400023462244934200D170BDC1F80C056C6886
:10EA500013F8016B2670C1F80805F3E708B500212B
:10EA60001030FFF7ABFF012008BD000010B50A4BC6
:10EA700082699A420ED000F1180400212046FFF767
:10EA80009DFF0420FBF7EEFF20460121FFF796FFD4
:10EA9000012010BD0020FCE7DC7106002DE9F041EB
:10EAA0002DED028B3B4A836E0126934286B00446CD
:10EAB000B0EE408A80F8996012D1DFED377A60EECF
:10EAC000277A6830FCEEE77A17EE903A99B2FCF7B5
:10EAD0008EF8002384F8993084ED228A012517E00E
:10EAE0002E4A93420CD1DFED2E7AB4EEE70AF1EE16
:10EAF00010FACCBF012100216830FFF75FFFE8E783
:10EB0000B0F88C30B3F5807F08D1002580F899509B
:10EB1000284606B0BDEC028BBDE8F08100F1080884
:10EB20004046FCF771FF0546E8B1DFED1E7A94F828
:10EB3000971094F88C20676AA0688DF8142068EE0E
:10EB4000277AFCEEE77ACDED037A9DF80C3081B19F
:10EB50008DF8153002230093324605AB0021B847EB
:10EB60004046FCF754FF002384F89930002DCFD0A5
:10EB7000B2E78DF81330324605AB00960391B847E3
:10EB80000399676AA06800960A460DF1130331469F
:10EB9000E5E700BF208C060000FF7F47A831060094
:10EBA000A4707D3F00007F4310B5044601211C3056
:10EBB000FFF704FF636800221A7210BD10B50A4BFC
:10EBC00042699A420ED000F1140400212046FFF75A
:10EBD000F5FE0420FBF746FF20460121FFF7EEFE7D
:10EBE000012010BD0020FCE7DC71060007B543687A
:10EBF00001A81B790193FBF725F8019B03F5E0734E
:10EC000050F8230000F0010003B05DF804FB0000A1
:10EC1000F7B5374E3318054693F92430002B0F46CD
:10EC200064DA8B78C3F34003002B0BBF0824002465
:10EC3000092108218C4202D12E4803B0F0BD56F8BC
:10EC40002400013042D1711946F8242081F8244073
:10EC500013B9331983F84C50BB785A0717D4D80727
:10EC600036D501A80195FAF7EDFF019B00EB830073
:10EC7000D0F8003723F00203C0F800371E49EA0835
:10EC800005F0070001238340885C03438B54BA7866
:10EC90003B78910721D5A40004F1804404F5C044D9
:10ECA0002D02D4F8102522F44F3222F44072C4F819
:10ECB00010251B04D4F8102505F47C5503F44033CB
:10ECC0001D431543C4F810550C48B6E70134B1E7AD
:10ECD00079782846FEF7D8FCD0E7083C344494F80D
:10ECE000545045EA831384F85430EDE70448A4E710
:10ECF000E04D01200200AD0B354E01200000AD0BB0
:10ED00000B00AD0B2DE9F743002406460F4600F536
:10ED1000A0754FF48038A1462B688BB1D6F8043328
:10ED200008FA04F21A420BD0C5F800902B68019340
:10ED3000019BA30003F5A07398B2D7E9003198476F
:10ED40000134042C05F10405E6D103B0BDE8F083DD
:10ED500001490248FFF7D6BF244D012000A0004022
:10ED600001490248FFF7CEBF184D01200090004036
:10ED70007FB50222ADF814203B4A002303210493FF
:10ED80008DF81630C2F8F0150121C2F8F435C2F83A
:10ED9000001519461A0102F1804202F5E0420133E2
:10EDA000082BC2F81415C2F81015F3D104A8FEF709
:10EDB00045FB2D4B0922C3F81425C3F810250DF18E
:10EDC0000202C3F82C260122C3F830261A6003F58C
:10EDD00080731A68002AFCD000221A601B68019315
:10EDE000019B224B01221A6003F580731A68002AE6
:10EDF000FCD000221A601B680293029B1C4B01226C
:10EE00001A601C4A1368002BFCD0002313601268A0
:10EE10000392039A144ADFED186AC2F80035BDF96F
:10EE200002209A42B8BFADF80230BDF9023007EEB9
:10EE3000103AB8EEC77AC7EE267A9FED107A67EEE1
:10EE4000877AF4EE677AF1EE10FA7DBF17EE903A0A
:10EE500023F0030040F00200094878BFA0F1FF4012
:10EE600007B05DF804FB00BF007000400470004074
:10EE70000870004014710040FFA66A4633335340C7
:10EE80006C540600044A8B881278DBB29A4201D097
:10EE9000FAF730BB01207047AC2F012007B543685B
:10EEA00002461B79019301A8FAF7CCFE019B03F5FA
:10EEB000E07350F8233013F0010F536808D118792C
:10EEC000FBF73FFA003818BF012003B05DF804FBE0
:10EED0001B79019301A8FAF7B5FE019BD0F8040550
:10EEE000D84000F00100F0E738B500F10C04012132
:10EEF0002046FEF7EFFB2046FFF7D0FF0122054634
:10EF000011462046FFF761FD284638BD10B504467E
:10EF10000434FBF7B1FD012200212046FFF755FD27
:10EF20000620FBF79FFD00212046FEF7D3FB0620BD
:10EF3000FBF798FD2046FFF7B1FF04463720FBF7AB
:10EF400091FDFBF7B3FD204610BD10B50446043417
:10EF5000FBF792FD012200212046FFF736FD4FF41A
:10EF6000F070FBF77FFD00212046FEF7B3FB462043
:10EF7000FBF778FD2046FFF791FF04464FF4CD7074
:10EF8000FBF770FDFBF792FD204610BDF8B52E494A
:10EF9000D1E90023541C43F10005C1E900452B4B86
:10EFA0001A685AB11A68012A15BF1A68284802F16E
:10EFB000FF32027008BF4FF47A721A60254B1A684C
:10EFC0009AB1186801280DD1234A127852B1234A08
:10EFD00012783AB9224A147824B9224C04F138053F
:10EFE000A56510701A68013A1A60D1E90001002382
:10EFF00000F01F02134326D11A4BD3F8B81011B3F7
:10F0000011F003041FD10A68174B9A421BD10E1D41
:10F0100001F12407012556F8040B38B1FFF73EFF34
:10F0200000B12C436D00BE42EDB2F4D191F8263010
:10F030005C4091F8243091F825202340134381F857
:10F04000253081F82440F8BD4851012034220120A8
:10F05000784A0120B4460120B8460120B946012073
:10F0600015510120804E012088480600F8B5134F45
:10F0700006460A25002447F00107002201213068D6
:10F08000FFF7A3FC4FF42070B84700213068FEF76B
:10F0900021FB42F20F713068FFF700FF28B9013DF4
:10F0A000ADB2002DE9D12046F8BD8C4202D8013422
:10F0B000A4B2F0E742F21074F5E700BF302F06006B
:10F0C00007B50121019001AA0248F9F78FFCFFF76B
:10F0D00041F800BF7470060008B5064B1B683BB1D1
:10F0E0001B681A68044B9A4202D00420FAF734F9DC
:10F0F00008BD00BF3C510120EF2978012DE9F04106
:10F100000025D0F800808D75836906460C46002BDB
:10F1100055D0C36A01330AD001F11607D8F8103070
:10F1200033F8150000284CD125440023AB7500238B
:10F13000A07D19462E27F5696A5C202A01F101019C
:10F1400021D0052A08BFE522092904D1E51800B914
:10F15000AF756F72013304EB030C8CF8092088B98A
:10F16000A2F14105192D0BD8F569082995F80CE095
:10F170008CBF102508251EEA050F1CBF2032D2B215
:10F180008CF8162001330B29D5D130B9E2189075CF
:10F19000F269127B002A08BF0023234400225A721E
:10F1A000F369DB7A2372F0691C30FAF769FA2060A0
:10F1B000F0691630FAF764FAE080000CA080BDE830
:10F1C000F0817F2802D9FAF7B1FA30B10135B5F5EF
:10F1D000807F02D007F8010BA0E70025A4E700001C
:10F1E000034B044801221A70034B00221A70704727
:10F1F000B84601206C5406001551012038B501466F
:10F2000000680E4C40F30730FAF7FAFC0B68002058
:10F21000D3F80022C3F800020B684FF0FF32C3F8A6
:10F2200008230A68012313610A790C2505FB0242B1
:10F2300013720B7905FB0343187238BD184D01207A
:10F24000104B98420CD003F10802904215D003F104
:10F250001002904213D01833984212D1032300E0D9
:10F260000023094A0021D1540379084A0C2101FBEB
:10F2700003231B7A2BB1FFF7C1BF0123F1E7022360
:10F28000EFE7704748220120DD500120184D012092
:10F2900043687BB15A681B7AC2F86035064A00237E
:10F2A00043601378013BDBB213701BB9034B186842
:10F2B000FFF7C6BF704700BF145101205451012011
:10F2C00008B5FFF7E5FF014808BD00BF6C54060014
:10F2D00008B50868FFF7DCFF004808BD6C5406005D
:10F2E00007B5400040F00100019001AA0121024849
:10F2F000F9F77CFBFEF72EFF5472060037B5044683
:10F30000F9F7E9FEC56815B91620FFF7E9FF01AB6B
:10F31000002201212046A847013001D10198F4E7DD
:10F32000014803B030BD00BF6C54060037B5044639
:10F33000F9F7D1FE01ABC568002204212046A84799
:10F34000013002D10198FFF7CBFF014803B030BD77
:10F350006C5406000868FFF7E9BF10B50446006862
:10F36000FFF7E4FF2046BDE81040FAF70BB8086845
:10F37000FFF7DCBF38B5044600F10803456800F12B
:10F380000C0101220068A847A36813B11846FFF7D3
:10F39000A7FF00B92073207B38BD08B5838803F030
:10F3A0003003302B02D11E20FFF79AFF08BD00006A
:10F3B0001FB50223009303ABF9F792FE039B23B121
:10F3C0000B2B08D01846FFF78BFF400040F00100E0
:10F3D00005B05DF804FB0148FAE700BF6C54060075
:10F3E000FFF7E6BF10B50446C068F9F7CBFF00236E
:10F3F000C4E901330148E36010BD00BF6C5406004E
:10F40000074B1A78C2F34000920708D51B785B07B8
:10F4100004D4044B187900F00100704700207047B5
:10F420006C45012024260120FFF7EABF08B5FFF74D
:10F43000FBFF034A034B00280CBF1046184608BDCB
:10F44000645406007054060038B50546FEF70AFEFF
:10F4500010B90024204638BD0620FEF7CDFD044635
:10F460000028F6D015F00302F4D1044B0C20C3F8A9
:10F470001C55C3F82025FAF7A3FFEBE700900240E4
:10F480002DE9F041194C236801332BD0184BDFF8DC
:10F4900064801B681E680120A6F58056002507467B
:10F4A000D8F8002007FA05F3134209D130B12068DB
:10F4B00006EB452100EB4520FFF75EFA00F0010066
:10F4C0000135082DECD170B12068FFF7BDFF002594
:10F4D00021687019294405F50075FFF74DFAB5F557
:10F4E000805FF5D10120BDE8F08100BF784901209F
:10F4F0007C4A0120804901202DE9F84F2E4D2B68D0
:10F500000133074606D1002F53D1FFF7A3F801209E
:10F51000BDE8F88FDFF8A490DFF8A4A000244FF036
:10F520000108D9F8002008FA04F3134211D1E600CB
:10F5300006F1080BDAF8C830286899594FF4807240
:10F5400000EB8610FEF7A0FD0028E1D00436B3459D
:10F55000F0D10134082CE4D12868DFF86490DFF89A
:10F5600064A0FFF771FF4FF000081FE0D9F8C83022
:10F57000286899594FF4807200EB8610FFF7B8F9AC
:10F5800057B9DAF800303BB9D9F8F83023B1D9F8D7
:10F59000C8309859F9F7F6FE0436B442E6D108F1BE
:10F5A0000208B8F1100F04F10804ACD04FEA880645
:10F5B000DCE73846ACE700BF7849012080490120EC
:10F5C000804E01204051012008B54368132118885E
:10F5D000FBF73CF8004808BD6C540600436843B193
:10F5E00019880548054B4FF6FF72914218BF18461F
:10F5F00070470148704700BF64540600705406000D
:10F6000073B5104D4FF46A244FF00106200B2E7095
:10F61000FAF7E4F908B9FAF7F3F904F58054B4F508
:10F62000722FF3D1084B019301A901224FF46A20F4
:10F63000FAF7F6F9012201A90448FAF7F1F902B044
:10F6400070BD00BF3951012031304442FC1F0F0012
:10F6500010B54FF6FF720446FF210120F9F7E6FFCF
:10F6600038B1033424F00304044B083404449C42AE
:10F6700002D9FFF7C5FF024810BD00BFFB1F0F00F6
:10F6800004A00E0008B5FFF7BBFF014808BD00BF8E
:10F690006C54060010B50446406818B1FBF74EF9EB
:10F6A00000236360004810BD6C54060008B590F854
:10F6B0002330FF2B01D0FBF753F9014808BD00BFF1
:10F6C0006C54060008B583680BB1FEF77BFF014858
:10F6D00008BD00BF6C54060008B5837FFF2B01D026
:10F6E000FBF789F9004808BD6C54060007B520B93E
:10F6F0000648F9F782F9FEF72DFD0B6803480193E0
:10F7000001AA0121F9F772F9F5E700BFBC73060001
:10F71000C28B4FF6FF739A420AD04368188A1728A3
:10F7200038BF1720033880B2400040F00100704716
:10F730000020F9E74FF01023D3F80C220379D20709
:10F7400003D5A3F10902012A0DD95909012203F0B9
:10F750001F0302FA03F3054A52F8212013420CBF9B
:10F760000120002070470020704700BF6C49012035
:10F77000084BD3F8183182B04BB1074B0748002231
:10F780001A601B680193019B02B0FAF79DBA02B0A0
:10F79000704700BF0030024018310240D04C0120B9
:10F7A00008B5044BC2689A4202D00430FEF72CFE22
:10F7B000004808BD6C54060038B543680246186816
:10F7C0001B790624C0F800451C4CC0F88815342568
:10F7D00005FB0343022483F82D400023C0F8443581
:10F7E000C0F84835012303628360D0F850311BB95B
:10F7F000D0F82431002BF8D04FF4A871FAF7C2FAF0
:10F8000001234361D0F80431002BFBD04FF4827107
:10F81000FAF7B8FAD0F824316BB14FF49271FAF7D5
:10F82000B1FAD0F8C434C0F8C43400245068FAF7F0
:10F830009FFC204638BD0124F8E700BF304D012071
:10F840002DE9F04F89B005469DF8487016465FFADD
:10F8500081F81C464BB94146FFF7AEFF002814BFA4
:10F860000020132009B0BDE8F08F426813791268B8
:10F870000621C2F800151C4A342101FB0323002F86
:10F880004FF0020183F82D10914614BF002320236E
:10F890004FF0000A4FF6FF77A74228BF2746CDE971
:10F8A000047ACDE9066A69688DF80CA008798DF8AC
:10F8B0000D804FF0340C0968019303AA00FB0C90F3
:10F8C000FAF79EFA094B9842834603D1E41B019B49
:10F8D0003E44DFD16868FAF74BFC584609B0BDE8F2
:10F8E000F04FFAF7FBBF00BF304D01200000AD0B19
:10F8F0002DE9F04700248AB0CDE904445F4B60480D
:10F900006049012225461E6846B1D0F804631642BC
:10F9100004D01D601E680196019E144304338B427F
:10F920004FEA4202EFD1584B1A687AB100221A60AE
:10F930001B680293029B4FF0A04344F00044D3F8AD
:10F9400010350493514BD3F81035059314F0FF0F85
:10F950001AD04F4F01260025344210D0AB0003F1DE
:10F96000804303F5C043D3F81005D3F8101557F8BA
:10F97000253023B1C1F30141C0F30520984701357B
:10F98000082D4FEA4606E7D1002C70DA08AF0023B5
:10F9900008937B604FF0FF33CDE906333C4EDFF830
:10F9A000EC904FF0010896F9543096F8542001334A
:10F9B00022F0C0045BD00AAB03EBD40102F0070ACB
:10F9C00011F8103C23FA0AF3D8074FEAD40C4ED5AD
:10F9D0003319920993F9243056F823504DB9032A6C
:10F9E00045D117F80C0008FA0AF3034307F80C3066
:10F9F00001E0032AF5D003A80394FAF723F9039B47
:10FA000011F8181C03F5E07321FA0AF150F82330BD
:10FA1000C907C3F3014307D5022B28D1032A1CD001
:10FA20002DB34FF0000A1CE0032B20D1032AF7D19D
:10FA300002212046FAF772FC8DB94FF0A0430499D9
:10FA4000D3F81025D9F81035914213D00492089AB2
:10FA5000CDE90532099B0793A5E71146E9E74FF089
:10FA6000010A11462046A847BAF1000FE5D10AB0B5
:10FA7000BDE8F08705999942F9D0E7E700610040B9
:10FA800000600040206100407C61004000030050A5
:10FA9000E04D01202DE9F04F0025DFF8A0B085B042
:10FAA00004460E4690464FF4803700F5A079AA46EA
:10FAB000D4F804333B4210D059F825306BB1C4F868
:10FAC0004873C4F8087349F825A059F82530019304
:10FAD000019B5BF82630E8B298470135A8454FEA0C
:10FAE0004707E5D1D4F80433DA070ED5D4F800314E
:10FAF0005BB10023C4F80031D4F800310293029BBB
:10FB00000E4B042053F826309847D4F804339B0753
:10FB100011D5D4F8043173B10023C4F80431D4F8FA
:10FB200004310393039B054B53F82630052005B0A1
:10FB3000BDE8F04F184705B0BDE8F08F604E0120DA
:10FB4000024803220021FFF7A5BF00BF00B000401C
:10FB5000024804220121FFF79DBF00BF00100140B1
:10FB6000024804220221FFF795BF00BF0040024077
:10FB700010B4C3685A8B9B8B1344828E541C1A4456
:10FB800043798486042B04BFC36B43F822101721EA
:10FB90005DF8044BF8F78EB938B50D460121F8F73A
:10FBA000F1F92946BDE83840FFF7E2BF8968806A6D
:10FBB000FFF7F2BF38B50D4601210446F8F7E2F928
:10FBC0000E2D09D00F2D09D00D2D09D11021204661
:10FBD000BDE83840F8F766B91121F8E71221F6E7D9
:10FBE000BDE838400149FFF7C3BF00BF38540600E5
:10FBF000F0B54468164D2668A468A14228BF214686
:10FC0000002455F83470B94209D305EBC404616887
:10FC1000C6F824152AB9003B18BF012305E00134BA
:10FC2000EFE7002B14BF032302234268022B126864
:10FC300009D0032B09D0012B14BF00230223C2F8E3
:10FC400054350120F0BD0423F9E70623F7E700BF90
:10FC5000DC16060070B543681E7A044686B9012595
:10FC60001D7290F8313090F83020C16A4068FFF77B
:10FC7000BFFF04F11C003146FEF7A0FE284670BD10
:10FC80000020FCE738B50D4B04460425002253F84C
:10FC9000041B8C4208BF43F8042C013DF7D1A36834
:10FCA00001225A60E068E57784F82050F9F76AFB92
:10FCB0002069E560F9F766FB256138BD64460120DF
:10FCC00038B5084B1B6800250446C3F80055007979
:10FCD000FAF722FE60792571FAF71EFE0248657177
:10FCE00038BD00BF442201206C540600830710B5C4
:10FCF000014611D102680E4B9A420DD10D4B0340C3
:10FD0000062B07D1C008F7F79BFC4078400040F075
:10FD1000010010BD8068F9E70846F8F765FD436902
:10FD20001BB1BDE81040052018471846F1E700BF99
:10FD300040770600070080FF38B5154B984204460F
:10FD400023D0144DA84201D1012038BD124B984256
:10FD50001BD0C20704D5430814BF01200020F4E7DC
:10FD6000F8F742FD43693BB121460420984718B19A
:10FD7000431B58425841E8E72046FFF7B7FF0028E9
:10FD8000E2D0013818BF0120DFE70020DDE700BF27
:10FD900064540600705406006C54060010B5044606
:10FDA0000846FFF7C9FF2071004810BD6C540600DB
:10FDB000D1E9023249685B1A1344002ACCBF03F12F
:10FDC000FF330133042893FBF2F303D0052807D057
:10FDD00000207047054A0648002BC8BF10467047F0
:10FDE00023EAE370400040F00100704770540600C1
:10FDF0006454060010B5104A11F07F044FEAD11088
:10FE00000BBF012341F480715365C2F81815BFF38D
:10FE10006F8FBFF34F8F094B03EB4403034493F8F9
:10FE2000212042F0020283F8212093F8212042F0A1
:10FE3000010283F8212010BD007002406C450120B2
:10FE4000F8B5069D3C264FF461676E435F434D1E37
:10FE5000144B33F8155002290446154403D9F9F719
:10FE6000B9FC00B10135A4F2CD726FF4C863E1189A
:10FE70004FF4C870B1FBF0F101EB92010A4BA4F210
:10FE80006D726420B2FBF0F20798891A0D4407499D
:10FE900003FB0404214439440548314400FB0510A8
:10FEA000F8BD00BF402E06008033E10180569C5013
:10FEB000805101002DE9F04190F82E30448D264EFE
:10FEC000264FDFF89C806FF30003054680F82E3044
:10FED000013C631C01D1BDE8F0816B6853F834002C
:10FEE000830726D10368B34230D1B0F93830B0F976
:10FEF0003C2093421FD090F8511089071BD0838774
:10FF000090F8503023F0070380F85030836813F0E6
:10FF1000030105D1DFF84CC01A68624508BF1973A8
:10FF2000436813F0030204D11968414501D19A8254
:10FF30001A83013CCDE790F85010490701D4934251
:10FF4000DED1436C8363836CC363D9E7BB42F0D1DA
:10FF5000FFF7B0FFEDE700BF883C060064380600FD
:10FF6000D0330600703A0600062837B50C4619D182
:10FF70008D680D4B2B40062B12D1E808F7F760FB7C
:10FF8000007830B901A92846F8F7A4FE0199F7F7DF
:10FF900065FB23795840400040F0010003B030BDBC
:10FFA0006868EEE70020F9E7070080FF38B50446EF
:10FFB000FAF754FA236906480122002583F8212024
:10FFC0005D602169F9F71AFB0248256138BD00BF61
:10FFD000E15903006C540600F7B504460D46F9F7E5
:10FFE000FFFC58B34E4E0127200B3770F9F7F6FC93
:10FFF00010B1002003B0F0BDF9F702FD0228F8D0DF
:020000023000CC
:100000004FF40072294620463770F9F7E5FC0028C6
:10001000EFD1F9F7F5FC0228EBD04FF4007205F5AB
:10002000006104F500603770F9F7D6FC0028E0D1D4
:10003000F9F7E6FC023818BF0120DBE74FF08053E8
:100040001A69B4FBF2F302FB134363B9354B022286
:10005000C3F80425C3F80845D3F80024D007FBD51E
:100060000022C3F804252F4B0122C3F8042514F005
:10007000030351D04FF0FF32C3F10400019201AAF3
:100080002946E61A1A44054411F8017B02F8017B5F
:10009000A942F9D1019A234FD7F80014C907FBD51B
:1000A0003260BFF35F8F03F6FC7304449908DFF8F6
:1000B00074C02E1F04EB8101224656F8047FDCF841
:1000C000000410F00100FAD042F8047BBFF35F8F08
:1000D0009142F2D199071AD023F003024FF0FF3674
:1000E000A118019604F0030401AE2A4434441D44CF
:1000F00012F8013B04F8013B9542F9D1019B094CF0
:10010000D4F80024D207FBD50B60BFF35F8F054BFB
:100110000022C3F804256DE74FF48053C6E700BF03
:100120003951012000E001402DE9F043DFF8A480BF
:10013000DFF8A49085B005460C46002701266B8D9C
:10014000BB4217D895F82E30DB070ED5002E3BD0DA
:10015000B5F918302380B5F91A306380B5F91C3031
:10016000A380B5F91E30E380002686F0010005B0BB
:10017000BDE8F0836B6853F8370082070FD103683E
:10018000434513D1B0F93C20B0F93830934214D034
:10019000836B0193C38FADF80820ADF80A3076B1B8
:1001A000019B2360029B6360002606E04B45F6D16D
:1001B00001A9FFF7B9FF0028F1D10137BFE701A975
:1001C0002046FBF743FBEFE705F118012046FBF75C
:1001D0003DFBCAE7883C060064380600F0B543687A
:1001E00053F8314014F0030785B005462CD123683D
:1001F000204A93422AD1B4F93C30B4F938209A42CB
:100200001EBFADF80830E38FADF80A3094F85030D7
:100210001CBFA26B01926FF3041384F850304FF0AF
:10022000000314BF01263E46A3626EB195F82E303E
:10023000DB0718D4019BAB61029BEB6195F82E3074
:1002400043F0010385F82E3005B0F0BD0A4A934211
:10025000FAD101A92046FFF767FF39460646204636
:10026000FBF7BCFAE1E701A905F11800FBF7EEFA8C
:10027000E4E700BF883C06006438060070B5438D93
:10028000013B4385436803EBC10304465E680D46AA
:10029000FFF7A4FF618D6368A94209D8002243F8E3
:1002A0003120618D636803EBC10330465A6070BD35
:1002B000013503EBC50393E8030003E90300E9E715
:1002C00008B5074BD3F8C83033B9FFF7D9F8054B59
:1002D0004FF0FF321A6008BD0120FFF70DF9F6E775
:1002E000804E01207849012008B50A4B4FF47A72FC
:1002F0001A60FFF7E5FF084BD3F8C83033B9FFF7B2
:10030000BFF8064B4FF0FF321A6008BD0020FFF720
:10031000F3F8F6E734220120804E012078490120CD
:1003200008B5FFF7E1FFF9F705F87FB5D0F82461CC
:1003300005460C46002E5CD04FF49271F9F772FF1F
:1003400002238DF80030D0F88034C0F88034039355
:10035000D0F83C350293E36801930023C4E90633E7
:100360006846D4E900139847D5F844317BB14FF47F
:10037000A2712846F9F756FFA36943B10023C4E9E7
:100380000633E268D5F83C152046F9F753FFD5F857
:100390002031ABB14FF490712846F9F743FF0123A8
:1003A000EB60636963B1D5F84C2502920023A26823
:1003B0008DF8003063610192D4E9001368469847D4
:1003C000D5F858319BB14FF4AC712846F9F72AFFA4
:1003D000636963B1D5F84C2502920023A2688DF8B9
:1003E000003063610192D4E900136846984704B075
:1003F00070BDD0F81031002BB6D04FF48871F9F7EA
:1004000011FFA169D0F83C359942ADD1E369E268AA
:1004100073B1D0F8003223F02003C0F80032E36952
:10042000A3612369E360E6612046F9F703FF9BE7D8
:10043000A361F9E701490248FFF777BF984D012012
:100440000020004001490248FFF76FBFBC4D01206A
:10045000008002402DE9F84F1E460379D2F8009043
:100460000F780D46A3B3B2F80AA0B2F80CB050460C
:100470005946FBF745F8594680460AF12100FBF73B
:100480003FF80BF1210104465046FBF739F8102FD5
:100490004FEA194CC9F307225FFA89F321D100F022
:1004A0000700034408F00708FF2BE04428BFFF23A0
:1004B00004F00304B8F1FF0F28BF4FF0FF08144405
:1004C000FF2C28BFFF24240244EA084444EA03091D
:1004D000102F1BD14846FBF737F8306001233371EA
:1004E00051E0FF213941084053FA80F308EA01083E
:1004F000FF2B5CFA88F828BFFF230C40B8F1FF0FF0
:1005000028BF4FF0FF0852FA84F4D9E76B79002B2B
:1005100040D04846FBF724F8C7F1080738414FEAB6
:10052000194230605FFA89F08242144638BF0446AF
:1005300082421346C9F3072128BF03468B4228BFD6
:100540000B468C422CBFC3EB0403C3EB0103DBB2AD
:10055000102B2C7903D8002CC0D13460BEE748465C
:10056000FBF712F8AB78181A80B200F10A039BB2BD
:10057000142B05D900B210F1DB0F01DBDB2806DDFF
:100580001CB100233360BDE8F88F0123FAE7002C8B
:10059000F9D1F6E72B7953B1082F08D84846FAF776
:1005A000DFFFC7F1080740FA07F7376096E7002337
:1005B00095E7000079B3F8B5041F174E04EB8105E9
:1005C000032754F8040F030719D1D6F8F8309842DE
:1005D00015D3D6F8FC20904211D2C01A48BF0F3074
:1005E0000011D6F8ECC0810800F003031CF801E00C
:1005F0005B004EFA03F202F00302012A02D0A54288
:10060000DFD1F8BD07FA03F343EA0E030CF801301B
:10061000F6F738FFF3E77047804E0120F8B52E4C0F
:10062000B4F8083200220133A4F80832C4F80421D7
:10063000251D04F1D806032755F8040F020719D128
:10064000D4F8F830984215D3D4F8FC20904211D257
:10065000C01A48BF0F300011D4F8ECC0810800F078
:1006600003031CF801E05B004EFA03F202F0030200
:10067000012A1FD0AE42DFD1D4F83002030718D1CF
:10068000D4F8F830984214D3D4F8FC20904210D219
:10069000C01A48BF0F300011D4F8EC40810800F0B8
:1006A0000303655C5B0045FA03F202F00302012AD2
:1006B00009D0F8BD07FA03F343EA0E030CF8013042
:1006C000F6F7E0FED6E7032202FA03F31D43655472
:1006D000BDE8F840F6F7D6BE804E012003071CD1D6
:1006E000124BD3F8F820904217D3D3F8FC1088426D
:1006F00013D230B4801A48BF0F300011D3F8EC4049
:10070000810800F00303655C5B0045FA03F202F028
:100710000302012A02D030BC70477047032202FA5C
:1007200003F31D43655430BCF6F7ACBE804E012088
:1007300010F00F021DD11849D1F8F830984219D3A2
:1007400010B4D1F8FC40A0420FD2C31A48BF0F33F7
:100750001B11D1F8EC40990803F00300615C4000E4
:10076000014101F00301012906D010465DF8044B58
:10077000704700221046704701329918880801F02E
:100780000301205C490040FA01F101F00301022954
:10079000F2D01201E9E700BF804E012021F00F01E5
:1007A0002DE9F843384A394C0F1AFF00A2FB0732F3
:1007B0004FEA5228A1EB881C4FEA8806C4E93EC1E3
:1007C000073600EB080310F00301C4E93C834FEA4D
:1007D000D609C4F8EC0042D0B7F5037F36D34246C1
:1007E000002104F0FFF8D4F8F43013F003012DD108
:1007F000760906D0B6001846324604F0F3F80346F0
:10080000334419F0020F1CBF002223F8022B19F009
:10081000010F01D000221A70202200211C4804F090
:10082000E1F8D4F8F020D4F8F830501E03EB82132E
:1008300001210022C4F82C02C4F80031A4F80822D7
:10084000C4F8302284F80A12BDE8F883B9F1000F29
:10085000E2D04A461846002104F0C4F8DCE7D20A88
:10086000054604D097003A4604F0BCF83D4418F021
:10087000020F1CBF002325F8023B18F0010FB2D075
:1008800000232B70AFE700BFF32C23FA804E01202A
:100890008C50012008B510F00103024663D03D28BA
:1008A0004FEA600307DC0C2B17DC022B4ED0052B24
:1008B0004ED0012B4ED02D49002301EBC3004068E0
:1008C00082424BD151F83300C008F6F7D7FE0378C7
:1008D000002B014608BF002130E00D3B112BEAD868
:1008E00001A050F823F000BF55090300B70803002A
:1008F000B7080300B708030059090300B70803004D
:1009000031090300B7080300B708030041090300D9
:10091000B7080300B7080300B7080300B7080300CF
:10092000B708030045090300B7080300490903009D
:100930000F480388322BBED8F8F780FD084608BD63
:100940000C48F6E70C48F4E70C48F2E70C48F0E7EF
:100950000C48EEE70C48ECE70C48EAE70133172BAC
:10096000ABD10021EAE71946E8E700BF045D0600C5
:1009700066AA060064AD06007CAE0600B4B80600A8
:1009800016AD060040C6060060C50600C4B80600E5
:10099000836813F9012B002AFBDB13F9012B002AD2
:1009A000FBDB043313F9012B002AFBDB18887047AB
:1009B000136810B514463BB92B2905D1FFF7E8FFA2
:1009C000C00040F00600206010BD136810B514464A
:1009D00043B92B2907D14068FFF7DAFFC00040F088
:1009E0000600206010BD162904BF43681360F9E7B4
:1009F000024B1A690260186100207047804E012086
:100A000040EA0103F0B59C0709D0431E0A44914215
:100A100000D1F0BD11F8014B03F8014FF7E722F0C8
:100A20000303051F9608CC18A1420DD1910744BFBE
:100A300034F8021B20F82610034448BF0233D207C3
:100A400044BF22781A70E4E751F8047B45F8047F2C
:100A5000EAE713B504460193104629B9224601A9D5
:100A6000FFF7CEFF02B010BD01AB23441444A242F5
:100A7000F8D013F8011D02F8011BF8E738B54568F6
:100A80009542044628BF15462A460068FFF7B8FF7E
:100A9000236862682B44521B2360626038BD0000EB
:100AA0002DE9F84F0346002940F0B180421E0C4664
:100AB00000F2BD1002F8014F8242FBD1834A126856
:100AC000106883F8BE41A0F58050440A1FBFFF2282
:100AD00083F8BF2183F8C02183F8C1214FF00102C0
:100AE00002BF83F8BF4183F8C04183F8C14183F856
:100AF000C221002C40F0838083F8C34183F8C441B5
:100B000083F8C541012283F8C62183F8CA41002237
:100B1000440C400E83F8C72183F8C82183F8C9210B
:100B200083F8CD2183F8CE2183F8CF2183F8D0211B
:100B300083F8D12183F8D22183F8D32183F8D421FB
:100B400083F8D52183F8D62183F8D72183F8D821DB
:100B500083F8D92183F8DA2183F8DB2183F8DC21BB
:100B600083F8DD2183F8DE2183F8DF2183F8E0219B
:100B700083F8E12183F8E22183F8E32183F8E4217B
:100B800083F8E52183F8CB4183F8CC0183F8E62193
:100B900083F8E72183F8E82183F8E92183F8EA2143
:100BA00083F8EB2183F8EC2183F8ED2183F8EE2123
:100BB00083F8EF2183F8F02183F8F12183F8F22103
:100BC00083F8F32183F8F42183F8F52183F8F621E3
:100BD00083F8F72183F8F82183F8F92183F8FA21C3
:100BE00083F8FB2183F8FC2183F8FD21552283F84B
:100BF000FE21AA2283F8FF210846BDE8F88FFF22D4
:100C000083F8C32183F8C42183F8C5217AE7013A28
:100C10002E4FDFF8C080DFF8C0904E1E04465518F6
:100C2000AE4201D10021E7E73B681868A0F5805C7F
:100C3000B6EB5C2F01D30121DEE7D9F8002008EAEA
:100C4000462393424FEA46203BD100280346B8BFD3
:100C500000F2FF135B125A4202F0070203F007038F
:100C60001B4958BF5342DBB2012209689A40D2B2F5
:100C70000A4226D0DFF864A0DAF8C810B9B14FEA0A
:100C8000430B4FF4807251F82B102046FFF7B8FE4B
:100C9000DAF8C8100BF101034FF4807251F82310F9
:100CA000A018FFF7ADFE04F500740136B8E74FF465
:100CB000007221460CEB4320FDF7E6F90028F2D143
:100CC000B9E74FF400722146F6E700BF7C4A0120E5
:100CD0008049012000F0FFFF78490120804E01206B
:100CE00010B58389C288044600689BB202FB0300EA
:100CF000FFF786FEA389A1889BB20133B3FBF1F213
:100D000001FB12339BB2A38163899BB2994215BF49
:100D10006389A38901339BB216BF9BB2E3816381D0
:100D200010BDF8B5037A04460E46154633B942891C
:100D300083889B1A9BB29D4228BF1D460027BBB2E9
:100D40009D4201D82846F8BD31462046FFF7C8FF2E
:100D5000E38801371E44F2E738B50446154632B938
:100D60000378012B02BF104B8022C3F88420E38953
:100D700022899BB29A4204F1040001D1237B73B112
:100D8000FFF7AEFF75B901252378012B02BF064B93
:100D900080225A6035B9BDE83840F8F7ABBB002D6A
:100DA000F9D1F1E7012038BD00E100E04378023BD2
:100DB0000A46032B10D8DFE803F00225141C124B5F
:100DC00019786FF30001197019786FF341011970E8
:100DD00019786FF3820119700C4B01461868FFF700
:100DE000BBBF094B1978C9070CD5197841F004012C
:100DF000F1E705490B78DB0704D50B786FF3820325
:100E00000B70E9E7704700BF6C450120A045012049
:100E10001FB50023CDE9013301218DF8050001A89C
:100E200003938DF80430FFF7C1FF05B05DF804FBB4
:100E3000012813B5044600F0A18002284DD1634B70
:100E4000D3F800241205FBD54FF40062C3F8002448
:100E5000BFF36F8FBFF34F8F5D4B1B68082B0AD119
:100E60005C4B5D4A1868002840F0828049F2753179
:100E7000196010601960F8F793FE48B1554B574A56
:100E80001868002877D149F275311960106019602F
:100E90004F4B1B68082B09D1514B40F2E3721A608B
:100EA00040225A60BFF36F8FBFF34F8F474C4D49BD
:100EB0008022C4F81C25C4F804134B49C1F88421CE
:100EC0004A60F8F783FE0028FBD00123C4F80435FC
:100ED000BFF36F8FBFF34F8F48E0002846D13B4BE5
:100EE000D3F80025002A41D14FF40062C3F8002452
:100EF000BFF36F8FBFF34F8FF8F752FE48B1354BFA
:100F0000364A1868032128BB49F275301860116011
:100F100018602F4B1B68082B09D12E4B2E4A1868DE
:100F2000C021C8B949F27530186011601860274BAC
:100F30000124C3F80045BFF36F8FBFF34F8FF8F75D
:100F400045FE98B9F8F74CFD40B102B0BDE810403D
:100F5000F8F736BE1160DCE71160E8E7234B186054
:100F60001B680193019B4FF080431C6002B010BDD1
:100F7000002313607FE70023136089E7134BD3F846
:100F80000025002AF2D00022C3F80425BFF36F8F9A
:100F9000BFF34F8F14498020C1F88400D3F80013A9
:100FA000C3F80813C3F80025BFF36F8FBFF34F8F4B
:100FB000F8F716FD38B1F8F705FE022002B0BDE8DB
:100FC0001040FFF725BF0A4B1C60F6E70070024097
:100FD0003001001000EC064014EC064014ED064011
:100FE000007802400514800100E100E000010040AB
:100FF0000400004013B5274C402384F827330DF13B
:10100000030000238DF80330F8F7C4FA9DF803308D
:10101000EBB10120F8F7B8FA0120F8F7B3FA012094
:10102000F8F7B4FA01A8F8F7B3FA1B4B1A7862B1D3
:1010300000201870019BDA0701D5FFF7F9FE019B2C
:101040009B0702D50220FFF7F3FE02B010BD134B41
:101050001A788AB94FF08041C1F88025C1F8782507
:101060002268D10706D4E02284F800230122C4F8C4
:101070008021226001221A70094B0A4A1A604FF03F
:1010800080434FF46072C3F80423D3F838340193DB
:10109000CBE700BF00E100E038220120DC50012056
:1010A000744E0120310E03001FB50024CDE9014428
:1010B0008DF8040007208DF805008DF8081001A8B0
:1010C000194603928DF80940FFF770FE04B010BD79
:1010D0001FB5124B93F8C020BAB1114A5268C2F33F
:1010E000080272B10023019308238DF805300D4BDF
:1010F0000121CDE9023001A8FFF758FE05B05DF8E7
:1011000004FB93F8C020002AFBD1012283F8C02001
:101110000260BFF36F8FBFF34F8FEFE7E82E012020
:1011200000ED00E0D1100300F8B5104D104E00F5B1
:101130009473182455F823304443142202FB0052C0
:10114000DDB20C4B3159C2F8001703EB8000C2F836
:101150000457FFF7BDFF335937192B443351FB8830
:1011600015FA83F39BB2FB80F8BD00BF007002400C
:10117000E82E01202870024010B4104B182101FB0A
:1011800000314A8A0B8ACC689B1A0A7D9BB2934233
:1011900028BF13461422424302F1804202F51C325A
:1011A000C2F80046C2F804362344CB60044B5DF815
:1011B000044B03EB8000FFF78BBF00BFE82E01203C
:1011C00004700240F8B50446182300F07F001E4D5D
:1011D0001646E70903FB00F20C2303FB0723EA187A
:1011E000E95000239680D3802A4698B996B91748CB
:1011F000FFF76EFF95F8C0304BB9F8F7B9F9002347
:101200001A4621461846FFF74FFF0120F8BD85F822
:10121000C060F4E7AFB9182303FB00235B7A13B176
:10122000FFF782FFF1E70A4B30B90122DA64BFF31E
:101230006F8FBFF34F8FE8E700F5947043F820708D
:10124000F5E7FFF799FFE0E7E82E01205070024034
:101250000070024010B50C46204611461A46FFF7B2
:10126000B1FF60B1064B04F07F0103EB410303EBD8
:10127000D41191F8213043F0010381F8213010BDE1
:101280006C450120F7B58B79062B06460C461746B0
:1012900002D1CB79502B08D0154B1B68DA0702D44A
:1012A000002003B0F0BD00BEFAE7124D097805F149
:1012B0002E03019305F12F03009302231A462144C4
:1012C000FCF768FB28B90A4B1B68DB07E8D500BEB2
:1012D000E7E7A37885F82D3017233B8095F82F108A
:1012E0001F232A463046FFF7B5FF0028D9D1EAE789
:1012F000F0ED00E00C44012070B4104A104B4FF4A4
:101300000B6444431519E97801F07F0003EB4003B7
:1013100003EBD11393F8210010F001000CD16E8B78
:10132000AB8A9B1B9BB23F2B06D904F50364224476
:10133000402370BCFFF78EBF70BC7047242601208D
:101340006C450120F7B58B79022B0746154607D06F
:10135000274B1B68DB0700D500BE002003B0F0BDA3
:10136000CB79073BDBB2F72BF2D9224EB378002BB7
:10137000EED18B7833700C7809230C44138005E090
:1013800023782A8813442B8023781C446378242BE9
:10139000F6D0052B11D12046FCF7CAFA28B9144B18
:1013A0001B68DA07D9D500BED8E7A3787370237815
:1013B0002A8813442B8023781C446378042B12D191
:1013C00063790A2B0FD10C4B2178019301330093E1
:1013D00002231A4621443846FCF7DCFA0028DED006
:1013E0002B8817332B800020FFF786FF0120B5E7FD
:1013F000F0ED00E0242601202626012008B5084B48
:101400001B6899420AD1074B002058839883D883E0
:10141000FFF772FF044B03F128029A6508BD00BF75
:101420007C4E012024260120804E0120F8B51A4A66
:10143000D0788842144612D11646D51802F110070A
:10144000AE4211D1154B2BB1638B9BB213B100206F
:10145000AFF300800020FFF74FFF012003E09378F7
:101460005B1A58425841F8BD638BA28A9BB29A42DC
:1014700006F5036101D1237E13B13846FFF730FC36
:101480006379FF2B06D096F83018994202D10020DC
:10149000FFF7B4FF0136D3E7242601200000000047
:1014A00008B5074A93788B4208D110231832FFF70A
:1014B000D1FE20B9BDE80840F8F71CB8002008BDEF
:1014C000AC2F01202DE9F341244B5C7807460D46F3
:1014D00090461E46002C3BD10A781144996291F83F
:1014E00001C0BCF1210F0BD1AC5C5A1C023301923C
:1014F000009321442A790323FCF74CFA044650B99F
:10150000174B1B68DA0704D40024204602B0BDE85C
:10151000F08100BEF9E7AB79012B04BFEB79F370E2
:1015200000233371AB783370B36AB3F80730F380BC
:101530002B79C3EBC3031233A8F80030B17800292C
:10154000E3D0084A10233846FFF784FE0028DCD198
:10155000034B1B68DB07D7D500BED5E7AC2F0120B6
:10156000F0ED00E0C42F01202DE9F8431A4C1D4690
:10157000A3788B42064611D115F0030705D104F27A
:101580002D1904F10408BD420BD8144AA178402358
:101590003046FFF75FFE08B9F7F7EAFF0020BDE825
:1015A000F88319F8012C02F00F03052B12D00F2B32
:1015B00010D002F00B02022A04D00C3B012B94BF86
:1015C0000222032249464046FFF7ABFB043709F1EC
:1015D0000409D8E70122F5E7503201207C330120CD
:1015E0002DE9F8438B79012B80460D46164608D12C
:1015F0000A7809213180AA5C0A4432801846BDE885
:10160000F883032B01D00020F9E7CB79002BFAD126
:101610001E4F97F80190BA7859EA020934D18B78B5
:101620003B700C7809230C4433802B794B4508D848
:10163000174AB97840234046FFF70CFE0028DED158
:1016400006E06378052B18D12046FCF771F928B91C
:10165000104B1B68DB07D6D500BED0E7A378DA09AC
:1016600014BF7B70BB702378328813443380237897
:1016700009F101091C445FFA89F92378328813447F
:10168000338023781C44D0E71B70FFDE50320120EA
:101690007C330120F0ED00E010B5154A0446507B84
:1016A000F7F78AFF936892F82F1068B993620123C5
:1016B00082F82C3042F2077382F83E00938720466E
:1016C000BDE81040FEF796BB926B9B1AB3F5805FA6
:1016D00028BF4FF48053074A9BB22046FFF7BAFD5C
:1016E00020B9054B1B68DB0700D500BE10BD00BF4D
:1016F0000C4401200C340120F0ED00E010B40A4C41
:1017000008680B464968224603C20022C4E9022247
:1017100093F900305DF8044B93421146ACBF802032
:101720001046FFF74FBD00BFD42E012013B5124B5A
:101730009889D98993F90040421A92B2402A28BF69
:101740004022002C0EDA884212D099680B48019290
:10175000FFF756F90949019A802002B0BDE8104010
:10176000FFF730BD88424FF0000003D10021F4E7BD
:101770008020FBE70149F0E7D42E01202C45012011
:10178000F8B51B4E0D46844608684968B260374676
:1017900003C714460022F281E9888B4228BF0B461A
:1017A000B381A3B13CB9134B1B68DA0701D4002005
:1017B000F8BD00BEFBE76046FFF7B8FF08B10120A7
:1017C000F6E70C4B1B68DB07F1D500BEF0E795F997
:1017D0000020002AACBF802000201A461946FFF7DF
:1017E000F1FC0028EBD1BDE8F840F7F783BE00BF5D
:1017F000D42E0120F0ED00E037B50B7803F0600344
:10180000202B05460C4621D14B78FE2B06D0FF2B12
:101810001CD1FFF773FF012003B030BD01238DF809
:1018200007300B4B1BB1AFF300808DF807009DF81C
:1018300007000028F0D0431E8DF807300DF1070295
:10184000012321462846FFF79BFFE4E70020E3E75A
:101850000000000038B50B7803F06003202B0C4625
:1018600009D10F4A8B8815789D4204D14B78212BE2
:1018700003D81F2B0ED8002011E0222BFBD14B8860
:101880001371FFF73BFF608810F0010007D1FCF7F0
:101890003DF803E007230632FFF772FF012038BD51
:1018A00024260120F0B50B7803F01F05012D85B02B
:1018B00006460C4601D000201AE04A4A8F8892F86A
:1018C00000C0FFB2BC4517466AD0474B1B68DB0718
:1018D000F1D500BEEFE76378062BECD163881B0AD5
:1018E000212B07D1926A002AE5D01378FFF748FF31
:1018F00005B0F0BD222BDED1D3883C4AFFF740FF74
:1019000035E063881A0A012ADFD1DAB2384B0021A8
:1019100018461D7A954210D10C22E388019302FBF0
:1019200001011A4649683348FFF76AF8019B002B0A
:10193000CBD0304A21463046E0E70131042903F19B
:101940000C03E6D100235B68FFDEE388102BB2D8DE
:10195000294AEFE76088294B000A78711BB1AFF381
:1019600000800028A7D021463046FFF7C7FE01209F
:10197000BEE7234A0123DDE73B79C3F101038DF87C
:101980000F300DF10F020123D4E760881D4B0138A1
:1019900018BF01203871002BE5D0AFF30080E2E7DB
:1019A00013F0600397D0202B85D16378013B0A2B7D
:1019B00081D801A252F823F0031903007319030020
:1019C00079190300B7180300B7180300B71803000C
:1019D000B7180300B71803004B190300551903008B
:1019E0008B190300AC2F0120F0ED00E094490600B4
:1019F0008C230120B42F0120C42F012000000000FF
:101A0000B12F012000000000F7B50E46144600F18A
:101A100008054FF0FF37042C2246314628BF042228
:101A200001A80197FEF7ECFF012201A92846F7F76C
:101A3000F7FF042C04D9043CA4B204360435EAE7C9
:101A400003B0F0BDF7B50288112A04460D464FF0E9
:101A5000000344D0262A40D0102A64D1334988207C
:101A60004FF6FF760A4600FB03F77F5AB74203D0D2
:101A70000133052BF7D104232D4E88204343D11881
:101A8000A088D6F8D070D0522A48C865C1E918712C
:101A90000020294F81F85A00A1F876008F6603F1E3
:101AA00060011144C6F8D01004F10801A86151F892
:101AB000080F6C334968134403C36846F8F7C6FC43
:101AC000BDF80030228A9A4202D8628A9A4203D232
:101AD000A0886946F8F7B4FC0023EB6020E0134AC5
:101AE00081881746882000FB03F6B65A8E4203D041
:101AF0000133052BF7D1042388265E43B9190E481C
:101B0000F7F77CFD4FF6FF73BB530023CA6D81F8D6
:101B10005A3008498A421EBF5360217A1172AB6164
:101B2000012003B0F0BD1846FBE700BFC04601200E
:101B3000804E01206C5406009951030038B503888B
:101B4000362B0C4615D1B1B182888B899A4212D1BD
:101B5000C388CB81C5894A68954228BF154600F1E4
:101B600010012A462068FEF74BFF0120A560207473
:101B700038BD0020FCE70120FAE700002DE9F04F16
:101B800015464268DFF860A01368DFF86080DFF870
:101B900060B087B081460E4601930DB901201BE06D
:101BA000D9F80420019BD768AF4228BF2F46534580
:101BB00015D13A4631464046FEF722FF4246D9F853
:101BC0000400002402A9CDE90227CDE90444FBF773
:101BD0008FFD584505D0204607B0BDE8F08F32464E
:101BE000EDE73E44ED1BD8E700F002400000012085
:101BF0000000AD0BF8B51C464B1E59421746594123
:101C000005461430069EFCF7D9FE012F17D1264455
:101C100005F11C07B44200D1F8BD012221466868D5
:101C2000FFF7ACFF01213846FCF7C8FE0120F8F7AA
:101C300019FF00213846FCF7C1FE0134EAE7686865
:101C400032462146BDE8F840FFF798BFF0B5ADF544
:101C5000805D81B0044617461E460D4649B9B2F56F
:101C6000805F06D11946FEF7B7F90DF5805D01B02A
:101C7000F0BD4FF4805221466846FEF7C1FE314662
:101C80003A460DEB0500FEF7BBFE69462046EAE743
:101C9000F8B544680C44C4F30B0116461D46641A9B
:101CA0000DB90120F8BDC1F58057AF4228BF2F46BE
:101CB00033463A462046FFF7C9FF0028F2D0ED1B15
:101CC0003E4404F580540021EAE72DE9F04184B058
:101CD00002AF0C463A6A054619460CBB5300D81DA4
:101CE00020F007006E46ADEB000D02A84FF0800C0F
:101CF0000DF1090E94420BD10122A98B00920246EC
:101D00006868FDF79DFDB5460837BD46BDE8F08122
:101D100011F8048000F814C00EF814800134E9E7CB
:101D200002F1080020F007006C46ADEB000D4020EA
:101D3000531C8DF808000DF109007B60FEF760FE72
:101D40000122A98B009202AE7B6868683246FDF7DB
:101D500077FDA546D8E7F8B54589ADB204460E46ED
:101D600055B143899BB29A428ABF45891546ADB2A7
:101D70000027BBB29D4201D82846F8BDE389E2881E
:101D800021689BB202FB03113046FEF739FEE3895E
:101D9000A1889BB20133B3FBF1F201FB12339BB27A
:101DA000E3816389013B9BB26381E38801371E4471
:101DB000DFE700002DE9F047564C23780F469046A8
:101DC000002B40F0A08000252846BDE8F0871A09C6
:101DD000A2F10801032901D90E2A23D184F8242174
:101DE00084F829610135A84549D094F828017B5D24
:101DF00094F8241100286AD14FF0020C042984F8C9
:101E0000253184F828C1E2D1F72B06BF052384F8D9
:101E1000243184F8281194F8282194F829319A4221
:101E2000E0D123E0A2F10C01012905D884F8242196
:101E3000032384F82931D5E70F2A40D1F02B02D1B2
:101E400084F82461CCE703F0FD02F12A02D184F882
:101E500024C1EDE7F22B03D1032384F82431BFE73B
:101E6000052384F82431022384F829312A480422E6
:101E70005146FEF756FF032842D8002839D1627830
:101E8000264B02F07F0103EB410303EBD21393F8DF
:101E9000210010F0010697D121494022A1F5AC7034
:101EA000FFF759FF034600288ED01D4A617830465F
:101EB000FFF7D0F9002887D1F7F71CFB84E70F2341
:101EC00084F82431A4F8260184F829C1CEE7221829
:101ED000042982F8243100F10102D2B284F82821C9
:101EE00099D1F72B97D1043084F8240184F8292163
:101EF000BCE70C4B1B68DB077FF565AF00BE62E7F4
:101F000084F828916EE70025042604F5927AA94604
:101F100069E700BF50320120643201206C45012086
:101F2000BC330120F0ED00E008B510461AB10248BC
:101F300092B2FFF710FF08BD54320120814210B465
:101F400010D28B1898420DD2531E194403449A1A8A
:101F50009A4202D15DF8044B704711F8014903F829
:101F60000149F5E75DF8044BFEF74ABD38B5044674
:101F7000154662688A42084603D929448A4201D834
:101F8000606038BDA368521A18441944FFF7D6FFA1
:101F90006268521B6260F4E72DE9F04F2DED028B71
:101FA00083B00C460092F2B901F10C05D4F800A000
:101FB0000AF10203EB1808EE103A574606464FF0B6
:101FC00000094FF0610B33780BB1292B0DD1B9F11A
:101FD000000F58D0002D56D02368013BA3EB090316
:101FE00005F809304FE00025E0E73F2B00F029819C
:101FF00013D8243BDAB20A2A19D822680A2B16D839
:10200000DFE813F0AF01150015001500D900150029
:10201000420172011500150075005E2B00F09981D8
:1020200015D85B2B06F1010169D05C2B28D02768FD
:10203000002D59D07B1C23600123EB5523685A1CCB
:1020400022603278EA546368013363603BE07C2BA2
:10205000EDD1B9F1000F00F06181002D00F0618138
:102060002368013BA3EB090305F80930226818EE49
:10207000100AA2EB0A0205EB0A01FFF75FFF50E12D
:10208000737833B90026304603B0BDEC028BBDE84F
:10209000F08F276843F02000642807F1010205D083
:1020A00023F0040343F02003732B0ED1CDB105239D
:1020B0002260EB5523685A1C22607278EA546368E8
:1020C000013363600E4601367DE755B1012322607E
:1020D000EB5570782668F3182360F7F7E6F8A855F3
:1020E000EDE7BB1C2360EAE7BB1C2360ABE7531C96
:1020F00017462360002DA6D00223AB54A3E7276820
:1021000072787B1C5E2A236015D10DB10423EB5538
:10211000B11C2368013323606368013363600E469A
:102120004FF0000831785D290AD1002DCBD0EB1992
:1021300083F80180C7E7002DEBD00323EB55E8E7D8
:1021400000299FD023685C2903F1010225D1019366
:10215000711C05B370782260F7F7A7F8019BE8546B
:102160004B782D2B03D18B785D2B18BF02310E4697
:10217000236816F8010B5C2803F1010215D10193C5
:102180008DB148782260F7F790F8019BE85401364A
:1021900008F10108C6E72260E2E722600DB132785B
:1021A000EA543146DCE72260F1E722600DB10A789B
:1021B000EA540E46EBE773783F2B174627D1B378E6
:1021C0003A2B24D1002302369846701C009A0193C2
:1021D0002146FFF7E1FE064600283FF453AF0278A0
:1021E000292A7FF44FAF019B002B3FF46CAF23688B
:1021F0002DB35A1C22607E22EA5423684FEA480815
:102200005A1C08F10108226005F803801BE7A36847
:1022100003F10108C4F8088075B1531C23607E23C4
:10222000AB5423685A1C22604FEA4802EA546368A0
:10223000013363600123C8E702322260F7E702330B
:1022400053E72268BA423FF41DAF2DB1B81CD21B30
:10225000E9192844FFF772FE23680233236073787C
:102260003F2B07D10DB16223EB55013635B96368B9
:1022700001332CE0002DFAD005F807B02368EA19E5
:10228000023BDF1B5770F2E7BA423FF4FBAE2DB1C1
:10229000B81CD21BE9192844FFF750FE236802330B
:1022A00023603DB16022EA542368EA18C3F1FE03BB
:1022B0003B44537023680233236073783F2B09D16A
:1022C0000DB16223EB55013645B9636802332768C7
:1022D0006360F8E6002DF8D005F807B02368EA1926
:1022E000023BDF1B5770F0E7BA423FF4CBAE737886
:1022F0003F2B08D10DB105F802B001363DB9276872
:10230000023727609FE6002DF9D06223AB54236883
:10231000EA18C3F1FE031F445770F0E7002D7FF465
:10232000A5AE2368DA1C226015B12B4460229A7096
:10233000D4F8009009F101032360002DC5D005F801
:102340000AB0236805EB0A02023BA3EB0A035370B1
:10235000BBE72268531C2360002D88D05023AB5468
:1023600085E7531C2360002D81D05123F7E700003F
:102370002DE9F04F2DED028B0D4608EE103AD1B04D
:1023800016468346002802F012830968F9F7E8FE32
:10239000031E0293C2F20F832B6803442B60DBF809
:1023A0000080B8F1000F0BD1584618EE101AFAF75A
:1023B000B8FD6FF0060051B0BDEC028BBDE8F08FA8
:1023C000DBF80470002FEFD098F8004098F81C203C
:1023D000002C3CD1032A4FF009010CBF4FF011092A
:1023E0004FF0200939A8CDE93934CDE93B49F9F757
:1023F0005DFE386098F81C30032B0CBF05210321CB
:1024000039A8F9F753FE07F1180A7860DBF8BC37F2
:102410009C420CDB4FF0000ADBF8C4379A4580F28F
:10242000C780902303FB0A740023039391E0AAF171
:102430001003012139A80393F9F738FE039B43F8F1
:10244000040B5345F5D101340AF1100ADEE7032AE3
:102450004FF008010CBF4FF009094FF011093993F3
:1024600039A80023CDE93A33CDF8F090F9F71EFEF4
:10247000386098F81C30032B0CBF0121022139A8C9
:10248000F9F714FE7860C5E70C2139A8F9F70EFEBC
:102490000921A06239A8F9F709FE0821E06239A8EC
:1024A000F9F704FE206398F80030002B0CBF0421DC
:1024B000092139A8F9F7FAFD0121606339A8F9F774
:1024C000F5FDA063002855D0022139A8F9F7EEFDEB
:1024D0000121E06339A8F9F7E9FD0521206439A855
:1024E000F9F7E4FD0521606439A8F9F7DFFD002361
:1024F000E364A064032139A8F9F7D8FD032120651E
:1025000039A8F9F7D3FD0321606539A8F9F7CEFDA5
:10251000E36BA0652BBBC4E90A336363E36DC3F1CE
:102520001403236698F80030002B3FD1012139A80D
:10253000F9F7BCFD6066012139A8F9F7B7FD012163
:10254000A06639A8F9F7B2FD039BE0660133039357
:102550004834DBF8BC37039A9A4295DB0AF1010A4A
:102560005AE7022B04D1236C13B90823E365D5E79E
:102570000723FBE7C4E90F00052139A8F9F796FD09
:102580000521606439A8F9F791FD0521A06439A8F7
:10259000F9F78CFD0421E06439A8F9F787FD0321E0
:1025A000E06539A8F9F782FD2066BBE70020C1E7A6
:1025B0003B68CBF8D8372B684B442B60029B03EB6E
:1025C000090433681B1B3360DBF8B827DBF8B0372E
:1025D00072B1002B59D1DBF8CC2733689A4264DD05
:1025E000584618EE101AFAF79CFC4FF0FF30E2E65E
:1025F000002B4AD10123CBF8B037D5F80080D6F8AC
:1026000000A0A8EB0404474651463846FAF79DFC63
:10261000002807EB000324DB395C227891421BD1B0
:1026200059786278914217D1A1789A784A4012F08D
:10263000FC0F11D18F0748BF03F1FF33A3EB080351
:10264000002BCBF8B4370FDA584618EE101AFAF709
:1026500068FC6FF00200AEE60330DF1CAAEB000A54
:10266000D2E74FF0FF33EBE7029ADBF8C4171A44C6
:102670009144DBF8C027DBF8C83702FB09F2D2002F
:102680004B4392FBF3F2CBF8B827DBF80030DBF8D2
:10269000B4273BB15B69003B18BF01231344CBF85F
:1026A000CC3798E74FF0FF33F8E7DBF8DC07DBF8CF
:1026B000D8370BF11C01984208913EDBC11A1A462B
:1026C000089B19441846FFF739FC089BDBF8D8072C
:1026D000DBF8CC2729681844FEF792F9DBF8CC1711
:1026E000DBF8D8270A44CBF8DC272B680B442B6097
:1026F0003368DBF8CC279B1A3360DBF8DC37DB0070
:1027000011930BF5FC6319934FF0FF3310930023E3
:10271000CDE905330293DBF8C437029A9A4282F27C
:102720004E81902353431793059B0493199B149355
:10273000179B13934FF0000AE4E3089B29680344B6
:102740001846FEF75DF9DBF8CC17DBF8DC270A4406
:10275000CBF8DC272B680B442B603368DBF8CC27E5
:102760009B1A584618EE101A3360FAF7DAFB6FF02E
:10277000010020E6B8F1000F00F0A382DBF804307E
:102780000393002B00F09D82DBF80840002C00F042
:102790009882089B23930023CDE92433069A119B4A
:1027A0009A18D31D48BF02F10E03DB102693069B37
:1027B0001BB1194623A8F9F779FC029B98F8006031
:1027C00090225343482202FB0A32039B1A44536B64
:1027D000D16B002E40F03E819D4810F8135000EB65
:1027E000430302295F785CD1D2F84080B8F1000F32
:1027F0000DD0049B04EB0308294623A8F9F756FCE7
:102800000136082E08F8010BF6D14FF00308059B9E
:102810003E2606FB0A3608EB48031E4426440DF10B
:102820008C0929464846F9F741FC2946F075484687
:10283000F9F73CFC294630764846F9F737FC08F1B1
:102840000108B8F1060F707606F10306E9D1049B82
:10285000E61839464846F9F729FC394686F8290032
:102860004846F9F723FC394686F82A004846F9F726
:102870001DFC08F10108B8F10C0F86F82B0006F1D9
:102880000306E6D1029A7C235A433E2303FB0A2324
:102890001C44002384F83D3084F83C3084F83B30FD
:1028A0001AE0029B002B4BD13E2303FB0A44029EFD
:1028B000A1460DF18C0829464046F9F7F7FB013691
:1028C0000B2E09F8010BF6D139464046F9F7EEFB1D
:1028D000A0550136152EF7D1029A90235A4348236A
:1028E00003FB0A23039A1A44936A149A1360239AE7
:1028F000089BD31A259AC2EBC302D31002F0070239
:102900000A92069A14980A99C2EBC3020A4450F834
:10291000041B1490881A0390089818440E9011987C
:10292000002BA0EB02021A9202DB884280F2D081D7
:10293000584618EE101AFAF7F4FA6FF007003AE565
:102940004FEA0A13039A083302EB0308D658D6B1AC
:102950003E2303FB0A430622109813F8011B195467
:10296000013AF9D1D8F80430D3B9049B062604EB18
:102970000309294623A8F9F799FB09F8060001364F
:102980000B2EF6D11FE0049B04EB0309294623A874
:10299000F9F78CFB0136062E09F8010BF6D1E1E7B9
:1029A000029D3E2303FB0AF37C20E21800FB053363
:1029B000234491799971D179D971117A1972517A27
:1029C0005972927A9A72D8F808302BB33E2303FBDF
:1029D0000A430B330B22109813F8011B19540132D0
:1029E000102AF8D1D8F80C3023B33E2303FB0A4356
:1029F00010331022109813F8011B19540132152AB4
:102A0000F8D1029A7C235A433E2303FB0A231C4439
:102A100000236375A3755FE7049B0B2604EB030992
:102A2000394623A8F9F742FB09F806000136102EB3
:102A3000F6D1D7E7049B102604EB0308394623A8F8
:102A4000F9F734FB08F806000136152EF6D1D8E761
:102A500030000600D8F8206016F0010603D0BAF165
:102A6000010F00F0A580B3F5C87F6CDA18110522BC
:102A700090FBF2F2279202EB8202821A2892002047
:102A8000C3F3810203F0030329922A93024603460B
:102A9000022940F0C280029D4FF0900C0CFB05FC17
:102AA0004827039D07FB0AC72F443F6C002F08BF30
:102AB000012102EB4202854F114417F8212039927F
:102AC00007EB81014A783A928A783B92CA783C9225
:102AD000A6B1BAF1010F11D127AE04F1FC0239A958
:102AE00004F5867756F804CB42F804CB51F804CBB2
:102AF000C2F80CC0BA42F5D1C4F8F800029990228D
:102B00005143482202FB0A1203990A445366D36BCD
:102B1000022B40F0CC80176C002F00F0A980049BA2
:102B20000026E718279923A8F9F7C0FA0136062EE0
:102B300007F8010BF6D103230127059A4FF03E0950
:102B400009FB0A258CE0B3F5FA7F12DAA3F5C87306
:102B500098100522B0FBF2F2279202EB8202821A51
:102B600003F003030020289229932A9003460122B0
:102B70008EE7A3F5FA730322B3FBF2F202EB4200F5
:102B80001B1A0298039D27924FF0900C0CFB00FC3F
:102B900000274820CDE9297700FB0AC02844289364
:102BA000006C10B1CDE928233846012302226FE7DB
:102BB000B3F5B47F03F001004FEA630210DA242773
:102BC00092FBF7F307FB13220627279392FBF7F3F9
:102BD00007FB13222893002329922A93032257E705
:102BE000F32A0CDCB43A13112793C2F38103289320
:102BF00002F00302002329922A93042248E7F43AC0
:102C00000323B2FBF3F3279303EB4303D21A00230E
:102C10002892CDE9293305223AE7002149E727AB7D
:102C200023A853F827100791F9F740FA0799307550
:102C300023A8F9F73BFA0799707523A8F9F736FA34
:102C400008F10108B07539AA08EB090352F82710FA
:102C5000884506F10306E2DB0137042F3FF412AE8C
:102C600003EB43062E44994626444FF00008EAE75A
:102C70003B4662E727AB23A853F82610F9F716FA6C
:102C800008F8010B013755F826108F4207EB0903AE
:102C9000F0DB0136042E0DD1029A7C235A433E23E9
:102CA00003FB0A231C440023A375637514E6002369
:102CB0001E4639AD9946049B09EB0308A044002742
:102CC000E1E7069B0A934FF0FF331AE6B9FF0500D0
:102CD000DBF80040002C00F0B581DBF804300693EF
:102CE000002B00F0AF81DBF80830002B00F0AA8148
:102CF000DBF80C00002800F0A581039B002BC0F23C
:102D0000A181029B616B90255D434822069B02FBDB
:102D10000A551D44AB6B002B00F02081EB6B022B9E
:102D200040F01C812B6C002B40F00081EB6D0322E6
:102D3000013393FBF2F301EB4303B3F92E2002EBD3
:102D400042024FF41071029B90245C43482303FB22
:102D50000A43069C2344DC6A6300B3F5107FA8BFD6
:102D60004FF410739342D4BF3A933A9200EB8A0225
:102D70000793169202F590528B42D4BF3B933B913E
:102D80003C9307990023399311604FF4106202FBC2
:102D90000A020F9239AA0D920A9A0B920C930E9A7C
:102DA000139B0892069A4033D3181B930D9B1C6803
:102DB0000C9B01330C930D9B53F8045F0D932D1B5B
:102DC000002D40F36F82039B002BC0F23B810C9AD5
:102DD0001B9B089953F82260B44B03EBC6031B7985
:102DE00009930B9B09985B4213F007031EBF11F870
:102DF000017BC3F1200207FA02F20F9F08BF1A46B7
:102E000007EB8404002840F0BB80231D002244F817
:102E1000202043F8202002308542F7DC13460B9A2D
:102E200008991A4401EBE20102F007020B92039A9F
:102E30000891D31A03930C9B032BB7D1039B002B50
:102E400040F3B282029B079D90225A43482303FB22
:102E50000A23069A1A444FF00009D36E944A52F896
:102E60002300944A52F823600B9B5B4213F0070344
:102E700017BF11F8014B0899C3F1200204FA02F2BE
:102E80000F9C04EB85040694039CC6F12006A4EB7A
:102E90000305079C0796884EC4F50F74304408BF9D
:102EA0001A464F4601340990BC4200F30182169B3A
:102EB00003F5905213681F4417600023B7F5107F85
:102EC000C0F27482039A0B9B134403F0070206922C
:102ED000089A02EBE303139A48321392049A3E32A3
:102EE00004920E9A9B1A00F1AD800E9A1A44089231
:102EF0000A9AC2EBC303069A13441A9AD31A11937F
:102F00000AF1010ADBF8BC37DBF800809A45FFF6CE
:102F100031ACB8F1000F40F05182584618EE101A4B
:102F2000F9F7FFFF6FF00900FFF745BA23785BB9A7
:102F3000029C9023634302FB0A32069B1A44D36D22
:102F4000013331F91320FCE6B1F93630B1F9342000
:102F50009A1AB1F90C3003EB4202F2E6029A90237E
:102F60005343482404FB0A34069B1C44E36D246E3F
:102F7000013331F913202344013331F91310E2E610
:102F80004E4F57F826C04E4F07EB4C001190039858
:102F9000A0EB030E0998012840F0948037F81C60DC
:102FA00006F00F064FF00008C6F12006BEF10F0F25
:102FB00051DD0F46C3F1180017F802CB49780CFA1F
:102FC00000F0C3F1100C01FA0CF101430A43103375
:102FD000AEF1100E394604F1080722FA06F0119CF2
:102FE000013034F81000040B10F0F00F02FA04F274
:102FF000A3EB103318BF02F00044C0F3031C1EBF44
:10300000520003F1FF3344EA0C0C10F4706FC0F36C
:1030100003241FBF03F1FF3302F00040204352009E
:1030200008BF204643450DDB023D002D47E902C0A5
:103030003C4635DCA3EB0803039A7344D31A002BF8
:1030400080F23181584618EE101AF9F76AFF6FF0D6
:103050000800FFF7B0B90EEB03000028F2DDBEF167
:10306000000FC1BF11F8017BC3F1180C07FA0CF770
:103070003A43BEF1080FC1BF11F8017BC3F1100341
:1030800007FA03F31A434FF00047431E47FA03F3CE
:103090001A404FF00B0800F10B034FF0000E9AE7B7
:1030A0000A2B07F1080798DC80E700BFF8D006007C
:1030B00004FA0600FCF906000CFA0600F8D1060036
:1030C00078D206000998871E012FBBD8BA48119FF5
:1030D00050F836C0002012900CF101001590CCF190
:1030E00020001890BEF10F0F2ADD8846C3F11806A4
:1030F00018F8029B497809FA06F6C3F1100901FA9B
:1031000009F131430A431033AEF1100E41460A2B48
:10311000E8DDB7F8008008F00F08C8F1200622FAB1
:1031200006F6013637F816605FEA16392FD107EB3D
:103130004607A3EB080302FA08F226463446E6E700
:103140000EEB0306002E7FF77DAFBEF1000FC1BF6F
:1031500011F8018BC3F1180908FA09F842EA0802CC
:10316000BEF1080FC1BF11F8018BC3F1100308FABB
:1031700003F31A434FF00040731E40FA03F30B2091
:103180001A40129006F10B034FF0000EBFE7C6F392
:103190000318B8F10F0FC6F30326A3EB090302FAD5
:1031A00009F2374627D10998032827D1159803EB50
:1031B0000E09002E18BF0130484580463FF742AF48
:1031C0009845A9EB030E56DCBEF1000F0ADA7344F2
:1031D00003F1FF3E4FF0004040FA0EFE02EA0E02FD
:1031E0004FF0000E189822FA00F808F10F08A3EB30
:1031F0000C0302FA0CF2B8F1000F05D002F00049FE
:1032000049EA08085200013B0F2E21D109980328F2
:1032100043D1159803EB0E0948453FF713AF1598B6
:103220009842A9EB030E30DCBEF1000F08DA7344BC
:103230005E1E4FF0004040FA06F632404FF0000E9E
:10324000189822FA00F70F37A3EB0C0302FA0CF2DE
:1032500027B102F0004637435200013B12988342E7
:10326000FFF6F0AE2646023D002D46F8088B67605B
:1032700015DD119F62E711F801EBC3F118000EFA9A
:1032800000FE42EA0E0208339AE711F8016BC3F11F
:103290001807BE4032430833C1E73746D9E7129AD0
:1032A0009B1AC9E60023039A93427FF7B8ADC9E69B
:1032B0000F2D57DD0E46C3F1180016F802CB4978E2
:1032C0000CFA00F0C3F1100C01FA0CF101430A43AF
:1032D0001033103D3146069E1036079822FA00FC46
:1032E000099810F80C004FEA101C02FA0CF210F0CA
:1032F0000808A3EB10131FBF02F0004803F1FF33CF
:10330000520048F0010810F0040E1FBF02F0004EFA
:1033100003F1FF3352004EF0010E10F0020C1FBFFC
:1033200002F0004C03F1FF3352004CF0010C10F09E
:1033300001001FBF02F0004003F1FF3340F0010025
:1033400052004B45FFF6B3AD0437A74246E9048E61
:1033500046E902C00696BFF6A7AD092B06F1100696
:10336000BBDCA1E5E81800287FF7A1AD002DC1BFA7
:1033700011F8016BC3F1180C06FA0CF63243082D54
:10338000C1BF11F8015BC3F1100305FA03F31A433F
:103390004FF00045431E45FA03F31A404FF00A0967
:1033A00000F10A03002596E7002780E50F9A42F80E
:1033B0002730013782E500BFF8D00600DBF8047043
:1033C000002F3FF4AAADDBF808300793002B3FF441
:1033D000A4ADDBF80C90B9F1000F3FF49EADDBF823
:1033E00010A0BAF1000F3FF498AD09F590530A937D
:1033F000029B179A7C246343503216931744079B11
:10340000169A13440C93002354460B93DBF8BC37F5
:103410000B9A9A424EDBD8F82030002B40F068819E
:10342000D8F820305A10039240F0AA81D8F8203002
:10343000D90740F1A68209F5905298F8005010681B
:103440005B100493DAF83033002D40F09783002BA3
:1034500040F0DB81DAF84443D8F83420DAF82C5312
:1034600009930134013532F91410049EAB4A079FC9
:10347000A0EB010A1C2000FB0622059E0A923E36A4
:10348000BE190E96049FA64E002206EBC7060392B5
:103490000F96AC4203DABAF1000F00F3CF81079C1C
:1034A00005985534201814909D4C049804EBC000E6
:1034B00015905FE20B9B4FF4106202FB0393139392
:1034C00057F8143C022B46D157F8106C002E46D00A
:1034D00098F800300322002B03920CBF0826062622
:1034E00000233993BB69D8F8202001335B00129385
:1034F00057F8203C520818BF023B9A1C17920C9AAE
:103500000E92C3F1D003002209921546049214933F
:10351000B54226D10023C4F81833399AC4F81C33B5
:10352000C4E9C833C4F82833039BC4F82C230B2BFD
:103530004BDD0998F9F7FEF90A9B013898600B9B5F
:1035400001330B930A9B04330A930C9B3E331834CC
:1035500048370C935AE70D2303931626C0E70396CA
:10356000BEE76B1C0F93D8F8343003EB4502B2F979
:10357000021033F915208B1A0E9A0D9312F8013BA5
:103580000E927A6922B1674A691C0A4412F8012C2A
:1035900004981399134401EB8001129A149802FBCA
:1035A00003030D9A0846F9F7D1F9049A0D9B1344C9
:1035B000049300B13995099B049A034309930A9B2C
:1035C0001B689A42A6DA0F9DA2E7039B3B93CDE9C5
:1035D00039330C9B14331893039B0F9301330F9AC9
:1035E0000393D8F83430159703EB42030026B3F960
:1035F0003010B3F92E20039B8A1A189903EB43036A
:10360000CB181493930004990E93139B03EB81053D
:10361000179B0D95C3F1D20351461A93159850F894
:10362000043B1590149810F801CB14901A9800EBF5
:10363000C303129800FB0C330D98CDE91B12F9F768
:1036400085F9DDE91B1220B10DF1E40C0F9B4CF85C
:103650002630099B03430993DDE90D30013603440D
:10366000032E0D930144D9D1049902EB420319446E
:103670000346534404911E460AEBC20100239A42BA
:1036800005F10C0526DC0A9B049A1B689A4202DAB3
:10369000039B0D2BA0D10A9B1A46049B136057F87D
:1036A000103C002B14BF02230123C4F81833399BAC
:1036B000C4F81C333A99C4F820138B423B9AC4F8DF
:1036C0002423B8BF0B469342ACBFC4F82833C4F8D8
:1036D00028232EE75AF8230045F80C0C56F8040B63
:1036E00045F8080C51F8040B45F8040C0133C6E703
:1036F00041F2082359F80330002B06DD41F20C2378
:1037000059F80330002B3FF78BAE09F59053064C68
:1037100019686FF04040002310E000BFB0CE0600F3
:10372000A0CE060080890600010000C059F82320C1
:10373000B2F1404F19DC49F8234001338B42F5DBED
:1037400041F20423674D59F80300002209F5106384
:103750006FF040448242BFF663AE1968B1F1404F4A
:1037600009DC1D6001320433F4E7B2F1804FA8BFD9
:1037700049F82300E1E7B1F1804FA8BF1C60F1E7F1
:10378000D80737D5DAF83023D8F834304ABBDAF81E
:103790004423013233F912300022A9F104010392CB
:1037A00015461646AB427FF741AE51F804CFD1F82B
:1037B00000490CEB0407ACEB04040F60C1F80049AE
:1037C000B44687EAE77CACEBE77C039840EA0C0060
:1037D0000390374684EAE477A7EBE4773A43013570
:1037E000E0E7DAF8402303EB4203B3F9303003EBB0
:1037F0004303D1E741F2042309F5905259F803102D
:1038000013688B42B8BF0B46C6E7013B012B10D8AB
:10381000DAF82823DAF8401301320992D8F8342074
:1038200002EB41024B1CB2F930102C4601EB410176
:103830001BE609952B462C46294616E60E9E365D5C
:10384000072E274623D10498274E56F830C00F98EC
:103850004068D8F834600C9006EB470E36F91760D4
:10386000BEF902E00B91AEEB060001340D9009EBBE
:10387000810700260D980B99B0423144AAEB060E41
:1038800003DD56450AD14FF0000EF24601E60A98D4
:1038900050F826C08669A6EB0C00DAE757F8041B3F
:1038A0000C9880FB01E18900C7F8FC184FF0000E6E
:1038B00081EAE17EAEEBE17E57F8041C42EA0E029B
:1038C0008CFB01E1890047F8041C4FF0000E81EAEF
:1038D000E17EAEEBE17E039941EA0E0103910136F0
:1038E000C8E700BF010000C0A0CE0600149803EB9B
:1038F00043060644002516F8014B072C40F0D580FE
:1039000004989D4C54F8304027A840F8254015985D
:10391000446839A840F825400135032DEBD1D8F88B
:1039200034400791013304EB430504EB4C0CB5F92B
:103930002E50BCF92E40281B0B9039980C902798DC
:103940000D903A980E9028980F903B98129000276F
:103950002998139009EB8104BC46079807EB4701AF
:1039600001440B98B84205DDBAF1020F04F10C04D2
:1039700000F3A580099883429C4602DABAF1020F4F
:10398000B4DCD8F82030E3B10398F8F7D3FF41F264
:103990000823013849F803001046F8F7CBFF41F23D
:1039A0000C23013849F8030041F2042209F5905133
:1039B00059F8023008688342B8BF03460B6049F8E3
:1039C000023000230393039ADBF8BC379A42C0F21B
:1039D0001182029ADBF8C847544318EE102A5C4360
:1039E00002EB4404DBF80C20002A00F0D787DBF858
:1039F00014200392002A00F0D187DBF81850002D24
:103A000000F0CC87022B02F5D85303F1180307937B
:103A100040F03A8605F1800302F5D85907EE903A56
:103A20001746002605F5085809F11C09079B1B6875
:103A3000009306F0010A3846D8F80020534629467C
:103A4000F8F764FCD9F80030009317EE901A07F5E8
:103A50001060D8F800205346F8F758FCD8F800302A
:103A60004FF4886101FB0A3104EBC61005EB8101BC
:103A7000F9F77EFAD8F800300136A3EB0A0303F019
:103A80000703122EC8F8003007F18007CED1029B41
:103A900001330293059B7C330593199B08331993DB
:103AA000109B7C331093FEF736BE0A9850F82470B2
:103AB00027A840F825700A988469E41B29E754F880
:103AC0000C1C0C9880FB01518900C4F8F418654661
:103AD00081EAE175A5EBE17554F80C1C0D9880FBAB
:103AE00001618E0044F80C6C614686EAE671A1EB38
:103AF000E67154F8086C0E9880FB06E6B000C4F836
:103B0000F808664680EAE076A6EBE07635430F9843
:103B100054F8086C2A4380FB0656B60044F8086C3B
:103B2000654686EAE675A5EBE67529430398129D7E
:103B300008432E4654F8041C86FB01518900C4F842
:103B4000FC18654681EAE175A5EBE175139954F817
:103B5000046C2A430D4685FB0616B60044F8046C37
:103B6000614686EAE671A1EBE67101430391AAF191
:103B7000030A0137F1E600BFA0CE0600079A0499B8
:103B8000D2F8F82001EB4202A04901EB821209921F
:103B9000079A002402F1FC0102F5867C4FF0010E29
:103BA00051F8042B39AD0EFA02F2CE6805EB84070A
:103BB000013A0025B54251DB002EA8BFA4198C455F
:103BC000EED10121002B40F08580D8F834200393FA
:103BD000CDE94E11DAF84413DAF82C430B94013195
:103BE0000DF1E40E32F911701A46059B03F13E0403
:103BF000079B2344C51B0C930498854B03EBC00320
:103C00000D930B9B8B42FFF6BCAE0C9B5C5C5EF88D
:103C100021309C420E4625D17D4B049853F830301C
:103C20000A930D9B5B680793D8F8343003EB460486
:103C300033F91630B4F90240E41AAC4201F1010143
:103C4000A8BF2C4609EB87064FF0000C64451CDC2E
:103C5000002CA8BF3F192D1BD3D192E647F8042BA7
:103C60000135A7E7631C5B1014F00104099814BF29
:103C70004FEA830CA44650F80C000A901CB99B0034
:103C80000998C358CFE70023FAE756F8043B079892
:103C900080FB03A39B00C6F8FC384FF0000A83EAC0
:103CA000E37AAAEBE37A56F8043C0A9842EA0A025D
:103CB00080FB03A39B0046F8043C4FF0000A83EA14
:103CC000E37AAAEBE37A039B43EA0A0303930CF13A
:103CD000010CBBE70AF54773169C0A93079B4591B5
:103CE0005534234404991C46494B002203EBC1037D
:103CF000039294460D930A9B1846996950F8043B29
:103D00000C93D8F834300A9003EB41034D1C1E8EFF
:103D1000032316FB03C60C9BAB4207DA0CF1010C24
:103D2000BCF1030F04F10104E5D12AE605EB4503DC
:103D30002F4614F803E039AB53F825108E451FD1F8
:103D4000334B049953F831300B930D9B5B68079309
:103D5000D8F8343003EB47030135B3F93010B3F929
:103D60002E3009EB8607C91A4FF0000E714507F196
:103D70000C071ADC21EAE17101EB41010E44CAE7AC
:103D80000EF101031EF001014FEA6303099814BF0D
:103D90004FEA830E8E4650F80E000B9019B99B0027
:103DA0000999CB58D3E70023FAE757F80C3C07985A
:103DB00080FB03A39B00C7F8F4384FF0000A83EAA6
:103DC000E37AAAEBE37A57F80C3C0B9842EA0A0232
:103DD00080FB03A39B0047F80C3C4FF0000A83EAEA
:103DE000E37AAAEBE37A039B43EA0A0303930EF117
:103DF000010EBBE7DBF8003063B9584618EE101A25
:103E0000F9F78FF86FF00A00FEF7D5BAE8CE060092
:103E1000A0CE0600DBF804200D92002AEDD0DBF8DE
:103E20000C200492002AE8D0DBF81450002DE4D0D6
:103E30005A6B1B780398002B0CBF08230623122112
:103E400032F91330029A93FBF1F30C9390235A4307
:103E5000482303FB00230D9A1344DA6B022A00F077
:103E6000E380049A00F5906352F8236040F2262321
:103E70009E42CFBF2023073696FBF1F14B1C0B93DC
:103E80000B9B5A1E039BDFF8A49407924FF4106A11
:103E90000AFB03FA049B534414930799002900F387
:103EA000CB80DDE9033101EB830000F59054122152
:103EB00023680D9E4A4308329A42B8BF1A462260D0
:103EC000113292FBF1F31593039B05EB83030A93E5
:103ED00003F5D85341F608321B681A930A9B9B5886
:103EE000169341F610320A9B9B581793039B4FF091
:103EF000480909FB03F1029B90225343CC18344438
:103F0000246C002C0C9C08BF00240C9441F2082463
:103F10000059129003984FF4906404FB005404F588
:103F200090501B9005EB0A0013901298C0F1070007
:103F30000990129806280998C8BF002007EE100AB9
:103F4000139800F508600F9014983C300E90CDE95E
:103F50001E911B980790CDE92023002004908246F3
:103F60000B9B534500F3228123EAE377149A1E9BAF
:103F7000079703FB07291B9B242404FB0733149397
:103F800003EB0408139B03EB87030B93A8F12403B3
:103F900007EE903A079A159B934200F32382BB42A7
:103FA000A3EB07004FF02404149B04FB00F4AEBF06
:103FB0000646002400263E4423441C46B0463546AF
:103FC00000271A9BAB4200F30183B342B8BF3346CC
:103FD0001E4600221F2E40F34583049B002B00F059
:103FE00051830022049B002B80F247830A9B029995
:103FF000039803F5D853C3F800809023594348230E
:1040000003FB00130D99194441F60830CB6B0A9954
:104010000B5041F610300C9B0B50531E41F61832DA
:104020008B50039B0133CDE41A6C1AB10C9B0B939C
:104030005A1E27E70B9225E75C6CB04E214686FBA3
:104040000171AF4E9F6C304686FB07C7C91B490004
:104050005964AA4E996C86FB017180FB04740C4470
:1040600064009C641C6CA74E214686FB017100F124
:10407000AF6000F5A430DF6C9F3080FB07C7C91B21
:1040800049001964D96C86FB017180FB04740C44EF
:104090006400DC64DC6B9C48214680FB01719B4E14
:1040A0001F6D86FB07C7C91B4900D963196D80FBCB
:1040B000017186FB04740C4464001C6500F1896086
:1040C0009C6B00F5FA20214600F50D7080FB017114
:1040D0008F4E5F6D86FB07C7C91B49009963596DF9
:1040E00080FB017186FB04740C4464005C655C6BAE
:1040F000214689FB0171874FD3F858C087FB0CEC30
:10410000A1EB0C0149005963996D89FB01C187FB43
:1041100004C40C4464009C651C6BDFF814C2214687
:104120008CFB01717C4FD3F85CE087FB0E8EA1EB1A
:104130000E0149001963D96D8CFB01E187FB04C4B2
:104140000C446400DC65DC6ADFF8E8C121468CFBC6
:104150000171724FD3F860E087FB0E8EA1EB0E0168
:104160004900D962196E8CFB01E187FB04C40C4441
:1041700064001C669C6ADFF8C0C121468CFB01719B
:10418000674FD3F864E087FB0E8EA1EB0E01490068
:104190009962596E8CFB01E187FB04C40C440799BA
:1041A000640001395C660791483376E6219A1F9BCB
:1041B00013440D9A1344D3E90F731BB10C9B534561
:1041C000C8BF0027DDE916325245C8BF0023984614
:1041D0000F9BA3F508631893129B062B2FAB7CDC77
:1041E000079A0E9C002602F124003246A168099D20
:1041F0002941891A62682A418E1B521A5E6243F86D
:10420000042950F8041D2941016007998142A4F155
:104210000804EBD1309B5B103093279B27A85B10E1
:104220002793F8F763FC30A8F8F760FC57EA080416
:1042300000F0848039AE424607983146F8F72CFDED
:10424000209B384803FB07004AAB00241D93364BE4
:104250001C9300F1480922460DF1BC0E3146A046E0
:104260001C9DDEF8243055F804795EF804691C952D
:1042700087FB03C3079DC3EBA60C03EBA60345F81E
:10428000223050F822608CFB06361D9D51F82230FA
:1042900059F8047D334455F804691D959B008CFB47
:1042A0000757189D3E44D701B600EB516FF07F05CC
:1042B00005FB02F70F9DEE51474683EAE377A7EB34
:1042C000E377434686EAE673A3EBE67301321F43C6
:1042D000092A44EA0704C3D16DE00E98002422465F
:1042E000A0F148068168891A426808380C1B521AE6
:1042F00086425C6243F80429F4D18BE7F053C26D27
:10430000AA0025BEE4EBDC70736E8D794A3FE3D7DB
:104310007611B7E82FFEE4F3C7A3C1FAC6BD2EFE9F
:104320005DC286FF9CF30600302A0600B7206D7F31
:10433000407EE47F63B2FC7F94C6FF7F079FA04E60
:10434000DFF8849220460DF1BC0CA646DCF8242050
:1043500059F804395CF8041983FB0282A2EBA1032B
:10436000D7F8008002EBA10247F8042BC8F1000146
:1043700056F8082BC91A81FB025203EB820256F849
:10438000043C81FB03534142189D6A500F99C8EBCE
:1043900083030B50714682EAE271A1EBE27172462F
:1043A00083EAE372A2EBE3728038114310F5906F59
:1043B00044EA0104CAD117EE103A524607991898F8
:1043C000F8F7F4FC049B204303430493079B243336
:1043D00007930F9B04330F930E9B48330AF1010A96
:1043E0000E93BDE5DDE9163107988142C8BF002371
:1043F0001A46129B062B13DC17EE901A4B4609F156
:1044000048041868099D2841186058682841586078
:1044100051F8040B083328419C4241F8040CF0D1B8
:1044200027A948460E92F8F7EBFB2DA909F10400E5
:10443000F8F7E6FB33A909F10800F8F7E1FB0E9A5B
:1044400017EE900A39A9F8F727FC29AA0E920B9AC1
:104450005C49002002F5C07639AB27AD0F901F965E
:1044600053F8046B0446B60086EAE674A4EBE674DF
:1044700016609E681894B600044686EAE674A4EBBB
:10448000E674C2F8806151F8046BD5F80CE01B9417
:1044900086FB0EAE5E6904460EEB860686EAE6747F
:1044A000A4EBE674DDF838E0C2F800631C94DEF893
:1044B0000CA08C6884FB0A6A1E6A04460AEB860616
:1044C00086EAE674A4EBE674C2F880641D94AEF14B
:1044D00004044E69DEF800E00E9486FB0EAED5F8BB
:1044E00024A051F8044C84FB0A6ADE6AD6440EEB21
:1044F0008606044686EAE674A4EBE674C2F8006613
:10450000D5F800C00E6A1E94043586FB0CEC0E9C98
:104510008E68D4F828E086FB0EAE9E6BF4440CEB5C
:104520008606844686EAE67CACEBE67C189CC2F8FC
:104530008067A6461B9C4EEA040A1C9C4AEA040AB1
:104540001D9C4AEA040A1E9C4AEA040A0F9C4AEA95
:104550000C0A44EA0A040F941F9C803294427FF4B0
:104560007FAF2D9B9B1048F8243C2E9B9B1048F856
:10457000203C2F9B9B1048F81C3C33A9A8F1180342
:1045800051F8042B921043F8042B4345F8D117EE51
:10459000103A079A0B9817EE901AF8F707FC0F9B42
:1045A00003431846049B03430493079B013307937B
:1045B0000B9B043309F1480908F124080B93E5E447
:1045C000F4400600BCF40600302A0600DDE916318E
:1045D000A942C8BF00231A4639A92046F8F75CFB58
:1045E000139B03EB850105F00103099304F12003FC
:1045F00045F3000A39A8A4F1040E4FF0000C0B9308
:1046000003684FEA8309C1F800903B4689EAE973E1
:10461000A3EBE973079343688AEA83031A46099B6D
:104620001A4449EA02094CEA090CC1F88020B9464B
:1046300082EAE279A9EBE279079B4EF8047F43EA2C
:104640000902049B134304930B9B734500F108007C
:1046500001F58071D4D1BCF1000F18BFA8462434F5
:104660000135AEE4139B03EB86000023D90101332F
:10467000122B4250FAD10136ACE4049B5B000132AC
:104680000493AFE42022B1E405F508531E344FF043
:10469000000A04930AF001030993079B049A1B681C
:1046A000039800932946099B126800EBCA10F7F79C
:1046B0002DFE049B09991A684FF4886303FB0123BC
:1046C00005EB83074FF0000C55F82310FA6D4FF0FF
:1046D00000736046C1FB003C6FF07301C2FB013CFC
:1046E0004FF455797968BA6DC1FB093CB549C2FBF5
:1046F000013C41F6D478B9687A6DC1FB083CB249F7
:10470000C2FB013C46F2B860F9683A6DC1FB003C5F
:10471000AE49C2FB013CAE4A3969C1FB023CAD491E
:10472000FA6CC2FB013C7969BA6CC1FB003C45F2F2
:104730008401C2FB013CB9697A6CC1FB083C40F2C0
:104740002C71C2FB013CF9693A6CC1FB093C742134
:10475000C2FB013C4FEA936343EA8C1324F81E3CEE
:1047600007F580534FF0007219684FF4D0700023A2
:10477000C1FB002341F2040141F67C007958C1FBE2
:10478000002341F2080149F2FC707958C1FB002373
:1047900041F20C0190487958C1FB002341F210010D
:1047A0008E487958C1FB002341F214016FF0B30029
:1047B0007958C1FB002341F218014FF41270795867
:1047C000C1FB002341F21C016FF013007958C1FBBB
:1047D00000234FEA926242EA8312A4F11E030A9375
:1047E000DFF8FCC1628004F122030B93DCF844E0A3
:1047F000D7F85C91D7F80031DCF840104FF0007228
:104800000020C3FB01204FF00073D7F800610021A6
:10481000C6FB0E31CEF1000EC9FB0E20DCF8406065
:10482000C9FB0631D7F80461DCF84C90D7F858E1A1
:10483000B046DCF84860C8FB0620C8FB0931C9F166
:104840000009CEFB0920DCF84860CEFB0631D7F822
:104850000861DCF85490D7F854E1B046DCF85060B9
:10486000C8FB0620C8FB0931C9F10009CEFB0920AD
:10487000DCF85060CEFB0631D7F80C61DCF85C90B8
:10488000D7F850E1B046DCF85860C8FB0620C8FBFA
:104890000931C9F10009CEFB0920DCF85860CEFBD4
:1048A0000631D7F81061DCF86490D7F84CE1B046D7
:1048B000DCF86060C8FB0620C8FB0931C9F10009BB
:1048C000CEFB0920DCF86060CEFB0631D7F814611E
:1048D000DCF86CE0D7F84891B046DCF86860C8FBBB
:1048E0000620C8FB0E31CEF1000EC9FB0E20DCF80D
:1048F0006860C9FB0631D7F81861DCF874E0D7F8B6
:104900004491B046DCF87060C8FB0620C8FB0E314D
:10491000CEF1000EC9FB0E20DCF87060C9FB063139
:10492000D7F81C61DCF87CE0D7F84091B046DCF8A1
:104930007860C8FB0620C8FB0E31CEF1000EC9FB23
:104940000E20DCF87860C9FB06314FEA926242EA39
:1049500080120A9820F8022F0A904FEA936343EAE4
:1049600081130B9A22F8023D84420B920CF1400C09
:1049700007F580777FF43AAF049B099A1B680AF128
:10498000010A9B1A049A03F00703BAF1120F13608D
:1049900004F140047FF47EAEFFF779B8584618EE74
:1049A000101AF8F7BEFA6FF00B00FDF704BD6FF0B8
:1049B0000400FDF700BD6FF00500FDF7FCBC002012
:1049C000FDF7F9BCD4F8FFFF7CAFFFFF3CB6FDFF5D
:1049D00078940400C44902004CE803002464FFFFFB
:1049E000DCF5060000F0030370B553EA010406D0BD
:1049F00002440346934213D003F8011BFAE722F066
:104A000003039608034405469D420AD1910742BF1D
:104A1000002120F826100233D20701D500221A7097
:104A200070BD45F8044BEFE770B531220021064612
:104A30000E480F4DFFF7D6FF1022FF210D48FFF75C
:104A4000D1FF1022FF210C48FFF7CCFF0B481422A6
:104A50000021FFF7C7FF0024AB680BB13046984731
:104A60000134042C05F12005F6D170BD6C45012000
:104A7000500106006D4501207D450120D42E012006
:104A80002DE9F04FBA4B87B01B780093002B00F054
:104A9000CC82B84EB84FB94B1C682378012B02BFAB
:104AA000B74B8022C3F88420B4F80E801FFA88F830
:104AB000B8F1000F18D0638A628961689BB202FB6B
:104AC000031103A8FBF79CFF638A2189DDF80080AE
:104AD0009BB20133B3FBF1F201FB12339BB2638251
:104AE000E389013B9BB2E3812378012B02BFA44BF6
:104AF00080225A60B8F1000F00F073829DF80D30EB
:104B0000013B072B00F2248201A252F823F000BFE0
:104B1000314B0300314B030047500300974A030019
:104B2000974A03003B4B0300174F030061500300FB
:104B30009DF80C00FFF778FFADE7924C9DF80C5004
:104B4000237843F00103237000233B619DF810306C
:104B500003F06002602AA14605D13368D90740F10D
:104B6000E58000BEE2E0402A0FD1874B002B00F029
:104B7000DD80864B03B13B6104A92846AFF300807A
:104B80008046B8F1000F86D1D0E003F01F03012B5F
:104B900000F03881022B00F05281002BDDD1002A79
:104BA000DBD19DF81130092BD7D801A252F823F0A0
:104BB000EF4D0300DF4D03005B4B0300CF4D0300BF
:104BC0005B4B0300D94B0300194D03005B4B030003
:104BD000074C0300214C030006AB13E9030000223D
:104BE000C7E9022287E80300694BD3F80014D3F821
:104BF00000040143C3F80014C3F858214FF48002A5
:104C0000C3F8042347E72378C3F340038DF80A3041
:104C100001230DF10A0204A92846FCF7B1FD3AE789
:104C200023789DF812A0C3F340029B0718D4BAF171
:104C3000000F15D02378DFF870B1019223F0300314
:104C400043F0100323709BF801300B2B16D19BF817
:104C500000309B444F4B9B45F5D34F4B00221A70BD
:104C6000BAF1000A237818BF4FF0010A6AF3410332
:104C7000237004A92846FCF741FD0CE7042B14D14E
:104C80009BF80530022B08D0082B14D0032B15D02D
:104C9000012B0AD14FF0030801E04FF000089BF808
:104CA00002304B445A78FF2A0BD03368D8077FF57F
:104CB00054AF00BE51E74FF00108F0E74FF0020893
:104CC000EDE783F80180019BADF80A30334B03EB2D
:104CD00048130DF10A02DB68594628469847002818
:104CE000E3D0BDF80A000828DFD95A4600235178DE
:104CF000052909D192F802C00CF07F0109EB4101AE
:104D000001EBDC1181F8118011780B449BB29842C1
:104D10000A44ECD883449DE7BDF81230190A0329F0
:104D200047D010D8012918D002293FD0184B0122B2
:104D30005A65BFF36F8FBFF34F8F5A65BFF36F8F05
:104D4000BFF34F8FA7E60F29F0D1154B002BEDD005
:104D5000AFF300804388024601E0124A122304A9FF
:104D60002846FCF70DFD00287FF495AEDEE700BF76
:104D7000D82F0120F0ED00E0D42E0120A045012025
:104D800000E100E06C450120000000000000000090
:104D90000070024046A606003022012050010600A5
:104DA0000000000046A6060075A50600B04ADA23FA
:104DB000D5E7DBB2EE2BB9D00B2B3FF6CEAEAD4A2A
:104DC00052F82320002A3FF4C8AE1378C7E7BDF895
:104DD0001230012BAAD1237843F0080348E7BDF82D
:104DE0001230012BA2D123786FF3C30340E723785D
:104DF000C3F340129B0803F002031343ADF80A30DB
:104E0000022306E79DF814100F298FD80C4461780F
:104E100003298BD82AB99DF811000A2806D00B283F
:104E200007D004AA2846F4F76FFB9CE78DF80A2008
:104E3000EFE69DF81230002B7FF48FAE19E79DF856
:104E4000141011F0780C7FF488AE01F07F0004EBB1
:104E5000400404EBD1144FEAD11E94F811A04FEA9C
:104E6000400B002A55D19DF81120012A27D0032A92
:104E700047D0002A7FF471AE94F82120C2F340029B
:104E8000ADF80A2004A90DF10A022846FCF778FCC7
:104E9000BAF1FF0F0BD0BAF1030F3FF65EAE04AAD2
:104EA00051462846F4F730FB002818BF80469DF88D
:104EB000103013F060037FF464AE3B6161E6BDF82F
:104EC0001230CBB950B16C4BC3F8181541F4807156
:104ED000C3F80C15BFF36F8FBFF34F8FD944CE4487
:104EE0009EF821306FF341038EF821309EF8213077
:104EF0006FF300038EF8213004A92846FCF7FEFB6F
:104F0000C6E7BDF81230002BF6D12846FAF772FF3B
:104F1000F2E7E046BCE79DF81010584B01F07F0423
:104F200003EB440303EBD1134FEAD11C93F8212088
:104F30006FF3000203F1200083F82120002C48D1F8
:104F40003B789DF80C80059DBCEBD31F0FD02DB195
:104F50003368DB077FF59FAD00BE9CE5484B002B17
:104F60003FF499AD39464046AFF3008093E597F999
:104F70000030002B07DBB86800283FF48CAD4149B6
:104F80002A46FBF73DFDBA68FB892A442B44BA60E8
:104F9000FA889BB29A42FB8101D03F2D15D83B691C
:104FA0006BB997F900300022002B1146B4BF2046A0
:104FB0008020FCF707F900287FF46DADC8E739467B
:104FC000404698470028ECD1B0E64046FCF7AEFBDF
:104FD000F1E75A7C032A2BD92B4B1B68DA0700D543
:104FE00000BE2A4C254BA27802F07F0103EB41035F
:104FF00003EBD21393F8210010F0010515D104F54D
:105000000761402204F12000FCF7A5FE014660B1D3
:10501000FAF7F6F948B10B4604F50762A17828467D
:10502000FCF718F908B9F4F765FA07B0BDE8F08F96
:10503000174B9DF80C0003EB42139DF811209C695F
:10504000059BA04727E5124D0024EB6913B19DF89D
:105050000C0098470134042C05F12005F5D11AE520
:10506000049B002B3FF417AD0598984713E500BF4C
:105070006CA5060070990600007002406C45012086
:10508000000000002C450120F0ED00E02426012066
:1050900050010600024840220021FFF7A3BC00BFD8
:1050A0000C440120024840220021FFF79BBC00BFB6
:1050B0000C440120054B00225A831A609A831A710E
:1050C000DA835A859A85DA85704700BF2426012045
:1050D00008B5134B4FF40B6200211846FFF782FC12
:1050E0004FF44241C180012101810821FF22017357
:1050F00000F130014271016100224FF48231034618
:105100004283428182834161C283027600F58660D8
:10511000C3E908015A8583F828209A85DA8508BDF5
:105120002426012002482C220021FFF75BBC00BF8F
:10513000AC2F01200020FFF7F5BF0000044B002238
:10514000DA811A601A825A82DA831A845A84704782
:10515000503201200E4B10B54FF4D6720021184684
:10516000FFF740FC00F124020346426009489860C2
:1051700003F1A404C3E9054000220121DA81197377
:105180001A8219775A82DA831A845A8410BD00BFB2
:10519000503201208000010030B50388A3F11002D5
:1051A0001F2A89B00C4606D88188228891421AD1DC
:1051B000242B16D907E0A3F150021F2A0FD88188AB
:1051C000228891420FD1503B9AB2072A0BD8072B65
:1051D00009D8DFE803F061087908084E0846242B57
:1051E00032D8102B01D80020B6E0113B132BFAD88F
:1051F00001A252F823F000BF63520300E9520300FA
:10520000FB5203005D530300E7510300E751030025
:10521000E7510300635203003F530300A15303000F
:10522000E7510300E7510300E7510300E751030092
:10523000D7520300E75103005552030063520300A5
:1052400067520300635203003A2BBCD14389A1F893
:10525000763006E000238088ADF800306946F5F727
:1052600001F9012078E0002220881146F5F7FCF8CA
:10527000F7E7B4F87610C38841B9172B38BF172366
:10528000B3F5007F194628BF4FF400712088A4F8B9
:105290007610F5F7E9F9E4E722884FF6FF739A42B2
:1052A000DFD094F85A30022BDBD183684E4A23F0CA
:1052B0007F4393424FF00105D3D184F87850F5F73E
:1052C00025FCC4E92001CCE7002320881A461946B2
:1052D000F4F7A8F9C5E7012500F1080184F8745036
:1052E0002088F5F7ADF8BCE750F8083FE36643685F
:1052F0002367002384F87430B3E704F108035022D5
:1053000000211846FFF76EFB04F1240300210493EB
:1053100004F14003CDE90531A37800908B424FF6AC
:10532000FF72A4F858202088304A03916B4618BFBA
:105330000A46CDE901110791F5F78CF991E7037A57
:1053400084F85B309BBB638BA4F8583001200223A8
:1053500084F85A3084F8790009B030BD028AA07808
:105360000121F4F763F9A0B1C288502A11D104F1E8
:10537000080500F108012846FBF742FB22460023FE
:1053800032F8400B2946F5F767F9638BA4F85830DB
:1053900067E7002320881A461946F5F75DF960E7AC
:1053A000037A03F00F02012A05D81F2B03D800232C
:1053B00084F85A3055E7B4F85820A0780221F4F761
:1053C00035F938B9002320881A461946F4F72AF926
:1053D0000223EDE7C28800F1080103232088F4F7D7
:1053E00021F90028F4D0EDE70229010072840600BB
:1053F0002DE9F04FA84BA94AD3F80003002385B04C
:105400001C4601251E4605FA03F1084209D052F850
:10541000237037B10C4342F82360BFF36F8FBFF3A3
:105420004F8F0133192BEED1E7071AD50022114611
:10543000930003F1804303F51C330132082A5960BD
:105440009962F5D1944B59629964954BC42200211D
:105450001846FFF7C7FA4022027502720120FBF7D7
:10546000D7FCA60202D50320FBF7D2FC650213D5B8
:10547000894ED6F8005405F44073E805C6F80034A8
:1054800005D50420FBF7C4FC0123C6F82C35A9057B
:1054900002D50520FBF7BCFC824B814E234033B183
:1054A00096F8C030002B40F0D380F4F761F8220268
:1054B0003BD5794BD3F880E4D3F88424D3F888140F
:1054C000D3F88C74D3F89054D3F894045FFA81FC29
:1054D000D3F89814D3F89C341EF07F0F5FFA8EF83F
:1054E000D2B2FFB2EDB2C0B2C9B2DBB201D1052A6D
:1054F0001BD04FF0000EADF806E08DF80D004FF414
:10550000C06E8DF80E1001A80121ADF804E08DF8F1
:1055100008808DF809208DF80AC08DF80B708DF881
:105520000C508DF80F30FBF741FC5D4FDFF86891B0
:10553000B84600254FF0010A4FF0140B05F10C039B
:105540000AFA03F32342E9B21BD00BFB05930020B8
:10555000D3F80827182303FB0563D2B2587298F8D2
:1055600008C094457DD1DB88B8F804209BB29A42EC
:1055700077D9002D70D1C9F84CA0BFF36F8FBFF35E
:105580004F8F0135082D08F11808D7D1464B23401D
:10559000002B5AD0404BD3F86C84C3F86C84BFF313
:1055A0006F8FBFF34F8F14F4806407D0D3F880441B
:1055B000D3F880341B06C4F3C0145FD54FF0000A43
:1055C000DFF8DC9000254FF0140B0123AB4013EA09
:1055D000080FE8B201D1ADB9A4B12F4B0BFB0533D5
:1055E000D3F80416182303FB05635A8A11FA82F2D2
:1055F00092B25A825A8AB9F8101092B2914240D9A6
:10560000FBF7BAFD0135082D09F11809DDD1002499
:1056100001254FF0180904F1100305FA03F313EA0A
:10562000080FE0B203D15CB9BAF1000F08D009FB52
:105630000462B988D3889BB299422BD9FBF774FDD9
:105640000134082C07F11807E5D105B0BDE8F08F4B
:10565000002386F8C0302AE705F5947349F8230043
:105660008BE7182303FB05630020DA88A8F80420E1
:10567000DA88012392B2FBF717FD82E74FF0010AA7
:105680009EE75A8A40F08001012392B20020FBF786
:105690000BFDB7E75572D3E700700240007102407E
:1056A000E82E0120FCFB1F000004000110B502449D
:1056B000904201D1002010BD10F8014B11F8013BC0
:1056C0009C4202D3F4D90120F5E74FF0FF30F2E716
:1056D0002DE9F84F80460D46F1F7C0FF134B5C698A
:1056E00007460CB920461EE0E36804F1100B0BEBF3
:1056F00083095E464E45B24601D32468F1E756F869
:10570000040B0378BB42F5D14378AB42F2D12A4671
:1057100041460230FFF7CAFF0028EBD16068AAEBD0
:105720000B0A00EBAA00BDE8F88F00BF804E0120F5
:10573000884237B504460D4608D1F3F73FF828B93B
:10574000A10766D12268374B9A4262D1364B9C4200
:1057500002D1002003B030BD9D42FAD0E20704D54B
:10576000EB07F6D423462C461D46304B2F4A2340E8
:10577000062B02EA050205D0A00733D120682C4988
:1057800088422FD1062A46D0A907E2D128682849A5
:105790008842DED1062B05D1E008F1F751FF0178F0
:1057A0006B6806E0062A6168FAD1E808F1F748FF5D
:1057B000037811B10BB19942CBD169462046F3F77A
:1057C00089FA01A904462846F3F784FADDE90023A3
:1057D0009A420146BDD12046FFF768FFB0FA80F03B
:1057E0004009B7E7062AB4D0AB0703D12A68104BAB
:1057F0009A42AED02046F2F7F7FF8369002BA8D07B
:105800002A462146022098470028A2D0094CA042EF
:1058100004E001209EE7062BC4D1AC4214BF002057
:10582000012097E76C7806006C540600070080FFA3
:10583000387F060070540600F8B51746044600EBA2
:1058400081060025B44203D1680040F00100F8BD94
:1058500054F8040B3946FFF76BFF0028F2D00135EE
:10586000F0E7000007B501910549F3F7AEFBD0E979
:105870000210019A03B05DF804EBFFF7DDBF00BF33
:10588000F07B06000A46083050F8041CFFF7D4BF2E
:10589000022838B50D46144613D1930701D00A48A3
:1058A00038BD1268094B9A42F9D1A168A868FFF780
:1058B0003FFF0028F3D022792B799A42EFD1044898
:1058C000EEE70020ECE700BF645406009C1B0600D6
:1058D000705406002DE9F0479942DDF820A080467B
:1058E00091461E4613D3BAF1010FA1EB030416BF74
:1058F00025460025002408EB050732464946384670
:10590000FFF7D4FE20B1A54201D05544F3E70027AC
:105910003846BDE8F08770B50446022C049E154653
:10592000184610D1B24226D1024608461146AE4270
:10593000324628BF2A46FFF7B9FE022C0ED1B0FA34
:1059400080F0400970BD2CB1032C05D032462E46A4
:105950001546E9E70124EAE70424E8E700280ADB22
:105960000BD1AE4203D02CBF01200020EAE7601E1D
:1059700018BF0120E6E70020E4E70120E2E72DE977
:10598000F74F9DF8306007468A46904699460024B6
:105990004C4502D386F0010619E018F804B0013432
:1059A000002508EB0401554501D35C44F0E77B5D1D
:1059B0000135002BF9D09B450DD85A467819019333
:1059C0000091FFF773FEDDE9001320B92EB13046D8
:1059D00003B0BDE8F08F002EF9D01D44E3E70000CE
:1059E0002DE9F04F03881B2B89B005460C460ED1DC
:1059F000057A012D4FF0000006D1486081F8215052
:105A00003548F3F7FBFD284609B0BDE8F08F1D2BA4
:105A100060D1F5F77BF804F1080602460B46CDE9A4
:105A20000623A98CA3892F7A95F80A80ADF8161061
:105A30003046039395F91BA0D5F82090F4F797FD15
:105A4000039B1331181A814207F0010B4FEA5808E3
:105A5000C7F3C00734DAE3699A4531DBA36943B180
:105A600001220092BDF8161062694846FFF787FFD1
:105A700030B359460FB14BF002013046F4F765FDE3
:105A8000082206A93046F4F70EFE5FFA8AF1304686
:105A9000F4F75BFD062205F10B013046F4F703FE37
:105AA00041463046F4F751FD02220DF11601304611
:105AB000F4F7F9FD9DF8162049463046F4F7F3FD5A
:105AC00061680020F4F7C8FC012308B184F8213094
:105AD000184699E7002097E7E159030003460020A4
:105AE0001A5C02B970470130FAE700002DE9F04F67
:105AF000814689B0144600260B461D4613F8012B3B
:105B000082B9A94211D30B78002B00F03A81013100
:105B100020234FF000080A4612F8015B7DB94FF0D0
:105B20000A0C2AE0252AE8D1EBE76F1AD9F80430ED
:105B3000D9F800003A4698473E442946E3E72D2D20
:105B400003D148F001081146E5E72B2D02D148F0BA
:105B50000208F8E7202D02D148F00408F3E7212DD0
:105B600002D148F00808EEE7302D21D148F0400876
:105B70002B46E8E70CFB0525303D0F4611F8012BBD
:105B8000A2F130000928F5D92E2A41D17A782A2AA3
:105B900010D000204FF00A0C0F4611F801BBABF1FA
:105BA0003002092A09D80CFB00BBABF13000F3E747
:105BB0000025B4E754F8040B023720EAE07B3A787A
:105BC0006C2A08BF013797F800A0BAF1000F00F067
:105BD000D880BAF1780F6AD8BAF1570F1BD8BAF14A
:105BE000470F61D8BAF1440F61D9073424F0070494
:105BF000F4E802010593F1F7D5FBCDE9005B00EE77
:105C0000100A059B424651464846F8F78CFD62E073
:105C10004FF0FF3BD3E7AAF15802202A47D801A151
:105C200051F822F0615D0300AF5C0300AF5C03003C
:105C3000AF5C0300AF5C0300AF5C0300AF5C03002C
:105C4000AF5C0300AF5C0300AF5C0300C15C03000A
:105C5000E35C0300455D0300EB5B0300EB5B0300CB
:105C6000EB5B0300AF5C0300AF5C0300AF5C0300C1
:105C7000AF5C0300AF5C0300AF5C0300AF5C0300EC
:105C8000AF5C0300775D0300F75C0300AF5C0300CB
:105C90001B5D0300AF5C0300335D0300AF5C0300DA
:105CA000AF5C0300615D0300BAF1500F63D0D9F817
:105CB0000430D9F8000001223946984701360BE03C
:105CC00054F8042BCDE9003543463AB12F4904225C
:105CD0004846F1F7E7FC0644791C0DE72C490522FC
:105CE000F6E754F8042B8DF81C20CDE9003501228D
:105CF000434607A9ECE707A954F8040B0593F1F70D
:105D0000C2FCBBF1FF3F059B014601D1DDF81CB091
:105D1000CDE900355A464346DAE7BBF1FF3F54F878
:105D2000041BF5D108460593FFF7D8FE059B834673
:105D3000EEE7CDE9023561230093CDF804800A2314
:105D4000002207E0CDE9023561230093CDF80480FD
:105D50000A23012254F8041B4846F1F701FDBAE773
:105D6000AAF1170ACDE90235CDF804805FFA8AF36B
:105D700000931023E4E7CDE90235CDF804806123D8
:105D8000F6E7304609B0BDE8F08F00BF92CE0500BF
:105D900097CE05000EB403B503AA52F8041B019276
:105DA000FFF7A4FE02B05DF804EB03B070470000FB
:105DB00013B5044608460191FAF7EAFD019B044930
:105DC0000246204602B0BDE81040FFF7E3BF00BF27
:105DD0009DCE050010B504468868FAF7D9FD024645
:105DE0000B4620460249BDE81040FFF7D3BF00BF75
:105DF000B3CE05004A680149FFF7CCBF3DCF05008F
:105E000030B4064B0D68064C0A4606498D420CBF5D
:105E10002146194630BCFFF7BDBF00BFE4CE0500E8
:105E2000D1CE0500747F0600CA880149FFF7B2BFD2
:105E3000F6CE05000A460149FFF7ACBF03CF0500C7
:105E40004A680149FFF7A6BF0BCF050013B504460A
:105E500008460191F2F7FFFC019B044902462046E7
:105E600002B0BDE81040FFF795BF00BF1ACF050094
:105E70004A680149FFF78EBF25CF050007B5094BDA
:105E80008B4214BFCF21A1214FF494730191009351
:105E900005494FF4A9734FF4CE72FFF77BFF03B0AF
:105EA0005DF804FB2829060034CF050007B5074B31
:105EB0008B4214BFB021D3210091842304494FF4B5
:105EC000F172FFF767FF03B05DF804FB483206008C
:105ED00037CF050007B5084B8B4214BF4FF49171C3
:105EE000D1210091862305494FF4F172FFF752FF4B
:105EF00003B05DF804FB00BFA832060037CF0500F1
:105F000007B5094A40F253138A4214BF194680214B
:105F100000914FF4977305494FF4F172FFF73AFF80
:105F200003B05DF804FB00BF2C33060037CF05003B
:105F300010B586B0044603AB084604AA05A9F5F7D8
:105F4000D1F8039B0093054940F2C32340F28F220E
:105F50002046FFF71FFF06B010BD00BF37CF05007A
:105F60000B4B994207B50FD00A4B994214BFC92178
:105F7000712100914FF49D73074940F28F22FFF782
:105F800009FF03B05DF804FB40F23D11F1E700BFEB
:105F9000485006001850060037CF05001FB50C46C4
:105FA000114602AA0092094A0192CDE902041A465A
:105FB0006846FFF79BFD24B1DDE902321AB903F808
:105FC000012C04B010BD00221A70FAE77D0A03000C
:105FD0000CB407B504AB53F8042B0193FFF7DEFFB5
:105FE00003B05DF804EB02B0704700000FB407B5D2
:105FF00004AA054852F8041B0192FFF777FD03B08D
:106000005DF804EB04B070472C5E060038B5054619
:106010000846FFF763FD044618B102466B6828681E
:106020009847204638BD00002DE9F0478CB0044663
:1060300000AF08460E46F2F7B1FF50B32A4B1B687B
:1060400023B11B681A68294B9A4222D107F1080232
:10605000391D3046F2F7D6FC7B68D3B1E8468AB0EA
:1060600069462348DFF89490F3F7E8F907F118013F
:106070002048F3F7E3F907F10C011F48F3F7DEF9C5
:1060800069462046FFF7C2FF7D68033D002D0DDA0B
:10609000C54602223146204608F08AF817492046B4
:1060A000FFF7B4FF3037BD46BDE8F087BA6802EBB2
:1060B000850307F118015B6852F825202046FFF799
:1060C00069FEBB684FEA850A53449A682AB9494673
:1060D0002046FFF79BFF033DD8E707F10C01204660
:1060E000FFF758FEF7E700BF3C510120EF29780188
:1060F00052B70600FACB06007ABA060025D9050089
:1061000010B594B0044602A80191F1F7A3F938B98B
:106110000199204602F08AFEF1F794F914B010BDFF
:1061200002480399FFF780FF0020F7E72C5E060086
:106130002DE9F04F6A4ED6F80431D6F8F08085B0DC
:10614000002B6AD000254FEA88024046C6F8045169
:10615000002A50D00024D6F8EC70A10804F0030304
:10616000795C5B0041FA03F303F00303032B32D0A5
:1061700001349442EFD3D6F80431002BE6D18046A7
:10618000D2B34FF0000E75464FF003094FF0020BEB
:1061900004E0012B4FD0013595422DD2D6F8EC10FA
:1061A000AF0805F00304C85D640040FA04F303F08F
:1061B0000303022B01EB950C32D0032BE9D10BFA30
:1061C00004F420EA0400C855D6F8F0804FF0000E21
:1061D0004FEA8802DFE72046F1F754F9D6F8F000DD
:1061E0000134B4EB800F4FEA8002B4D3D6F8043107
:1061F000002BABD1C3E78046202200213948FEF7AF
:10620000F1FBB6F8082208F1FF33013AC6F82C3248
:10621000A6F8082205B0BDE8F08F4FEA8802AFE784
:10622000BEF1000FB7D009FA04F420EA0400C85503
:10623000D6F8F080CCE7D6F8F4104FEAD50A05F08E
:10624000070811F80A3043FA08F2D20701EBD5012A
:1062500028D5D6F8F8002A01825800EB05100090E6
:10626000AAB100230022CDE90223F2F7BDFAC369E7
:10627000019013B3009802AA0C219847029810B11C
:106280000399FFF73DFFD6F8F41051440B78012233
:1062900002FA08F823EA08030B70D6F8EC30D85D50
:1062A00003EB070C09FA04F420EA04008CF8000060
:1062B000D6F8F0804FF0010E8AE7019A906B002823
:1062C000E4D01A460430662110F000FE0028D5D034
:1062D000426802ABDDE900010AF0A4FACEE700BF94
:1062E000804E01208C50012030B58BB0FAF796F922
:1062F0006846F0F785FE164C054604211548FAF766
:1063000059F9236C2BB1144A934214D1E06CFAF77B
:10631000E5F912480A21FAF74DF91148AA21FAF7CE
:1063200049F91049491B89082846FAF743F9FFF74C
:10633000FFFE0BB030BD0C4A9342EAD1E06CFAF795
:10634000CDF9D4F8B400FAF7C9F9D4F8BC00DEE707
:1063500088490120584F0120D8350600BC21012072
:10636000C046012000000420C43606002DE9F04F8D
:106370000F3087B005090591029200F09080B44B70
:10638000D3F8F820002A00F00281B149B1F80832B0
:10639000002B40F08480D1F8003191F80AE29B1A7A
:1063A000029A48BF0F33002A14BF032100214FEA8D
:1063B000231314BF4FF0FF384FF001080193082D4D
:1063C0004FEA41032A46039328BF0822A04B0091BD
:1063D000813203EB82038EF0010E0493049BD3F809
:1063E0000490029B002B5FD1994BD3F82CA24E4610
:1063F000974BD3F8ECB000220324B14549D8564559
:1064000047D8B8F1FF3F1BF806104FEA860052D07C
:10641000B8F1010F79D0009BBEF1000F00F08D8024
:106420005C000323A3401940002942D10132954268
:10643000FCD8009B03440299002940F0AB805C1C0F
:10644000072DA4EB020422D8814F05EB030107EBD3
:1064500085064FEA91013046C6F80812C6F80C12BC
:1064600015D0062DC0F8101211D0052DC0F8141249
:106470000DD0042DC0F8181209D0032DC0F81C123D
:1064800005D0012DC0F8201201D1C7F828121D46F1
:1064900088E0954240F2D980BEF1000F18D0002369
:1064A000184607B0BDE8F08F694BD3F82C62B246AE
:1064B0009EE70022B8E70323BEF1000F0DD15F0075
:1064C00004FA07F70F4213D0019F1A18BA425BD2A1
:1064D000FFF70AFF4FF0010E80E75F0004FA07F7AD
:1064E0000F420DD0013B00225F1CF6D1464484E7E9
:1064F0000132AA429ED2013B5F1CE0D146447CE7B8
:106500000132954296D9013BEEE7BEF1000F2AD148
:10651000734607E0019F1A189742D9D90133002228
:10652000042BE3D05F0004FA07F70F42F2D10132E7
:1065300095427FF67FAF0133F2E7DDF80CC004FA35
:106540000CF70F420AD00133042B4FF00002CDD0DC
:106550004FEA430C04FA0CF70F42F4D10132954292
:106560007FF668AFEBE7002303E001330022042B42
:10657000BCD05F0004FA07F70F42F6D10132954212
:106580007FF658AF0133F2E7013B0022B4E7082061
:10659000F2F7E2FE2E48591E8908D518C0F82C12D1
:1065A000013D1C46A00804F0030359001BF80060DD
:1065B00001238B40611C33438D420BF8003011D313
:1065C0000227234B8808D3F8EC6001F0030316F888
:1065D00000C05B0007FA03F3013143EA0C038D426C
:1065E0003354EED21A4B0299D3F8F850260105EB3A
:1065F000041331B11648D0F80011994288BFC0F891
:10660000003113F003014FEA021219D000211AB130
:106610001846FEF7E7F90346059A002A3FF440AF13
:106620000022AA510A4AE108D2F8F40004F0070453
:10663000455C012202FA04F444EA050242542FE7C1
:106640009008002AE8D08200E2E74FF0FF33F2E63C
:10665000804E01200A460021FFF788BE2DE9F34154
:1066600000240E460746194630464FF6FF73904603
:106670000094224603F022FC21461020FFF7EAFF97
:106680000F4DA04218BF05462F60AC602EB90D4CCF
:10669000EC60284602B0BDE8F081B71CBF0021467F
:1066A0003846FFF7D7FF04460028F0D0064BA7F185
:1066B0000802C0E9003641460830FAF7A1F9E7E7D9
:1066C000984E01205C540600EC7F06002DE9F04F47
:1066D0000D4687B0002100AF064610209046FFF718
:1066E000B9FFB5F800A00AF1010A0446002150469E
:1066F000FFF7B0FF4CB92346224621463046FFF74C
:10670000ADFF1C37BD46BDE8F08F07F1080968B939
:10671000C4E90200184B2360D4E90210F0F79EFF91
:10672000002360604A46BC600121E7E701233B7219
:10673000124B7B602B88C7F80CA00733EB46DB08B5
:10674000ABEBC3039D464FF0000A6946C7E904A0BE
:106750002846C7F80090F2F771FE4246694638466F
:10676000FFF7C4F9D7E9043202F803A03B69A3603C
:106770007B69E360DD46CDE7387F060001EC04006D
:106780000EB403B503AA52F8041B0192FFF79EFF53
:1067900002B05DF804EB03B0704708B519B9F2F721
:1067A0002CF9F7F7D7FCFFF7EBFFFAE7014608B53E
:1067B0000148FFF7F2FF00BF946E0600136870B542
:1067C00093B90468E56B4034AB4200D170BD54F816
:1067D000046BB14201D00133F6E7591CF6D0023305
:1067E00050F823301360F1E70148FFF7DFFF00BFE7
:1067F000B4BA060007B5436802461B7900936846A1
:10680000F3F720FA536801461B79019301A8F3F7C7
:1068100019FA019B03F5E07350F82330DA0702D52B
:106820000948FFF7C3FF009B03F5E07351F823000D
:10683000C0F38100012805D0C31E5842584103B05F
:106840005DF804FB0220FAE70EC9060008B501480E
:10685000FFF7ACFF6ACC0600014608B50148FFF718
:106860009CFF00BF0873060007B5064A136852680C
:1068700001A95B1A9A4202D80348FFF7EDFF03B063
:106880005DF804FB804E012098AF06002DE9F74F1C
:10689000DDF8308004460D4617469B46FFF7E4FFBF
:1068A0004FF002094FF0010A20784F2803D87B6887
:1068B000AB4240F2A880512804F1010600F0A58007
:1068C0000ED8052807D848B1831E032B23D8DFE84C
:1068D00003F027292945502800F091803446E3E74A
:1068E000622868D011D8602860D06128F6D1A61C33
:1068F0005B466478CDF800803A4629463046FFF77B
:10690000C5FF30B946FA84F6E8E77E2861D07F28D3
:10691000E4D1012047E02A7863789A4273D1A61C1B
:106920000135DBE7637804341A461AB9033818BF17
:1069300001200BE0297814F802CC8C450BD814F810
:1069400001CC8C4507D3C21E5042504158B319FBAD
:1069500003A31E44E4E70234013AE6E7637843F018
:10696000200164294FEA5312C3F340102B7806D15B
:10697000303B092B15D9D04300F0010011E07329F9
:1069800004D1202B0DD0093B042BF3E723F0200189
:106990004139192905D9A3F13001092901D95F2B02
:1069A000E9D10028BBD103B0BDE8F08F94F90160B4
:1069B0000236264492E794F90100CDF80080A61C27
:1069C0005B463A4629463044FFF760FF0028A0D1D5
:1069D00084E7A61C6478444580DA24B2CDF80080B0
:1069E0005BF824904BF824505B463A4629463046E3
:1069F000FFF74CFF00288CD14BF82490D3E73B687D
:106A0000AB423FF46BAF0020CDE77B68F8E70000B6
:106A100008B50148FFF720FF80B6060070B50546AF
:106A20000C468E18B44200D170BDD5E900039847DA
:106A3000431C01D1FFF7ECFF04F8010BF2E738B576
:106A400004460025D4E900039847421C01D1FFF712
:106A5000DFFF00F07F0343EAC5150306F2D42846A2
:106A600038BD000008B50148FFF7F6FE1EC006005D
:106A700008B50148FFF7F0FE36B9060008B5014831
:106A8000FFF7EAFED0BC060008B5037A0BB9FFF7A2
:106A9000F5FF08BD08B5037A0BB9FFF7EFFF08BD96
:106AA00008B5037F0BB9FFF7E9FF08BD08B501483A
:106AB000FFF7D2FE0CC4060008B50148FFF7CCFE74
:106AC00054BA060008B5F8F779F808B9FFF7F4FFEB
:106AD000004808BD6C54060008B5F7F7C7FF08B9B1
:106AE000FFF7EAFF004808BD6C54060008B50148EE
:106AF000FFF7B2FEAEB20600014608B50148FFF747
:106B00004CFE00BF38700600014608B50148FFF78B
:106B100044FE00BFAC74060008B50148FFF7F4FF5F
:106B200012C5060070B5054608466E680EB9FFF737
:106B3000F3FF7468A9688C420DD9641AB368944253
:106B400028BF144619442246F9F75AFFAB6823447C
:106B5000AB60204670BD0024FBE70000402808B56C
:106B600067D00DD800F0FD003C2809D1782907D85E
:106B7000612908D8422968D04839CBB2092B3CD9C1
:106B80006248FFF7C1FF62391629F9D801A353F80B
:106B900021F000BF4B6C0300816B03002D6C0300E0
:106BA000816B0300F16B0300816B0300036D030035
:106BB000F16B0300816B0300816B0300F16B030039
:106BC000816B0300816B0300816B0300816B030009
:106BD0002D6C0300816B0300816B0300816B03004C
:106BE000816B0300816B0300816B03004B6C03001E
:106BF0000121042002B1116008BD0929C0D801A3F8
:106C000053F821F0036D0300F16B0300816B030067
:106C1000816B0300F16B0300816B0300816B030048
:106C2000816B0300816B03002D6C030001210820A0
:106C3000E0E77829A4D8612909D85129A0D84729A3
:106C40003CD8012959D042299AD1012155E0623915
:106C5000162995D801A353F821F000BF4B6C03000F
:106C6000816B0300FF6C0300816B0300B96C0300B0
:106C7000816B0300096D0300B96C0300816B030095
:106C8000816B0300B96C0300816B0300816B03000F
:106C9000816B0300816B0300FF6C0300816B0300B9
:106CA000816B0300816B0300816B0300816B030028
:106CB000816B03004B6C030004219AE748390929D2
:106CC0003FF65EAF01A353F821F000BF096D03004A
:106CD000F96C0300816B0300816B0300F96C030006
:106CE000816B0300816B0300816B0300816B0300E8
:106CF000F56C030008219AE7042108467AE7082189
:106D0000FBE70121022075E70221F6E7FECA060033
:106D100070B50D460179044601F07F01164640200A
:106D20000022FFF71BFFE2682A60A36843436B6001
:106D3000237903F07F03AB602168094B99420BD1A3
:106D400094F90430002B01DBB30707D46368C3F365
:106D5000172300FB03202860002070BD0120FCE702
:106D6000687C060008B50148FFF7CEFE84B4060033
:106D700008B50148FFF7C8FEACCA060008B50148CF
:106D8000FFF7C2FE84CA060008B50148FFF7BCFE43
:106D90003ABA060008B50148FFF7B6FE6AAF06002A
:106DA00008B50148FFF7B0FE96B9060008B50148DE
:106DB000FFF7AAFE7CBF060008B50148FFF7A4FE56
:106DC00058AD060008B50E4B98424FF0804314D0E2
:106DD0000C4A904209D00C4A904202D00B48FFF76F
:106DE00093FE5722C3F81C2505E00022C3F81C259A
:106DF000074B084A1A60084808BD0022F2E700BFA6
:106E0000445006004850060018500600C8C306004B
:106E100060510120AF0900AD6C54060008B501486F
:106E2000FFF772FEA2C9060008B543680BB9FFF769
:106E3000F5FF08BD13B50446FFF7F6FF0DF1070097
:106E4000F3F74AFB04F10C00F3F791FB04469DF8BD
:106E50000700F3F79DFB600040F0010002B010BD99
:106E600013B50446FFF7E0FF0DF10700F3F734FB1D
:106E700000239DF807006382A382F3F789FB014892
:106E800002B010BD6C54060008B5034B42689A422C
:106E900001D1FFF7C3FF08BD6C54060010B50446CE
:106EA000FFF7F2FF2046F7F7A1FE034A034B002845
:106EB00014BF1046184610BD4832060024320600A2
:106EC00010B50446FFF7E0FF2046F7F7E7FF034A57
:106ED000034B002814BF1046184610BD705406001E
:106EE0006454060038B50D460446FFF7CDFF0A4B43
:106EF0009D4205D100212046F6F7ECFB074838BD3E
:106F0000074B9D4205D1002211462046F7F75DFD53
:106F1000F4E70448FFF7F8FD243206006C5406003D
:106F2000483206008AAF060038B504460D46FFF722
:106F3000ABFF2046F7F75AFE10B90648FFF736FCBC
:106F40002846F8F7F9FE01462046F7F737FD0248D4
:106F500038BD00BFEEB906006C54060013B50446F8
:106F6000FFF792FF2046F7F741FE08B9FFF76EFCE6
:106F7000636801A81B790193F2F764FE019B074A3D
:106F800003F5E07350F823300548C3F30223063BB2
:106F9000012B98BF104602B010BD00BFA8320600FA
:106FA000AC32060038B504460D46FFF76DFF2046AB
:106FB000F7F71CFE08B9FFF749FC04496B1A594260
:106FC00020465941F7F758FC014838BDA832060061
:106FD0006C54060010B50446FFF756FF2046F7F73D
:106FE00005FE012802D10848FFF7E0FB2046FFF725
:106FF00001FC012806D0054B054A022814BF18469B
:10700000104610BD0348FCE788B706006C54060024
:107010002C3306008C33060038B505460C46FFF7C6
:1070200033FF2846F7F7E2FD012802D10C48FFF7AD
:10703000BDFB0C4B9C4208D00B4B9C420BD00B4B26
:107040009C420AD00A48FFF75FFD01212846F6F767
:1070500036FB064838BD0221F8E70021F6E700BFFD
:1070600088B706008C3306002C3306006C540600EB
:1070700016BE060010B586B00446FFF705FF334B79
:107080009A88ADF814201868314A9B798DF816302B
:10709000032304900121C2F8F0350023C2F8F4352F
:1070A000C2F8001519461A0102F1804202F5E042C9
:1070B0000133082BC2F81415C2F81015F3D104A837
:1070C000F6F7BCF963685A79214BC3F81425C3F865
:1070D00010250DF10202C3F82C260122C3F8302638
:1070E0001A6003F580731A68002AFCD000221A6027
:1070F0001B680193019B174B01221A6003F58073F3
:107100001A68002AFCD000221A601B680293029BB6
:10711000114B01221A60114A1368002BFCD0002386
:10712000136012680392039A094AC2F80035BDF948
:1071300002209A42B8BFADF80230BDF802008000CC
:1071400080B2400040F0010006B010BD58CE0500EE
:10715000007000400470004008700040147100404E
:1071600008B5FFF791FE014808BD00BF3233D3C018
:1071700008B590F82330FF2B01D1FFF74FFE08BD73
:1071800010B50446FFF7F4FF054B064801225A608C
:1071900094F8263043F0040384F8263010BD00BF75
:1071A000005002406C54060010B50446FFF7E0FFA3
:1071B0000A4BD3F8082142B194F826206FF341021C
:1071C00084F826200022C3F8082194F826300448C9
:1071D00013F0020F034B08BF184610BD00500240C9
:1071E000705406006454060010B50446FFF7C0FF53
:1071F00094F82630034813F0080F034B08BF1846D5
:1072000010BD00BF705406006454060010B504465B
:10721000FFF7AEFF94F8263003481A0744BF6FF318
:10722000C30384F8263010BD6C54060010B5044624
:10723000FFF79EFF0C4BD3F8082142B194F82620AB
:107240006FF3410284F826200022C3F8082194F845
:1072500026309A0701D4FFF70BFC43F008030348DC
:1072600084F8263010BD00BF005002406C54060068
:1072700008B543680BB9FFF7D1FD08BD10B504464A
:10728000FFF7F6FFA06A400040F0010010BD10B506
:107290000446FFF7EDFFA07E400040F0010010BD66
:1072A00010B50446FFF7E4FF94F82400400040F0D6
:1072B000010010BD08B543680BB9FFF7AFFD08BD6D
:1072C00010B504462C34FFF7F5FF14F8082C002302
:1072D000D9B2914201D3054810BD54F8041B896806
:1072E00001330029F4D00248F6E700BF64540600D9
:1072F0007054060010B50446FFF7DCFFA06A10BD0D
:1073000010B50446FFF7D6FF6069400040F0010069
:1073100010BD08B543690BB9FFF780FD08BD10B576
:107320000446FFF7F6FFA06A10BD10B50446FFF74C
:10733000F0FF606A400040F0010010BD08B5FFF7A3
:10734000E8FF212008BD10B50446FFF7E2FF94F8DE
:107350002D00400040F0010010BD08B583680BB956
:10736000FFF75CFD08BD000010B50446FFF7F5FF10
:107370002046F8F787FC014810BD00BF6C5406009A
:1073800010B50446FFF7E9FF2046F3F79BFA034ADE
:10739000034B002814BF1046184610BD7054060059
:1073A0006454060010B50446FFF7D7FF94F8200098
:1073B000034A044B002814BF1046184610BD00BFF6
:1073C000705406006454060010B50446FFF7C5FF6C
:1073D00094F820307BB1A3680421002284F8202097
:1073E000C3F80012A368D3F8041121B1C3F8042133
:1073F000A36801229A60014810BD00BF6C540600CA
:1074000010B50446FFF7A9FF2046F3F75BFA08B969
:10741000FFF72EFB012384F82030A36802480222E4
:10742000C3F8002210BD00BF6C54060008B5034B22
:1074300082689A4201D1FFF7F1FC08BD6C54060046
:1074400010B50446FFF7F2FFF3F716FB237F1BB1DD
:10745000F3F72CFB034810BD01232377F3F726FB3A
:107460000148F8E7645406007054060010B504465D
:10747000FFF7DCFF00230148237710BD6C540600A2
:1074800008B5034B82689A4201D1FFF7C7FC08BDDB
:107490006C54060010B50446FFF7F2FF2046F7F7DC
:1074A00054FD034A034B002814BF1046184610BD74
:1074B000705406006454060010B50446FFF7E0FF60
:1074C0002046F7F723FD034A034B002814BF10465C
:1074D000184610BD705406006454060038B50D46B9
:1074E0000446FFF7CDFF2846F8F726FC0146204664
:1074F000F7F777FA004838BD6C54060008B5034B1F
:1075000082689A4201D1FFF789FC08BD6C540600DD
:1075100010B50446FFF7F2FFF3F7AEFA94F8203007
:10752000DB0603D5F3F7C2FA054810BD94F8203006
:1075300043F0100384F82030F3F7B8FA0148F4E779
:10754000645406007054060010B50446FFF7D6FFD9
:1075500094F8203002486FF3041384F8203010BDF3
:107560006C54060008B5837AFF2B01D1FFF756FC57
:1075700008BD000010B50446FFF7F4FF237A1BB9DD
:1075800001230248237210BD0148FCE77054060035
:107590006454060010B50446FFF7E4FF00230148D9
:1075A000237210BD6C54060008B5034BC2689A42A2
:1075B00001D1FFF733FC08BD6C54060010B504463A
:1075C000FFF7F2FF201DF7F7C0FC034A034B00282A
:1075D00014BF1046184610BD7054060064540600CF
:1075E00010B50446FFF7E0FF201DF7F78FFC034AB4
:1075F000034B002814BF1046184610BD70540600F7
:107600006454060038B50D460446FFF7CDFF284602
:10761000F8F792FB0146201DF7F7E3F9004838BD63
:107620006C54060008B5437AFF2B01D1FFF7F6FB37
:1076300008BD000010B50446FFF7F4FF0023014821
:10764000237210BD6C54060010B50446FFF7EAFF24
:1076500063681B68D3F82435B3F1805F23D013D857
:10766000B3F1006F21D00BD8B3F1007F1FD01348C6
:10767000B3F1806F18BF0020400040F0010010BD42
:107680000F48B3F1206FF5E7B3F1804F11D006D862
:10769000B3F1A05F0FD00B48B3F1005FEAE70A48EF
:1076A000B3F1004FE6E70948E6E70948E4E709488F
:1076B000E2E70948E0E70948DEE700BF90D00300B1
:1076C0000024F40080841E0000127A0040420F0063
:1076D00020A1070048E8010000093D000048E8013A
:1076E00008B5837FFF2B01D1FFF798FB08BD10B5CC
:1076F0000446FFF7F5FFA068400040F0010010BD10
:1077000010B50446FFF7ECFF04F11000F2F72FFF6D
:10771000400040F0010010BD10B50446FFF7E0FF47
:10772000D4ED037A9FED077AF8EE677AC7EE877A91
:1077300017EE900A20F0030040F00200A0F1FF4095
:1077400010BD00BF00007A4410B50446FFF7C8FF23
:107750006368186840F30730F2F752FA0023E382B7
:107760002383636806481B68012143F30732C3F390
:10777000043301FA03F35209024941F8223010BDE3
:107780006C54060000E100E0F8B50F461E460546C1
:107790001446FFF7A5FF40F201139F4216D114F0E3
:1077A000010006D005F11000F2F7E1FE003818BF25
:1077B0000120630709D56B68074A1B79242101FB67
:1077C00003235B690BB940F00400F8BD1623336056
:1077D0004FF0FF30F9E700BF984D012008B543682E
:1077E0000BB9FFF71BFB08BD10B50446FFF7F6FF0A
:1077F0006089400040F0010010BD10B50446FFF75D
:10780000EDFFE068400040F0010010BD08B50379CD
:10781000FF2B01D1FFF702FB08BD000010B50446A5
:10782000FFF7F4FF2079F2F7A9FD01230148A371C6
:1078300010BD00BF6C54060010B50446FFF7E6FF0C
:10784000A37913B92079F2F799FD0023E38123820C
:10785000A37913B92079F6F73FF9014810BD00BFAD
:107860006C54060038B50446FFF7D0FF238A9BB25C
:1078700013B91248FFF740F9A37913B92079F2F749
:107880007DFDE389A268A1899BB232F81350E38998
:107890009BB20133B3FBF1F201FB12339BB2E381E4
:1078A000238A013B9BB22382A37913B92079F6F78F
:1078B00013F9680040F0010038BD00BFE0C10600C8
:1078C00010B50446FFF7A2FFA089400040F0010078
:1078D00010BD000010B50446FFF798FFA079034AD9
:1078E000034B002814BF1046184610BD7054060004
:1078F0006454060038B50D4604460846FFF786FF77
:107900002B8A042C9BB203D0052C07D0002038BD55
:10791000044A0548002B18BF1046F8E7580040F00D
:107920000100F4E7705406006454060008B543688B
:107930000BB9FFF773FA08BD10B50446FFF7F6FF61
:10794000201DF7F793FB2189034A044B814234BF82
:107950001046184610BD00BF70540600645406005F
:1079600010B50446FFF7E2FF201DF7F77FFB40004C
:1079700040F0010010BD10B50446FFF7D7FF208985
:10798000400040F0010010BD08B503790BB9FFF7C6
:1079900045FA47F6015008BD08B543680BB9FFF733
:1079A0003DFA0069400040F0010008BD222808B5FA
:1079B00008D8431E1F2B09D81138012806D90448BE
:1079C000FFF7A2F8312801D04128F8D108BD00BF47
:1079D000CCBE060070B50E46054617493046F1F795
:1079E000F4FA08350446D8B914493046F1F7EDFAEF
:1079F000044610B91248FFF787F890F85030D906BE
:107A000001D51048F7E723F0140343F0140385620F
:107A100080F85030F3F728FEF3F769FE204670BD7A
:107A200090F82E309A07ECD443F0020380F82E3001
:107A30002946F3F7D3FEF1E764380600883C0600D8
:107A4000D4C8060052C30600F8B51646838D428D91
:107A50009A4204460D4602D10E48FEF7FDFE31461D
:107A6000FFF7B8FF628D0746AA42636809D843F85A
:107A70003570616801EBC5014E60638D013363852C
:107A8000F8BD03EBC20313E90300013A83E80300E6
:107A9000EAE700BF92B806007FB50446C08A984264
:107AA00002D82948FFF730F894F85000050745D56B
:107AB00004F12405208B02FB0050435494F850300D
:107AC000258BD807238CA1EB030191FBF5F305FB74
:107AD00013110EB254BF04F12C0001A8002EA38B89
:107AE000BCBF6D182EB213FB06F39BB20380A18BB3
:107AF0000B448380638C618BD21A92FBF1F301FB00
:107B0000132215B2002DE38BBCBF89180DB213FBF5
:107B100005F39BB24380E28B1344C38094F850304A
:107B2000DB0704D501A904F12C00F3F78FFE94F8CC
:107B3000503043F0010384F8503002E0656A002DB4
:107B4000B8D104B070BD00BFA2B70600F8B50025DB
:107B5000C0E901250446C1600582E3681A8BAFB213
:107B6000BA4215D84FF480321A6293F8502042F08E
:107B7000020283F85020F8BD00233946FFF78CFF3E
:107B80000136E068438BB2B29342F5D80135E4E7A1
:107B90000026F6E72DE9F047B0F80A8004460E46C5
:107BA0000D468F184FF00009BD4202D3A81BBDE857
:107BB000F0872846EFF736FE01462846EFF74FFEDE
:107BC0007F29054678D8A1F120035E2B0BD8606889
:107BD000F4F784F8034662892189E068FFF75CFFC7
:107BE000238901332CE00D291ED1A4F80890E36805
:107BF00021891A8B8A4208D8628901326281188BE6
:107C0000B1FBF0F200FB121222815A8B6189914282
:107C100022BFB1FBF2F302FB131363816389434577
:107C2000C2D04FF0000A56E00A2903D1638901331C
:107C30006381DCE7082905D12389002BD7D0013BDC
:107C40002381D4E71B29D2D103785B2BCFD1437892
:107C50004B2B11D1B4F808A0E0686289038B53451F
:107C600001D80235C3E7514600230AF1010AFFF7A4
:107C700013FF1FFA8AFAEFE7012100236A5CA2F1E1
:107C8000300CBCF1090FC8B20CD803EB830302EB34
:107C900043030131303B06299BB2EFD10846013046
:107CA000054481E7442AFAD122899A422ABFD31A8D
:107CB000A4F808902381F2E76068F4F70FF8FF2832
:107CC000034694D087E762890023FFF7E5FEB4F806
:107CD0000A800AF1010AE068038B1FFA8AF18B42DD
:107CE000F1D8418BA0F8209008EB01030133B3FBDE
:107CF000F1F201FB1233438490F8503043F0020359
:107D000080F8503050E7FFF745BF0000F8B50A464D
:107D100006460D4601460B480B4FFFF73BFF00247C
:107D2000AC4202D2F7F780FB00B9F8BD2A1B92B231
:107D300022B131193846F8F7F4FF02461444FCF733
:107D40009FFEEDE7AC22012044260120014608B544
:107D50000148FEF722FD00BF3474060008B5F0F7B5
:107D600091FD10B90148FFF7F1FF08BD62BA0600A6
:107D700010B50B4688B0044605A998680122FFF7A4
:107D8000EDFF059908780B794A79039048780290BD
:107D900088780190C978009120460249FDF7FAFFE2
:107DA00008B010BD40CF05007FB5044608466368A3
:107DB0000BB9FFF733F8022201A90834FFF7CEFF11
:107DC0002046DDE90165F2F7D2FB012820D9022225
:107DD0000DEB02012046F2F77CFC0DF10100F2F7F9
:107DE0007BFBBDF802309D4238BFADF802509DF8D4
:107DF000022031462046F2F76CFC9DF80100F2F7B4
:107E0000C7FBBDF80200400040F0010004B070BDA7
:107E10000020F8E72DE9F04F0C680D4685B02046AC
:107E2000FFF76CFB6868022201A9FFF797FF029E2B
:107E3000EEB12B6893F82030DD0601D4FEF71EFE6C
:107E400094F82030019DD80702D42E48FEF75CFE3E
:107E50009907E76904D5002104F10C00F6F7AEFD9F
:107E60002E4404F1040804F1140BAE4203D1264859
:107E700005B0BDE8F08F4FF0080A4FF0000994F804
:107E800020100A0728D43846F2F7ECFD94F82010A9
:107E9000C1F3800181F0010101F001014046F6F7D4
:107EA0008DFD5846F6F7FAFF94F8201040EA490095
:107EB0000B075FFA80F91CD43846F2F7D3FD94F82B
:107EC00020104046C1F38001F6F778FDBAF1010AAF
:107ED000D5D105F8019BC8E7C1F3800181F001010C
:107EE000404601F00101F6F769FD3846F2F7BAFDA8
:107EF000D7E74046C1F38001F6F760FD3846F2F758
:107F0000B1FDE3E73ABD06006C5406002DE9F04FE1
:107F10000D4685B00446FFF7F1FA012201A9284673
:107F2000FFF71CFF029FB7B194F82030D90601D4A7
:107F3000FEF7A4FD94F82030019D9A0702D428484A
:107F4000FEF7E2FDD4F81C802F4404F10C0B04F181
:107F50000409BD4203D1234805B0BDE8F08F15F8F0
:107F6000016B4FF0080AF1095846F6F727FD94F81F
:107F700020100B071DD44046F2F774FD94F8201032
:107F8000C1F3800181F0010101F001014846F6F7DB
:107F900015FD4046F2F766FD94F820104846C1F3FF
:107FA0008001F6F70BFD7600BAF1010AF6B2DAD1DC
:107FB000CFE7C1F3800181F0010101F001014846E2
:107FC000F6F7FCFC4046F2F74DFD94F820104846C9
:107FD000C1F38001F6F7F2FC4046F2F743FDE2E719
:107FE000F4C606006C5406002DE9F04F8DB004462F
:107FF0000091104604A902220193FFF7AFFE059BF2
:108000001699039303AA01A8F1F7AEFC039D0DB9DD
:10801000FEF7B4FE6268019B049E1E441379126849
:108020000621C2F800151B4A342101FB032302215B
:1080300083F82D1090464FF6FF794FF0010A009B10
:108040008DF81D300023CDE909364D4561680B934D
:108050002F4628BF4F46089708798DF81CA04FF08F
:10806000340C096807AA00FB0C80F1F7C9FE0A4B23
:108070009842834602D1ED1B3E44E0D16068F2F79E
:1080800077F85846F2F72AFC08B1F7F729F90DB04E
:10809000BDE8F08F304D01200000AD0B30B589B048
:1080A00004460D46104605A901220393FFF756FE2C
:1080B000069B0C99049304AA03A8F1F755FC9DF8BC
:1080C00034300093DDE90431039A20460A44A9B212
:1080D000F7F7B6FB08B1F7F703F909B030BD08B5FB
:1080E00003799B0702D50020FFF730FE08BD000092
:1080F00010B50446FFF7F3FF23799B0702D4E0682D
:10810000F1F740F96368054803F00C0343F00103FD
:1081100063600023C4E9023310BD00BF6C54060045
:1081200008B503691830834202D10348FFF70EFEF9
:108130001868196008BD00BFE8B506002DE9F341D5
:108140008B070646019115D10B68124A93420AD15A
:10815000012701ACDFF850800025BD420DD10E484B
:1081600002B0BDE8F0810D4A934203D14F6801F19E
:108170000804EFE70A48FFF7E9FD54F825104145E8
:1081800005D03046F0F7C6FE08B90135E5E70548E9
:10819000E6E700BF2880060064540600EC7F060076
:1081A00090BF060070540600E07C0600820708B508
:1081B00003D10268044B9A4202D00448FFF7C6FD7F
:1081C000BDE80840FFF7BABF2880060050C8060087
:1081D00008B5F0F709FBBDE80840FFF7AFBF0000A6
:1081E00008B5074B0340062B05D0830706D102686C
:1081F000044B9A4202D10448FFF7A8FD08BD00BF16
:10820000070080FF387F060032C7060008B5014826
:10821000FFF79CFD22BD060008B50148FFF796FD5B
:1082200050BD060007B500230DF1030001938DF842
:108230000330F1F7AFF99DF80330EBB101A8F2F785
:108240000FFC18B115491648FEF7A7FADDED017AC3
:10825000FAEECF7AF4EE677AF1EE10FA7DBF17EE00
:10826000903A23F0030040F002000E4878BFA0F1DE
:10827000FF4003B05DF804FB0B4B01221A60D3F8FA
:108280000021002AFBD00022C3F8002103F5A162DF
:10829000D2ED007A01225A60DAE700BFACA90600ED
:1082A000547206006C54060000C00040014608B538
:1082B0000148FEF772FA00BF1872060008B50148BF
:1082C000FFF7F4FF86BB060008B50148FFF7EEFF95
:1082D00026AD060008B50449F0F777FE034B83424C
:1082E00001D1FFF7F1FF08BDE886060030810600E6
:1082F00008B5FFF7EFFF007B400040F0010008BD2C
:1083000008B5FFF7E7FF406908BD000008B5FFF7B3
:10831000E1FF044A90F82800034B002814BF1046E0
:10832000184608BD705406006454060038B505466A
:108330000846F7F701FD04462846FFF7CBFF80F813
:108340002840014838BD00BF6C54060008B5FFF74F
:10835000C1FF806920F0030040F00200A0F1FF405F
:1083600008BD000008B50346042B084608D0052BBD
:1083700008D1FFF7AFFF4068400040F0010008BDA2
:108380000148FCE70020FAE77054060008B50449EC
:10839000F0F71BFE034B834201D1FFF795FF08BDA9
:1083A000C43606003081060008B5FFF7EFFFD0E9BC
:1083B0000423134312D0F3F72FF907EE900A9FED31
:1083C000087AF8EE677AC7EE877A17EE900A20F0FF
:1083D000030040F00200A0F1FF4008BD0020ECE7E0
:1083E00000007A4408B5FFF7D1FFB0F8480040001C
:1083F00040F0010008BD08B5FFF7C8FFB0F84A001B
:10840000400040F0010008BD08B5FFF7BFFF8068DD
:1084100008BD000008B50449F0F7D7FD034B8342BF
:1084200001D1FFF751FF08BDD835060030810600A5
:1084300008B5FFF7EFFF044A90F89500034B0028BA
:1084400014BF1046184608BD705406006454060058
:1084500038B50D46FFF7DEFF04462846F7F76CFCFB
:1084600080F0010384F8950084F89630004838BD08
:108470006C54060038B50D46FFF7CCFF044628467D
:10848000F7F75AFC84F89800004838BD6C54060091
:1084900008B5FFF7BFFF044A90F89800034B002887
:1084A00014BF1046184608BD7054060064540600F8
:1084B00008B5FFF7AFFFB0F84800400040F00100FA
:1084C00008BD08B5FFF7A6FFB0F84A00400040F02D
:1084D000010008BD08B5FFF79DFFB0F84C00400053
:1084E00040F0010008BD08B5FFF794FF806808BDA3
:1084F00008B5FFF78FFFD0F8880007EE900AF5EE79
:10850000C07AF1EE10FA01D5FEF7D0FA20F00300A0
:1085100040F00200A0F1FF4008BD000008B504498A
:10852000F0F753FD034B834201D1FFF7CDFE08BDA9
:10853000883C06003081060008B5FFF7EFFF90F891
:108540005130034813F0010F024B08BF184608BD15
:10855000705406006454060038B50D46FFF7DEFF80
:1085600004462846F7F7E8FB94F8513060F300031F
:1085700084F85130004838BD6C54060008B5FFF748
:10858000CDFFB0F90C00400040F0010008BD08B577
:10859000FFF7C4FFB0F90E00400040F0010008BD35
:1085A00008B5FFF7BBFF90F85030034813F0200FD9
:1085B000024B08BF184608BD7054060064540600FC
:1085C00038B50D46FFF7AAFF04462846F7F7B4FB77
:1085D00094F85030C3F3401282421EBF60F345133B
:1085E00043F0020384F85030004838BD6C54060054
:1085F00008B5FFF793FF90F85030034813F0400F91
:10860000024B08BF184608BD7054060064540600AB
:1086100038B50D46FFF782FF04462846F7F78CFB76
:1086200094F85030C3F3801282421EBF60F3861369
:1086300043F0020384F85030004838BD6C54060003
:1086400008B5FFF76BFF90F850300348DB09034B88
:1086500008BF184608BD00BF7054060064540600E9
:1086600038B50D46FFF75AFF04462846F7F764FB76
:1086700094F85030B0EBD31F0DD060F3C713228AAB
:1086800084F85030638A9A4207D194F8503043F00E
:10869000020384F85030064838BD2046F2F7E4FF64
:1086A000F3F725F894F8503043F00403F1E700BFE6
:1086B0006C54060008B5FFF731FF806808BD000064
:1086C00010B50C46FFF72AFFA30706D12368094A15
:1086D000934205D0084A934202D00848FFF736FB80
:1086E00090F85030846043F0020380F85030044822
:1086F00010BD00BF703A06006434060000A90600F1
:108700006C54060010B504460079FF2813D0F1F729
:1087100035FE2079F5F77EF90A4A0023114652F812
:10872000040B844208D1002241F823202079F2F77B
:10873000F3F8FF23237110BD0133082BEFD1002084
:10874000FFF7B4FD4C44012008B5FFF7DBFF0148FB
:1087500008BD00BF6C54060008B50868FFF7D2FFDB
:10876000004808BD6C54060008B50148FFF79EFD9F
:10877000F0C3060010F0010310B501D0401010BD89
:10878000D0E9022101EB4202914205D30279D207DE
:1087900048BF5B421846F2E7B3F5004F04D232F807
:1087A000024D44EA0343EFE701490248FDF7F5FFB4
:1087B00006AB0600907206000F4A904210B50C46B8
:1087C00003D100230B60012204E00C4A904203D144
:1087D00001220A60104610BD10F0010202D04310C1
:1087E0000B60F7E78107F5D10168054B9942F1D19C
:1087F000FFF7C0FF2060E6E76454060070540600EF
:10880000B47B060010B58AB0044608466946FFF7F7
:10881000D3FF10B90F48FEF777F910238DF80C300D
:10882000009B06930023ADF82430ADF82230079367
:108830008DF8203001938DF80830204601AB06AA50
:1088400003A9F7F707FE0198400040F001000AB0C5
:1088500010BD00BFF2B3060013B50446084601A9D7
:10886000FFF7AAFF08B9FEF7A1FA6268019B044866
:108870000C2101FB032300225A7202B010BD00BF7D
:108880006C54060013B50446084601A9FFF794FF8F
:1088900008B9FEF78BFA6268019B04480C2101FBC2
:1088A000032301225A7202B010BD00BF6C540600AF
:1088B00070B5446803460021A14216D0DA6810461C
:1088C000EFF78AFF4D1CA0B19E6852F82100013ECF
:1088D0009E60B5FBF4F304FB135452F82430002BD4
:1088E00018BF042342F8213028B903490348FDF793
:1088F00054FF2946E0E770BD0EAF06007470060015
:1089000008B502490248FDF748FF00BF60C40600F1
:108910009072060010B50C46014640F2D920F0F7DF
:10892000CEFB20B1012C0CBF436883681BB9024900
:108930000248FDF732FF10BDAAB6060054720600C9
:1089400070B5061D044601213046F6F737F820467B
:10895000A569F5F733FE3046F6F7A0FA48B91DB918
:1089600005490648FDF719FF0120F2F77BF8013DA4
:10897000F1E7002DF4D070BDBCBE0600F873060010
:1089800038B5044604F10C05F5F718FE0021284619
:10899000F6F714F82046F5F711FE2046FFF7D0FF52
:1089A00028460121F6F70AF82046BDE83840F5F7D9
:1089B00005BE38B500F10C05044601212846F5F73F
:1089C000FDFF2046F5F7FAFD2046FFF7B9FF2846E0
:1089D0000021F5F7F3FF2046BDE83840F5F7EEBD7E
:1089E0002DE9F0410446261D8846F5F7E7FD0021F4
:1089F0003046F5F7E3FF072504F10C0748FA05F3C5
:108A000013F0010118BF01213846F5F7D7FF2046C2
:108A1000F5F7D4FD2046FFF793FF00213046F5F728
:108A2000CDFF013DEAD201213846F5F7C7FF2046C8
:108A3000F5F7C4FD2046FFF783FF2046F6F754FA0A
:108A400005462046F5F7BAFD30460021F5F7B6FF9A
:108A500085F00100C0B2BDE8F0812DE9F04387B098
:108A600004460E46104603A9012201939DF83C805E
:108A7000FFF774F9049B0E99029302AA01A8F0F77C
:108A800073FF2046DDE90197039DFFF792FF710018
:108A900001F0FE012046FFF7A3FFD8B14D442F445B
:108AA000AF4205D1B8F1000F0BD107B0BDE8F0839C
:108AB00015F8011B2046FFF793FF0028F0D105258C
:108AC00009E000252046FFF75BFF002DEDD028468A
:108AD000F6F706FC1325B8F1000FF3D1F7E7000015
:108AE0002DE9F04F87B004460D46104603A9022237
:108AF0000193FFF733F9049B1099029302AA01A88E
:108B0000F0F732FF029F0FB9FEF738F92046DDF883
